:1000000000800020BD0100008D6F0000596F0000CE
:10001000596F0000596F0000596F0000596F0000C0
:10002000596F0000596F0000596F00008D6F00007C
:100030008D6F0000596F00008D6F0000496F000048
:100040008D6F00008D6F00008D6F00008D6F0000C0
:100050008D6F00008D6F00008D6F00008D6F0000B0
:100060008D6F00008D6F00008D6F00008D6F0000A0
:100070008D6F00008D6F00008D6F00008D6F000090
:100080008D6F00008D6F00008D6F00008D6F000080
:100090008D6F00008D6F00008D6F00008D6F000070
:1000A0008D6F00008D6F00008D6F00008D6F000060
:1000B0008D6F00008D6F00008D6F00008D6F000050
:1000C0008D6F00008D6F00008D6F00008D6F000040
:1000D0008D6F00008D6F00008D6F00008D6F000030
:1000E0008D6F00008D6F00008D6F00008D6F000020
:1000F0008D6F00000D7800008D6F000001920000F0
:100100008D6F0000AD9600008D6F00008D6F0000B8
:100110008D6F00008D6F00008D6F00008D6F0000EF
:100120008D6F00008D6F00008D6F00008D6F0000DF
:100130008D6F00008D6F00008D6F00008D6F0000CF
:100140008D6F00008D6F00008D6F00008D6F0000BF
:10015000658700007D87000095870000AD8700005F
:10016000F1650000317B00008D6F00008D6F000095
:100170008D6F00008D6F00008D6F00008D6F00008F
:100180008D6F00008D6F00008D6F00008D6F00007F
:100190008D6F00008D6F00008D6F00008D6F00006F
:1001A0008D6F00008D6F00008D6F00008D6F00005F
:1001B0008D6F00008D6F00008D6F0000564B4CF26C
:1001C000205210B51A804DF628121A8000BF00BFC9
:1001D00006F0E0FE514B4FF010621A60504A9A60F0
:1001E000504ADA60A3F53043203B1A6812F480725B
:1001F00004D14D490A604FF4A8521A604B4B1A784B
:10020000110703D51A7842F008021A70484B2A22C7
:100210001A700023474A48499818884204D247492F
:10022000595899500433F5E7454A464B9A424FF0E6
:10023000000302D242F8043BF7E74349434A5958C6
:1002400099500433B3F5DE7FF7D1414B802103F899
:10025000011B40498B42F9D13F4B1A603F4B0A22A8
:100260001A70A3F5805324225A70A0221A709A792A
:100270009207FCD59A79D406FCD4394B9A7902F0CE
:100280000C02082AF9D103221A7140225A719A7974
:100290009006FCD5324B9A795106FBD5314A32494A
:1002A00011600221516020221A702D4B9B7903F0BE
:1002B0000C030C2BF9D12D4B2D4A1A602D4B2E4AD5
:1002C0001A6000225A60072243F8042C2B4AC3F814
:1002D0000C2D62B606F0F8FF134B1B68DA0705D544
:1002E000274806F08DFE274B274A1A60274B1B78BC
:1002F0005B0609D5234C244A2368934204D1204845
:1003000006F07EFE002323600AF0EEFB06F048FEB6
:1003100008F009FBFEE700BF0E20054030800440D6
:10032000823F04000100002B14D0034002D007409C
:1003300000E007406087FF1F7C88FF1FA8FD0000CA
:100340007C88FF1F3498FF1F000000000082FF1F01
:1003500000E400E05FE400E008ED00E0005006404B
:100360000040064044800440000003010480044033
:10037000C010050014E000E0FF760100000020201E
:1003800091E951571CE00340A5C3945A00F007407F
:10039000FFFFFFFFFFFFFFFFFFFFFFFFFFFFFFFF6D
:1003A000FFFFFFFFFFFFFFFFFFFFFFFFFFFFFFFF5D
:1003B000FFFFFFFFFFFFFFFFFFFFFFFFFFFFFFFF4D
:1003C000FFFFFFFFFFFFFFFFFFFFFFFFFFFFFFFF3D
:1003D000FFFFFFFFFFFFFFFFFFFFFFFFFFFFFFFF2D
:1003E000FFFFFFFFFFFFFFFFFFFFFFFFFFFFFFFF1D
:1003F000FFFFFFFFFFFFFFFFFFFFFFFFFFFFFFFF0D
:10040000FFFFFFFFFFFFFFFFFFFFFFFFFEFFFFFFFD
:1004100010B5054C237833B9044B13B10448AFF33E
:1004200000800123237010BD7C88FF1F00000000A6
:10043000A8FD000008B5064B1BB106480649AFF3FE
:1004400000800648036813B1054B03B1984708BD07
:1004500000000000A8FD00008088FF1F7C88FF1FAF
:100460000000000038B5044608460D460AF099FC25
:10047000236802465B6820462946984738BD38B550
:100480000446FFF7EFFF0546204608F085FA2844AA
:1004900038BDFFFF10B5002304460371437180F897
:1004A00054300349142206300AF09AFC204610BD4D
:1004B0001CBA00000079704710B50121044690F87D
:1004C000550006F0ADFD0120207110BD10B50021D2
:1004D000044690F8550006F0A3FD0A2006F0DEFE63
:1004E00000232371012010BD40797047063070470A
:1004F000006D704710B50446006803681B6A984792
:100500002046FFF7E3FF94F85600012106F0A8FD0E
:10051000012194F8560006F083FD2046FFF7CCFF3A
:100520000D20012106F07CFD206803684FF4164180
:100530009B69984740F2EE2006F0B0FE012384F854
:10054000543010BD10B50446006803681B6A984714
:100550002046FFF7BBFF002194F8560006F060FD2F
:100560000A2006F09BFE2046FFF7A6FF0D20002183
:1005700006F056FD206803684FF4E1319B69984707
:10058000002184F8541094F85600BDE8104006F09D
:1005900067BD10B58EB0322201A80C460AF020FCCF
:1005A00000233A2101A88DF835300AF0DBFB014623
:1005B00008B9207003E0204601310AF0EAFB0EB0D2
:1005C00010BD2DE9F84300250746884691460D7079
:1005D0002C462E46386803689B68984738B33868BD
:1005E0000368DB689847C0B20EB945282BD00136A6
:1005F0000D28F6B203D1002308F8043009E009F110
:10060000FF339C42F7D008F804000134E4B200251F
:10061000E0E70A2006F042FE38680368DB68984786
:10062000386803689B6898470028F2D10EE00135CE
:100630000A20EDB206F032FE312DCBD9201C18BFB6
:100640000120BDE8F8833046BDE8F8830120BDE80D
:10065000F883FFFF70B5044625460679FFF74AFF89
:10066000002355F81A0B0E496371FFF708FF204667
:1006700029463222FFF7A5FF38B128460949022250
:100680000AF097FB08B9012300E0002363712046BC
:10069000FFF758FF16B92046FFF718FF607970BDC5
:1006A0002DBA000030BA0000437970B50446F3B1AA
:1006B00090F854600EB9FFF71DFF25460C4955F818
:1006C0001A0BFFF7DCFE322229462046FFF779FF9E
:1006D00020462946FFF75DFFA01D294614220AF097
:1006E0007FFB26B92046BDE87040FFF72BBF70BDE9
:1006F00033BA0000437970B50446EBB190F854600A
:100700000EB9FFF7F7FE25460C4955F81A0BFFF70F
:10071000B6FE322229462046FFF753FF20462946DF
:10072000FFF737FF28460AF0B6F9206526B92046BC
:10073000BDE87040FFF706BF70BD00BF3CBA0000C7
:100740007FB501600446324800F0F9F9032848D12A
:100750002123182084F85530172384F8563084F864
:100760005700012106F07CFC2A4E94F8573056F8C9
:100770003330012583F8805094F85600294606F05E
:100780006FFC94F8563056F8333083F8005194F8E3
:100790005500294606F064FC94F8553056F833307D
:1007A0000D2083F88050294606F05AFC2046FFF7BA
:1007B00051FF63792BB32046FFF79CFE2046FFF7DD
:1007C00099FF2046FFF770FF2046FFF7BBFE20464B
:1007D000FFF772FE206803684FF4E1319B69984788
:1007E0000FE00D49684608F099F9684603F038FEB5
:1007F000684608F053F9064800F0A1F903F06EFED0
:1008000004E094F85600002106F02AFC04B070BD04
:10081000D088FF1FF0F8000045BA0000F8B5437912
:1008200004460F4643B390F854600EB9FFF762FEDA
:1008300025463A461149206808F0C4F855F81A0BC5
:100840000F49FFF70FFE204629463222FFF7B9FE77
:1008500060B128460B4902220AF0ABFA30B9A01D5C
:10086000394614220AF0BCFA012500E0002516B929
:100870002046FFF767FE2B461846F8BD95BA0000E4
:10088000A0BA000030BA0000F8B5437904460F461C
:1008900023B390F854600EB9FFF72CFE25463A4674
:1008A0000F49206808F08EF855F81A0B0D49FFF72C
:1008B000D9FD204629463222FFF783FE40B1284663
:1008C000094902220AF075FA10B92765012500E0EE
:1008D000002516B92046FFF735FE2B461846F8BD11
:1008E000A3BA0000A0BA000030BA0000F8B54379FE
:1008F00004460F4600F11A050BB9837615E090F80F
:1009000054600EB9FFF7F6FD39462068FFF7AAFDDF
:1009100007492068FFF7A6FD204629463222FFF747
:1009200050FE16B92046FFF70DFE2846F8BD00BF61
:10093000A0BA00001FB500230446C3600361012173
:100940004FF4BF700AF0B0F8206050B90A49684609
:1009500008F0E4F8684603F093FD684608F09EF856
:1009600007E04FF4BF7004210AF09EF8034B60606B
:10097000A360204604B010BDB0BA00000F03010010
:100980000A23034AB1FBF3F1B2FBF1F38360704732
:1009900080DBC41610B5044600680AF0D3F860681E
:1009A0000AF0D0F8204610BD0268036970B5D15432
:1009B00004460669456806F053FC236945F826009D
:1009C0005A1CB2F5BF7FA5BF6FF4BE729B1822619F
:1009D000236170BDC26803699A42CABFC2F5BF7283
:1009E000C2EB0300D018704730B585B00C46054601
:1009F000FFF7F0FF84420EDB0C49684608F08EF8E2
:100A0000684603F02DFD684608F048F8204603F0DC
:100A100065FD002008E0E9682B682144B1F5BF7F3F
:100A2000A8BFA1F5BF71585C05B030BDBEBA0000CB
:100A300030B585B00C460546FFF7CCFF84420EDB8F
:100A40000D49684608F06AF8684603F009FD6846F3
:100A500008F024F8204603F041FD002009E0E96891
:100A60006B682144B1F5BF7FA8BFA1F5BF7153F8F2
:100A7000210005B030BD00BFF3BA0000C3680069B3
:100A80005A1E48BF03F27D12131A5842584170474C
:100A900030B585B00D460446FFF79CFF85420DDD5D
:100AA0000B49684608F03AF8684603F0D9FC6846F6
:100AB00007F0F4FF284603F011FD07E0E3681D444A
:100AC000B5F5BF7FA8BFA5F5BF75E56005B030BD22
:100AD0004EBB000038B5044606F0C2FBA368C51A39
:100AE0002046FFF777FF00280ADDE268636853F8C5
:100AF0002230AB4204D820460121FFF7C9FFEFE7BF
:100B000038BD10B5044640690AF01CF8204610BDF7
:100B100000787047042005F011B940687047007AEA
:100B200070474B000172C360052005F007B9C0682B
:100B30007047007C70470174062005F0FFB880699B
:100B40007047002005F026B9007F7047022005F0AD
:100B5000F5B8407F7047417703200A2105F0EEB8D1
:100B6000807F7047642005F0E9B8C07F704765203A
:100B700005F0E4B890F820007047662005F0DEB874
:100B800090F821007047FFFF436A044A9B10EE3B38
:100B900023EAE37352F82300704700BFD0BB000084
:100BA00090F828007047007FC0F340007047007F36
:100BB000C0F380007047026BC36AD01A20EAE0706D
:100BC0007047026C836BD01A0028B8BF4042704750
:100BD000426CC36BD01A0028B8BF4042704790F8EF
:100BE0004C00704790F84C0040F6FF7340F2FF3223
:100BF00000280CBF104618467047806C704781640F
:100C0000704705299ABF4369585C00207047052941
:100C10009DBF436901205A5400207047052005F00C
:100C20003DB810B5044690F8210006F051F8636A0B
:100C300003EBC30318440A2290FBF2F3636210BD76
:100C400010B5044690F8340006F068FEA36B03EB81
:100C5000C3030A22034493FBF2F3A363236C40F221
:100C6000E73202FB03034FF47A7293FBF2F323643F
:100C700010BD10B5044690F8350006F04FFEE36B4A
:100C800003EBC3030A22034493FBF2F3E363636CB5
:100C900040F2E73202FB03034FF47A7293FBF2F364
:100CA000636410BD38B5044690F82A000D4606F07E
:100CB0000FF8820040F22713104445B1E16A4FF467
:100CC000967503FB010393FBF5F3E36238BD216BDB
:100CD0004FF4967503FB010393FBF5F3236338BDD3
:100CE000064B90F82900012253F8303011B183F8F7
:100CF0008020704783F80021704700BFF0F80000A3
:100D00000078FB280CD0FC2803D0FA2803D1054832
:100D1000704705487047054B0130B3FBF0F0704752
:100D20000348704710552200C0C62D0080841E0065
:100D3000A02526001FB50446032004F0A3FF0A28BF
:100D4000607710D0082803D80520002104F0A6FF02
:100D5000637F092B03D820460021FFF7E2FE2046DF
:100D60000A21FFF7F8FE002004F092FFA0610220A4
:100D700004F088FF2077062004F084FF207404200C
:100D800004F080FF20702046FFF7BAFF6060052066
:100D900004F078FF20724000E060642004F072FFED
:100DA000A077652004F06EFFE077662004F06AFF0C
:100DB00084F82000052004F041FF003018BF012016
:100DC00084F84C000121062009F06EFE606150B9E4
:100DD0002C49684607F0A2FE684603F051FB6846BE
:100DE00007F05CFE4BE0A369012B06D1282384F8B1
:100DF0002130182384F828302EE09A1E012A2BD89F
:100E00001D2284F82120032B4FF0020284F82820B1
:100E100022D1237F9A070ED51220252384F829009A
:100E200084F82A30012106F01BF994F82A0005F015
:100E30004FFFE0622063237F5B070DD50F2319204E
:100E400084F8353084F8340006F068FDA06394F827
:100E5000350006F063FDE06394F8210005F038FFEB
:100E6000606294F8340006F059FDA063206494F8A1
:100E7000350006F053FD0023E0636064A364204660
:100E800004B010BDC1BB000010B501210446FFF73E
:100E900041FE2046FA21FFF744FE20460221BDE82C
:100EA0001040FFF748BEFFFF8369032B10B525D123
:100EB000037F03F0080303F0FF0003B3104802F0C0
:100EC00067FF104802F064FF0F4802F061FF0F480F
:100ED00002F05EFF642006F0E1F901211F2006F018
:100EE000BFF80B4B01241C604FF4FA6006F0D6F9F2
:100EF0001F20002106F0B4F8204610BD002010BDD0
:100F00003889FF1FFC89FF1FC08AFF1F848BFF1FCA
:100F100004F10F40044B80221A701A781206FCD498
:100F2000024B034A1A6070470C2107400CED00E0A9
:100F30000400FA0508B503681B68984708BD08B5A2
:100F4000FFF790FA08BD0A22002307F048BD07F01A
:100F50007EBD38B50446FFF7EDFF0546204607F095
:100F60001BFD284438BD38B50446FFF7ECFF0546A5
:100F7000204607F011FD284438BD38B5044607F077
:100F800066FD0546204607F007FD284438BDF8B544
:100F9000061D0446154630460F46FFF7CBFC30468B
:100FA0002946FFF7EDFC276025642046F8BDFFFFCA
:100FB00038B504469A490068FFF761FA99492068F4
:100FC000FFF7BDFF9848256802F0ACFC01462846B3
:100FD000FFF7B9FF944802F0BDFC10B120689349B7
:100FE00001E020689249FFF7AAFF8F48256802F0C8
:100FF000A2FC90490246284607F0E4FC8E4920688E
:10100000FFF79DFF8D48256802F08CFC01462846BD
:10101000FFF799FF894802F09DFC10B120688349D1
:1010200001E020688249FFF78AFF8448256802F0C2
:1010300082FC80490246284607F0C4FC80492068AB
:10104000FFF77DFF7F48256802F06CFC01462846CB
:10105000FFF779FF7B4802F07DFC10B120687349EF
:1010600001E020687249FFF76AFF7648256802F0C0
:1010700062FC70490246284607F0A4FC72492068C9
:10108000FFF75DFF7148256802F04CFC01462846D9
:10109000FFF759FF6D4802F05DFC10B1206863490D
:1010A00001E020686249FFF74AFF6848256802F0BE
:1010B00042FC60490246284607F084FC64492068E7
:1010C000FFF73DFF634B20681968FFF756FF624941
:1010D0002068FFF734FF61492068FFF730FF604860
:1010E0002568FFF71AFD0A2200230146284607F06B
:1010F00076FC284607F050FC5A492068FFF71FFF8E
:1011000057482568FFF70BFD01462846FFF71BFFF0
:1011100055492068FFF713FF51482568FFF707FD81
:101120000A2200230146284607F059FC4F4920684F
:10113000FFF7A5F94E492068FFF701FF48482568E9
:10114000FFF7F7FC01462846FFF70DFF49492068E5
:10115000FFF7F5FE48492068FFF7F1FE4048256893
:10116000FFF7EDFC01462846FFF707FF43492068DB
:10117000FFF7E5FE3A482568FFF7E6FC01462846FA
:10118000FFF7F1FE3E492068FFF7D9FE3448256895
:10119000FFF7E6FC102201460023284607F01FFC5B
:1011A0002F482568FFF7E1FC10220146002328465E
:1011B00007F015FC2A482568FFF7DCFC1022002305
:1011C0000146284607F00BFC284607F0E5FB2D49B1
:1011D0002068FFF7B4FE22482568FFF7BAFC0146F5
:1011E0002846FFF7C0FE28492068FFF7A8FE1C48E4
:1011F0002568FFF7F7FC01462846FFF7A8FE2068A0
:101200002249FFF73CF92248FFF76EF910B1206838
:10121000204901E020682049FFF731F938BD00BFBF
:10122000E0C7000011C800003889FF1F3BC800005C
:10123000CCE6000065C8000078C80000FC89FF1FEC
:101240009BC80000C08AFF1FBEC80000848BFF1F20
:10125000E1C80000F094FF1F04C9000033C900007A
:10126000D088FF1F45C900005AC900005DC90000B1
:1012700069C9000080C900009DC90000B0C9000014
:10128000C8C90000D5C90000E9C900000CCA0000A7
:101290009894FF1F1DCA00006CCA000070B5394D3C
:1012A000394904460068FFF74AFE28462668FFF7DA
:1012B00050FC01463046FFF746FE20683349FFF7F1
:1012C000DEF820683249FFF7DAF820683149FFF785
:1012D000D6F820683049FFF7D2F820682F49FFF789
:1012E000CEF820682E49FFF7CAF820682D49FFF78D
:1012F000C6F820682C49FFF7C2F820682B49FFF791
:10130000BEF820682A49FFF7BAF820682949FFF794
:10131000B6F820682849FFF7B2F820682749FFF798
:10132000AEF820682649FFF7AAF820682549FFF79C
:10133000A6F820682449FFF7A2F820682349FFF7A0
:101340009EF820682249FFF79AF820682149FFF7A4
:1013500096F820682049FFF792F820681F49FFF7A8
:101360008EF81F492068FFF7EAFD28462668FFF738
:1013700039FC01463046FFF7EAFD20681949FFF7BE
:101380007EF870BDD088FF1FBBCA000063C8000094
:1013900040D00000E3CA0000F7CA00002ACB0000DA
:1013A00047CB000065CB00009FCB00000ACC0000BB
:1013B0003FCC000070CC0000FDCC000057CD0000F9
:1013C000B2CD00003FCE00008CCE0000D9CE000090
:1013D00013CF00004FCF000087CF0000DACF00000E
:1013E000EAC900000CCA000070B53D4D3D490446F5
:1013F0000068FFF7A4FD28462668FFF7AAFB014610
:101400003046FFF7A0FD20683749FFF738F820681D
:101410003649FFF734F820683549FFF730F820687F
:101420003449FFF72CF820683349FFF728F8206883
:101430003249FFF724F820683149FFF720F8206887
:101440003049FFF71CF820682F49FFF718F820688B
:101450002E49FFF714F820682D49FFF710F820688F
:101460002C49FFF70CF820682B49FFF708F8206893
:101470002A49FFF704F820682949FFF700F8206897
:101480002849FEF7FCFF20682749FEF7F8FF20688F
:101490002649FEF7F4FF20682549FEF7F0FF206893
:1014A0002449FEF7ECFF20682349FEF7E8FF206897
:1014B0002249FEF7E4FF22492068FFF740FD284655
:1014C0002668FFF78FFB01463046FFF740FD206896
:1014D0001C49FEF7D4FF20681B49FEF7D0FF70BD02
:1014E000D088FF1FBBCA000063C800002CD00000DA
:1014F00052D00000DDD00000FFD0000044D1000039
:101500007ED10000BCD10000EFD1000018D2000055
:101510006FD20000BCD200003AD3000070D30000AC
:10152000C6D30000F2D3000034D400006CD4000015
:10153000A5D40000D9D4000016D5000068D500005D
:10154000E9C900000CCA0000D2D50000F8B50E1E93
:101550000446154640F3DD80022E03DD032E00F025
:101560008880D6E0B2F5FA6F006801D97C49D2E0F4
:101570007C49FFF7E4FC29462068FFF7E8FC7A493C
:101580002068FEF77CFF794802F09DFB784802F066
:101590009AFB764802F0D4FC754802F0D1FC7348FF
:1015A000002102F077FA7248002102F073FA4FF43A
:1015B0007A7005F073FE33276D4802F008FF0028AB
:1015C00040F0AC80694802F002FF002840F0A6809D
:1015D0002946664802F082FC0121644802F078FC4A
:1015E0006448FFF7FFFA0146604802F053FA2946C3
:1015F0005F4802F073FC01215D4802F069FC5D4820
:10160000FFF7F0FA01465A4802F044FA4FF47A70B4
:1016100005F044FE3325564802F0D9FE002840F07C
:101620008880524802F0D3FE002840F08280504863
:10163000002102F04DFC4D48002102F049FC012E32
:10164000206814D14C49FEF71AFF4FF4FA6005F0F8
:1016500025FE20684949FEF712FF4448002102F0A8
:1016600019FA43480021BDE8F84002F013BA444992
:1016700051E0531EB3F5FA6F006801D341494AE0C7
:101680004149FFF75CFC29462068FFF760FC3649BA
:101690002068FEF7F4FE354802F015FB344802F0EE
:1016A00012FB324802F04CFC314802F049FC2F4852
:1016B000002102F0EFF92E48002102F0EBF94FF47F
:1016C0007A7005F0EBFD3326294802F080FE0028F1
:1016D0003AD1264802F07BFE002835D1234829461E
:1016E00002F0FCFB2248294602F0F8FB1F480221C9
:1016F00002F0EEFB02211E4802F0EAFB4FF47A7082
:1017000005F0CCFD21492068FEF7B9FE206820498C
:1017100001E020681F49FEF7B2FEF8BD013F04D189
:1017200020681D49FEF7ABFE52E7C82005F0B6FD64
:1017300042E7013D04D120681749FEF7A0FE76E795
:10174000C82005F0ABFD66E7013E04D120681249D0
:10175000FEF795FEC2E7C82005F0A0FDB4E700BF84
:1017600001D6000035D600006AD60000C08AFF1FEF
:10177000848BFF1FD088FF1FA9D60000CDD60000A4
:10178000DFD60000F1D6000025D700007CD700008E
:10179000C5D70000EFD7000078D6000070B504462A
:1017A00016490068164E174DFEF769FE2068164967
:1017B000FFF7C5FB154B2068197800290CBF31468F
:1017C0002946FEF75CFE20681149FFF7B8FB114B74
:1017D0002068197800290CBF31462946FEF74FFED4
:1017E00020680D49FFF7ABFB0C4B206819780029E6
:1017F0000CBF31462946FEF742FE70BD72D800008C
:1018000036D800002ED8000099D800002089FF1F8C
:10181000B5D800002189FF1FC9D80000A488FF1F88
:10182000F8B504460E4600684749FFF788FB711C6F
:101830002068FFF7A2FB45492068FFF780FB444B77
:101840002768C42505FB0635284602F0CDFD014674
:101850003846FFF788FB3F492068FFF770FB2846B2
:10186000266802F0E3FD01463046FFF77CFB3A496B
:101870002068FFF764FB2846266802F0DEFD01467B
:101880003046FFF770FB2846266802F048F8334BD5
:101890003349002818BF19463046FEF7F0FD31499C
:1018A0002068FFF74CFB30482668FFF769F90146CE
:1018B0003046FFF758FB2D492068FFF740FB2846CC
:1018C000266802F08DFD01463046FFF756FB284999
:1018D0002068FFF734FB2846266802F083FD0146A6
:1018E0003046FFF74AFB23492068FFF728FB2846CC
:1018F000266802F097FD01463046FFF73EFB1E4981
:101900002068FFF71CFB2846266802F08DFD014683
:101910003046FFF732FB284602F01CF810B1206871
:10192000164901E020681649FFF709FB15492068B0
:10193000FFF705FB2846246801F0FBFF014620461F
:10194000FFF71BFBF8BD00BFDED9000011DA000075
:101950003889FF1F1CDA000027DA0000DED80000FB
:1019600066D9000036DA0000D088FF1F64DA000074
:1019700070DA00007BDA000087DA00003BC8000064
:10198000CCE6000092DA000070B50E4604464249EB
:1019900000681546FEF773FD052E74D8DFE806F0E3
:1019A000030A14263B5B3D492068FEF768FD20686A
:1019B0003B496EE03B48FFF767FA3B492068FEF77A
:1019C0005EFD2068394964E039492068FEF757FD1B
:1019D00038492068FEF753FD37492068FEF74FFD70
:1019E00020683649FEF74BFD012010E030492068A1
:1019F000FEF745FD32492068FEF741FD2E4920687B
:101A0000FEF73DFD20682D49FEF739FD0020BDE8B9
:101A1000704004F0EBB92B492068FEF730FD2A49ED
:101A20002068FEF72CFD29492068FEF728FDEDB25D
:101A300027492068FFF783FA29462068FFF793FAC1
:101A400029461848FFF766F822492068FEF717FD77
:101A5000206821491DE020682049FEF710FD20681C
:101A60000DB91F4902E0012D07D11E49FEF707FD00
:101A70000C482946FFF7D2F802E01B49FEF7FFFCAD
:101A800020681A4905E01A492068FEF7F8FC20682A
:101A90001849FEF7F4FC70BDA9DA0000CBDA0000AB
:101AA00028DB0000D088FF1F5CDB0000ADDB0000FE
:101AB0001DDC000067DC0000CBDC00007FDD0000E7
:101AC000ECDD000051DE000083DE00000CDF0000D2
:101AD000BFDF0000E7DF000039E00000B0E00000F9
:101AE000E2E000004FE10000B5E1000007E2000085
:101AF00051E2000065E2000070B50E4686B0044673
:101B0000644900681546FEF7BAFC072E00F2AF8064
:101B1000DFE806F004071223384D627720685E493B
:101B2000ABE020685D49FEF7AAFC5D492068FEF73E
:101B3000A6FC04F086F9A2E020685A49FEF79FFC53
:101B400020685949FFF7FBF929462068FFF715FA85
:101B500029465648FEF7F5FF91E020685449FEF704
:101B60008EFCFF2D206801DD52498EE05249FFF7BF
:101B7000E6F929462068FFF700FAE9B24B48FEF77C
:101B8000E5FF7CE020684D49FEF779FC642D206874
:101B900001DD4B4979E04B49FFF7D1F9294620682F
:101BA000FFF7EBF9E9B24148FEF7DCFF67E0206898
:101BB0004549FEF764FC0C2D206801DD434964E0D3
:101BC0004349FFF7BCF929462068FFF7D6F9E9B287
:101BD0003648FEF7CCFF52E020683E49FEF74FFC46
:101BE000FF2D206801DD3C494FE03C49FFF7A7F994
:101BF00029462068FFF7C1F9E9B22C48FEF7BDFF7E
:101C00003DE037492068FEF73AFC2848FEF7A8FF78
:101C100006462648FEF7A9FF05462448FEF7AAFF18
:101C200032462B4600902F4903A809F077F82E4939
:101C30002068FFF784F903A92068FFF780F92B4893
:101C400003A9FEF7EBFD10B12068294901E02068E7
:101C50002849FEF714FC28492068FFF770F9274946
:101C600022482568FEF742FE0146284605E0244941
:101C70002068FEF704FC20682249FEF700FC224998
:101C80002068FEF7FCFB20682049FEF7F8FB06B051
:101C900070BD00BF87E20000A2E20000D6E20000B3
:101CA00013E3000093E30000B1E30000D088FF1FBE
:101CB000CFE30000F1E3000021E4000043E4000072
:101CC00061E400009AE40000BFE40000DEE40000EC
:101CD00022E5000048E5000085E50000ABE50000D6
:101CE000D3E5000009E6000015E600009894FF1F08
:101CF00035E600003FE600007AE60000CDE6000091
:101D000051E20000E0E6000002E700003CE70000CE
:101D1000032938B504460D46006801D911491EE073
:101D20001149FFF70CF9691C2068FFF726F90F49E4
:101D30002068FEF7A4FB0E492068FEF7A0FB0D4BC0
:101D4000C42202FB0535284602F05AFA284602F062
:101D500013F909492068FEF792FB20680749FEF74E
:101D60008EFB38BDDEE70000F6E7000014E8000057
:101D70008EE800003889FF1FDFE800000FE900004F
:101D8000032970B504460D46006801D919492DE0B4
:101D90001949FFF7D4F8691C2068FFF7EEF81749D6
:101DA0002068FEF76CFB16492068FEF768FB154BB0
:101DB000C42606FB05363046002101F06BFE4FF4C9
:101DC000FA6005F06BFA00252946304601F062FE04
:101DD000304601F0B9FE4FF4FA7005F05FFA0735AE
:101DE00040F205439D42EFD120680749FEF747FBCB
:101DF00070BD00BFDEE7000049E9000014E8000004
:101E00007AE900003889FF1FC5E9000038B51B4991
:101E100004460068FEF733FB1948FEF765FB38B34C
:101E200020681849FEF72BFB17492068FFF787F851
:101E300013482568FEF75AFB01462846FEF71FFBAC
:101E40000F482568FEF754FB10490246284606F065
:101E5000B9FD0F492068FFF772F809482468FEF7BA
:101E600029FB0C4B0C49002818BF1946204601E0FD
:101E700020680A49FEF703FB38BD00BFDCE900001B
:101E80009894FF1FFAE9000015EA000027EA000015
:101E90003DEA0000D5E90000D8E900004DEA000065
:101EA00038B504460D4600681449FEF7E8FA1448B0
:101EB000FEF71AFB10B92068124907E0284608F01F
:101EC00070FF01381328206803D90F49FEF7D7FAAD
:101ED00038BD0E49FFF733F829462068FEF7CFFAE0
:101EE00007482946FEF79AFC10B12068084901E02E
:101EF00020680849FFF723F838BD00BF79EA0000E1
:101F00009894FF1FA1EA0000C8EA000016EB000049
:101F100041EB00005DEB000038B504460D4600685B
:101F20001449FEF7ACFA1448FEF7DEFA10B920683F
:101F3000124906E0284608F034FF042804D020683F
:101F40000F49FEF79CFA38BD284608F0A4FD054667
:101F50000C4920682A4606F035FD07482946FEF759
:101F600093FC10B12068084901E020680749FEF79A
:101F7000E6FF38BD9DEB00009894FF1FA1EA00002A
:101F8000C3EB0000FBEB000029EC00004DEC00006F
:101F900038B504460D4600681049FEF770FA20680F
:101FA0000F49FEF76CFA0F48FEF79EFA10B9206849
:101FB0000D4910E02B781BB920680C49FEF75FFA39
:101FC00020680B49FEF7BBFF294606482468FEF748
:101FD0008DFC01462046FEF752FA38BD95EC000014
:101FE000BBEC00009894FF1FA1EA00001CED00006C
:101FF0003AED000070B504460E4600681D491546CE
:10200000FEF73DFA20681C49FEF739FA6B1E632B78
:10201000206801D9194924E02B461949721C06F0A1
:10202000D1FC18492068FEF72AFA174BC42000FBA0
:102030000630E9B202F00AF9B0B114492068FEF79F
:102040001EFA13492068FEF71AFA642005F026F9F3
:102050001048FEF729FF10B120680F4901E0206801
:102060000E49FEF70CFA70BD20680D49FEF767FFB8
:1020700070BD00BF55ED000069ED00009FED000050
:10208000DDED00000BEE00003889FF1FF9EE0000C7
:10209000B2F00000D088FF1F0BEF000038EF000007
:1020A00009F000002DE9F0419846ADF5087D1D4B83
:1020B0008E9E15460446C4200F46002200FB0530C4
:1020C0008DF80C218DF81C2201F02CFC192F8DF8B5
:1020D000056005BF3612032302238DF80660042D28
:1020E0008DF802008DF801508DF804808DF80331D1
:1020F000684644A902D103F0C5FB01E003F010F9E2
:1021000020685B21FEF716FF9DF815122068FEF788
:102110001AFF20685D21FEF71CFF0DF5087DBDE864
:10212000F08100BF3889FF1FF0B51F46274BADF582
:10213000097D15460446C420002200FB05300E46EA
:102140008DF80C218DF81C2201F0ECFB02231B2ED4
:102150008DF8033118BF0123042D8DF802008DF88E
:1021600001508DF804708DF80530684644A902D1FD
:1021700002F064FD01E002F0C7F920685B21FEF780
:10218000D9FE9DF815122068FEF7DDFE20685D215E
:10219000FEF7D0FE20680921FEF7CCFE1B2E08BFFB
:1021A0009DF815319DF81451206808BF05EB0325F3
:1021B0005B21FEF7BFFE29462068FEF7C8FE2068B7
:1021C0005D21FEF7C6FE0DF5097DF0BD3889FF1FC4
:1021D00010B504460C490068FEF751F90B49206818
:1021E000FEF7ADFE20680A49FEF7A9FE0948FEF792
:1021F0005BFE20B10748BDE81040FEF78BBE2068AB
:102200000549FEF73CF910BD96F000004CEE0000C9
:10221000B1F00000D088FF1FC0F0000038B5051DE8
:102220002846FEF7D7FB032801DC002038BD002438
:102230002846FEF7CFFB8442F7DC28462146FEF70E
:10224000D3FB0A2807D028462146FEF7CDFB0D28F0
:1022500001D00134ECE7012038BDFFFF2DE9F04F3C
:10226000061D89B030460C4691469A46FEF7B2FBF1
:10227000032840F38C8100213046FEF7B5FB014670
:10228000684606F0BBFC01213046FEF7ADFB014677
:10229000684606F0D6FC02213046FEF7A5FB014653
:1022A000684606F0CEFC684606F00FFD6846002141
:1022B00006F0F1FC6228304630D1FEF78BFB4FF080
:1022C000000B80465F460BF10405454505DB149B7A
:1022D0009B4518D10BF1FF3B15E0149A9345F6DAB4
:1022E00030462946FEF780FB0D280CD00A280AD07C
:1022F000202801D127B106E0139A02F80B0001272C
:102300000BF1010BDFE7139A002302F80B30129A4E
:10231000C9F80030CAF8003013605FE0FEF75AFBDE
:10232000052853DD0421032008F0BEFB0746304694
:10233000FEF750FB4FF00008834603253046294640
:10234000FEF752FB0D2834D00A2832D030462946F9
:10235000FEF74AFB202840F01C815D45C0F21E813B
:1023600017E130462946FEF73FFB392814D85D4572
:1023700012DA29463046FEF737FB0D2801460BD00E
:102380000A2909D004A806F05CFC0135304629462C
:10239000FEF72AFB2F28E4D804A806F0A4FC47F88F
:1023A000080004A808F1040806F078FBB8F10C0F47
:1023B000C4D13B68C9F80030129A7B68CAF8003073
:1023C000BB681360384608F0BDFB07E0129A002393
:1023D000C9F800300325CAF8003013603046FEF714
:1023E000F9FAA84206DD30462946FEF7FDFA0D2827
:1023F00000F0D6803046FEF7EDFAA84206DD304602
:102400002946FEF7F1FA0A2800F0CC80304629462A
:10241000FEF73EFB6846664906F021FC08B1012341
:1024200005E06846634906F01AFC10B102232370E8
:10243000A8E06846604906F012FC08B10323F6E7FD
:1024400068465E4906F00BFC08B10523EFE76846D5
:102450005B4906F004FC08B10423E8E768465949E3
:1024600006F0FDFB08B10623E1E76846564906F091
:10247000F6FB08B10723DAE76846544906F0EFFB9C
:1024800008B10823D3E76846514906F0E8FB08B1D4
:102490000923CCE768464F4906F0E1FB08B10A235F
:1024A000C5E768464C4906F0DAFB08B10B23BEE7E6
:1024B00068464A4906F0D3FB08B10C23B7E76846E3
:1024C000474906F0CCFB08B10D23B0E76846454903
:1024D00006F0C5FB08B10E23A9E76846424906F09D
:1024E000BEFB08B11023A2E76846404906F0B7FBDF
:1024F00008B111239BE768463D4906F0B0FB08B1DF
:10250000122394E768463B4906F0A9FB08B1132360
:102510008DE76846384906F0A2FB08B1142386E728
:102520006846364906F09BFB08B115237FE76846ED
:10253000334906F094FB08B1162378E76846314921
:1025400006F08DFB08B1172371E768462E4906F0A7
:1025500086FB08B11A236AE768462C4906F07FFB20
:1025600008B11B2363E76846294906F078FB08B1E8
:1025700018235CE76846274906F071FB08B1192368
:1025800055E720706846EDB206F088FA0CE00025A9
:102590000AE004A8002106F0C1FAF7E60135D5E605
:1025A000013527E7013531E7284609B0BDE8F08F4E
:1025B00092F1000096F100009AF100009EF10000F7
:1025C000A2F10000A6F10000AAF10000AEF10000A7
:1025D000B2F10000B6F10000BAF10000BEF1000057
:1025E000C2F10000C6F10000CAF10000CEF1000007
:1025F000D2F10000D6F10000DAF10000DEF10000B7
:10260000E2F10000E6F10000EAF10000EEF1000066
:10261000F2F10000F6F100002DE9F04104460068F7
:10262000036888B09B68984720B92046FFF7F6FDFD
:10263000C0B906E2251D2846FEF74CFA206803685B
:102640009B6898470028F0D02846FEF717FA002824
:10265000EBD120680368DB689847C1B22846FEF7D3
:10266000A3F9EBE707AB04F118058DE82800282350
:1026700002930DF11301204605AA06ABFFF7EEFD0C
:102680009DF813101B2900F2C581DFE811F01C0032
:102690001F0025007600D600AC000501A800280028
:1026A00009010D01110119011F0125012D0135013C
:1026B00039013E01430148018501A001A901B7018B
:1026C000B701AD01AD0120689F49B7E120460599EA
:1026D000069AFEF73BFFA8E720689C49AEE1059B00
:1026E0009B4920689B4D013B0593FEF728FC05990B
:1026F0002068FEF742FC98492068FDF7C0FE059867
:10270000C42606FB005001F0DEFA059806FB0050D7
:1027100001F016FC059806FB00569048FEF762FA99
:10272000022190FBF1F1304601F0B4F93C27A846B4
:10273000059BC42000FB038001F0DAFB0646B0B124
:10274000B6F5805F206807DB8549FEF7F8FB256852
:10275000A6F6FF71284605E08249FEF7F0FB2568E2
:102760003146284606F073F9284606F015F9FA2096
:1027700004F094FD013FDBD12EE0059B7A492068EF
:10278000744E013B0593FEF7DAFB05992068FEF7CE
:10279000F4FB76492068FDF772FE059BC42000FB20
:1027A000036001F0F5FA3C25374671492068FEF7D1
:1027B000C6FB059B2668C42000FB037001F04AF9A4
:1027C0000146304606F043F9304606F0E5F8FA20B7
:1027D00004F064FD013DE8D1206866492EE1204601
:1027E000FEF7E6FB21E7059B013B032B04D920689C
:1027F0006149FEF7A4FB18E7206860490593FEF7DE
:102800009EFB05992068534DFEF7B7FB0598C4263B
:1028100006FB005001F0BCFA059806FB005001F0E1
:102820008FFB0598002106FB005001F051FB059835
:1028300006FB005001F082F8F7E6059B4748069D2D
:10284000013B0593FEF7CEF9854200F3E980069B34
:10285000002BC0F2E5804A4920683E4DFEF76FFB31
:10286000059920680131FEF772FB46492068FEF7A2
:1028700066FB06992068FEF76AFB43492068FDF76E
:10288000FEFD0598C42606FB005001F01CFA0598D1
:10289000069906FB0050C0E02046FEF7FFFCC4E6A8
:1028A0002046FEF7A1FDC0E62046FEF777FFBCE616
:1028B0000599013905912046C9B2FEF7B1FFB4E68A
:1028C00020460599069AFFF75FF8AEE6204605997F
:1028D000069AFFF711F9A8E60599013905912046F6
:1028E000C9B2FFF715FAA0E605990139059120460E
:1028F000C9B2FFF745FA98E62046FFF787FA94E653
:1029000020462946FFF7CCFA8FE620462946FFF7F6
:1029100003FB8AE620462946FFF73AFB85E61B497A
:102920002068FDF7ACFD18492068FDF7A8FD1848A0
:1029300001F0C9F90021164801F0ACF8154801F082
:10294000C2F91448002168E0FAF100004BF20000DF
:102950008AF200003889FF1FBEF20000D088FF1FF6
:102960003FF300004AF3000055F300008DF3000030
:10297000DCF3000039E60000EEF3000000F4000094
:102980001AF500002CF500005CF400004DF4000086
:10299000848BFF1FC08AFF1F2B492068FDF76FFD46
:1029A0002A492068FDF76BFD294801F08CF9294878
:1029B000FEF718F90146264801F06CF8264801F0A8
:1029C00082F92448FEF70EF90146234825E00599CF
:1029D000069A013905912046C9B2FFF70BFB24E6A0
:1029E0002046FFF7F5FB20E6059A9DF81830013ADE
:1029F00005922046D2B2FFF797FB16E6059A079894
:102A00000090013A05929DF818302046D2B2FFF7A7
:102A100049FB0AE62068114910E001F03BF804E6A2
:102A20000F492068FEF78BFA0A482568FEF7DAF8A6
:102A300001462846FEF78BFA20680A49FDF71FFD7C
:102A4000F3E508B0BDE8F081B4F400005CF40000E8
:102A5000848BFF1FD088FF1FC08AFF1FC3F40000B4
:102A60003AF50000FFD50000F8B505460E460024F3
:102A70000D4BC42000FB043000F054FF8542E7B248
:102A800001D137700BE00134042CF1D1074B1B68E6
:102A90009D4201D1347002E0FE2D02D1357001203B
:102AA000F8BD0020F8BD00BF3889FF1FF094FF1F5C
:102AB00030B5044685B0FDF73DFF04F5987304F585
:102AC000D062002503F8045C03F588739342F8D1C3
:102AD00004F5AE6000F0C4FC04F27C5000F0C0FCD1
:102AE00084F8945684F8A45784F8A8572576FF20D4
:102AF00008F020F8E06150B90749684606F00EF882
:102B0000684601F0BDFC684605F0C8FF01E0C4F866
:102B1000AC57204605B030BD76F5000010B5044630
:102B2000C06908F00FF804F27C5000F004FD04F5D1
:102B3000AE6000F000FD2046FDF72CFF204610BDE2
:102B400038B504460D461146FDF71AFF01236561AD
:102B5000237638BD10B50446406903689B689847E2
:102B6000E8B12046FDF7B6FF606903689B689847A7
:102B700018B12046FDF782FF40B194F8A83723B181
:102B8000074B1B68C4F8AC3710BD10BD6069036803
:102B9000DB689847C1B22046FDF706FFE4E710BDA9
:102BA0004095FF1F91F803218878931C18440B78F7
:102BB00010B50BB9CB7803E0012B0ED191F805319C
:102BC00018440023934204DACC18013324792044BA
:102BD000F8E7C04300F0FF0010BDFF2010BD8329BF
:102BE00006D003D80139042904D801E0922901D183
:102BF0000120704700207047C26938B5FF23137069
:102C0000C2695370C3698A789A7091F80321C369C5
:102C10000232DA70C36991F805211A710446002363
:102C200091F80351D8B2421D8542D2B2E06908D969
:102C3000FA2B05D0CA181844127942710133EFE714
:102C4000FD2291F8043183546069E169036801321F
:102C50005B68D2B29847606903685B69984738BD82
:102C60007FB50C46054604F0FBFAD4F808319842CB
:102C700004D928462146FFF7BFFF1AE04FF48870B9
:102C800007F058FF064650B90B49684605F046FF65
:102C9000684601F0F5FB684605F000FF09E02146B3
:102CA0004FF4887203F034FE05F5AE60314600F053
:102CB000DFFB04B070BD00BF84F500002DE9F041DA
:102CC00005461148FDF733FF0A27B0FBF7F705F576
:102CD000AE64204600F0C9FB002813DD204600F05A
:102CE000EBFBD0F808310646C7EB030804F0B8FA4E
:102CF000804507D228463146FFF77EFF204600F088
:102D000020FCE4E7BDE8F081D088FF1F2DE9F04109
:102D100091F80331012B0C46154602D80020BDE87E
:102D2000F08103230126CB7081F80C61FFF73AFF95
:102D300084F804016078A378AB7004284FF0000396
:102D400085F8033185F8053102D10E4B9C6115E001
:102D50000328E3D80C4F4FF0C40808FB007021464D
:102D600001F077FB607808FB007000F0F3FD28B1FC
:102D700095F8053143F0200385F805313046BDE86C
:102D8000F08100BFF094FF1F3889FF1F2DE9F04F3D
:102D90008B78FE2BC7B00C46174634D191F803311F
:102DA000032B30D991F8049091F805A0022594F8EE
:102DB0000331AB4225D904EB0508244998F804B047
:102DC00002A805F0ABFE02A801F04AFB02A805F03C
:102DD00065FE584601F06AFBBBF1FE0F0AF10106E1
:102DE0000CD058460DF10701FFF73EFE68B905E02B
:102DF000042902A8394623D102F044FD3544EDB23E
:102E0000D5E701201FE000201DE000239DF80710FA
:102E10008DF81431F2B28DF80AB08DF809108DF8E2
:102E20000B218DF80C900133D8B29042E0D208EB20
:102E3000030090F804E002A8184480F804E0F2E7E8
:102E400002F06EFADAE747B0BDE8F08FA8F50000AF
:102E5000F8B500F27C55044628460E4600F005FB06
:102E600000284DD02EB9284600F026FB90F80D71B1
:102E700022E03378012B45D1B7781DE0B37884F890
:102E80009A367378042B04F5D3671ED13046394641
:102E900001F0D4FE39462046FFF7AEFE1A4B94F8F7
:102EA0009A761B68C4F8AC37284600F04AFB2846DF
:102EB00000F0DBFA00281EDD284600F0FDFA90F84D
:102EC0000D31BB420646D9D015E0032BE2D830467F
:102ED000394601F019FB72780C4BC42000FB02301C
:102EE00000F038FD0028D5D094F89D3743F020033A
:102EF00084F89D37CEE7284600F0B7FA00B1F8BD58
:102F000084F8A807F8BD00BF4095FF1F3889FF1F50
:102F10002DE9F04F8B78FE2B89B005460F4662D124
:102F200001264FF0FF0997F80331023BB34241DD20
:102F3000BB190DF10F0193F8058093F804A093F8E5
:102F400006B04046FFF790FD80B34FF4887007F05D
:102F5000F1FD044650B9254904A805F0DFFD04A899
:102F600001F08EFA04A805F099FD3CE09DF80F20D1
:102F7000427000230222037080F80280C27080F841
:102F8000032180F804B080F805A02146284601936B
:102F9000FFF708FE84F80401019B84F80C3184F8E3
:102FA0000D9105F27C50214600F062FA0336F6B22C
:102FB000C146B8E705F27C54204600F056FA0028D6
:102FC00011DD012385F8A837094B1B68C5F8AC371C
:102FD000204600F071FA90F80D31FF2B03D12846FE
:102FE0000021FFF735FF09B0BDE8F08FC3F5000001
:102FF0004095FF1F2DE9F04115460E461146044647
:10300000FFF7D0FD95F8043183424FF0010040F006
:103010001D81002384F89D3794F8A83784F898061A
:1030200023B120462946FFF713FF0EE16878EA78BE
:10303000FE280BD1832A01D0922A01D1042A07E06D
:10304000204631462A4600F0B9F9FEE0042A7FD036
:1030500006D8022AA97828D046D8012A15D0B6E089
:10306000062A56D0C0F08D80832A07D0922A40F0DD
:10307000AE8020462946FFF74BFFB3E020462946A5
:1030800004F5D362FFF782FEACE0002384F89906D2
:1030900084F89B376B7884F89A16042B00F0A28092
:1030A0006B4AC42000FB032019E084F899066B7872
:1030B00084F89A16042B05D1284604F5D36101F053
:1030C000BDFD8FE0032B00F28D80284604F5D3610F
:1030D00001F01AFA6A785E4BC42000FB023000F05F
:1030E00039FC00287ED099E084F899066B7884F842
:1030F0009A16042B05D1284604F5D36102F0C2FBD1
:1031000070E0032B6ED8284604F5D36102F008F96D
:10311000E0E7042806D14F48FDF7C6FE4D48FDF70D
:10312000F9FE5FE003285DD84A48FDF7ADFE484B45
:103130006A78C42000FB023000F000FCAB7884F811
:103140009A366B7884F89936002384F89B3747E0E9
:10315000AA7884F89906687884F89A264FF48877D4
:1031600007FB004029463A46203003F0D1FB6B783C
:1031700007FB03412046203104F5D362FFF7C6FD6B
:1031800030E0042809D1344FBA695AB32046314699
:10319000FFF730FF0023BB6124E0032822D82C4F27
:1031A0004FF0C40808FB007001F04AF9D0B168780C
:1031B00008FB007001F04AF9314602462046FFF74D
:1031C00019FF687808FB007001F046F90AE0AA7858
:1031D00084F89A26002384F89B3784F899064023C4
:1031E00084F89D3794F89A36FE2B2ED0EB78832BFB
:1031F0002BD0922B29D095F80C3133BB1548FDF715
:1032000098FC02280FD01348FDF793FC0128EB78B7
:1032100001D1022B07D0012B17D104E094F89D3780
:1032200043F02003DCE704F5D36529462046FFF789
:10323000B9FC84F89C070748FDF779FC3044C4F8D2
:10324000A00729462046FFF70BFD0220BDE8F081CC
:103250003889FF1FD088FF1FF094FF1F037E2DE9E0
:10326000F0410446002B00F0A48090F8A8373BB151
:10327000514B1A68D0F8AC37D31AB3F57A7F35D8EA
:10328000002384F888352046FFF764FC2046FFF7CA
:1032900015FD01272046FDF79DFB052824DD20466E
:1032A0000021FDF7A1FBFF2816D120460121FDF7E3
:1032B0009BFBFF2810D102212046FDF795FB002340
:1032C00084F88A0584F8943604F28951FFF7CCFB20
:1032D00080B994F8A8376BB920460121FDF7D8FBD7
:1032E0002046FFF7EBFCD5E7BDE8F081002380F82E
:1032F000A837C5E720460321FDF776FB01280646DF
:1033000025DD2046FDF766FB06F1030880451EDA41
:1033100094F8A8374BB1012384F88835204604215E
:10332000FDF762FB84F88D0607E084F888352046B7
:103330000421FDF759FB84F88B05204694F88B1582
:10334000FFF74DFC60B994F8A8374BB9C4E7042FD8
:1033500004DC2046FFF7FEFB0137C1E7BDE8F08142
:10336000B31E84F88B365FFA88F80525EBB2434527
:10337000204607D22946FDF737FB6319013583F84C
:103380008705F3E74146FDF72FFB414684F88C069D
:103390002046FDF74DFB04F5B16201462046FFF7DC
:1033A00029FE022802D12046311D97E7012897D136
:1033B00092E7BDE8F08100BF4095FF1FF0B50646DB
:1033C00085B04FF488700F46154607F0B3FB0446EE
:1033D00058B92049684605F0A1FB684601F050F84D
:1033E000684605F05BFB05B0F0BD29464FF48872D6
:1033F00003F08EFA012384F80C310025164B65701A
:10340000C42000FB053000F08DFA2146A070304644
:10341000FFF7C8FB013584F80401394630462246DF
:10342000FFF7E8FD042DE9D10C4B65701B68A37014
:1034300021463046FFF7B6FB394684F804012246A0
:103440003046FFF7D7FD204605B0BDE8F04007F055
:1034500079BB00BFD1F500003889FF1FF094FF1F32
:103460000022026042608260704700687047FFFF80
:1034700030B5044685B008200D4607F05BFB50B917
:103480000C49684605F04AFB684600F0F9FF6846BB
:1034900005F004FB0CE000224260A268056012B94E
:1034A000A060606001E05060A06023680133236089
:1034B00005B030BDDFF500001FB544680CB12068D1
:1034C0000AE00649684605F029FB684600F0D8FF87
:1034D000684605F0E3FA204604B010BDEBF50000A5
:1034E00030B5044685B00D46002D19DD636853B92B
:1034F0000E49684605F012FB684600F0C1FF6846B9
:1035000005F0CCFA0CE0186807F01CFB6068436813
:10351000636007F017FB2368013B2360013DE3E78D
:10352000636803B9A36005B030BD00BF24F6000096
:103530000168FFF7D5BF10B50446FFF7F9FF204635
:1035400010BD0121FFF7CCBF10B50446084606495F
:1035500007F026F901464FF07E5007F0D5F90349F0
:1035600007F01EF9606010BDDB0FC94000247449EC
:1035700038B504461D4601701146FFF7E5FFE560CA
:103580002561656103F06CFEE06138BD10B504464D
:10359000FFF7EEFF204610BD38B503780446032B35
:1035A00020D8DFE803F00C020411C06838BD406881
:1035B0000D4907F0A9F9E16807F0F2F838BD406954
:1035C000E16806F0E3FF38BDE168406906F0DEFF20
:1035D00005490546606807F097F90146284607F057
:1035E00093F938BD002038BD0024744970B50446F5
:1035F0000E4603F035FE0546E069281A07F07CF810
:10360000E26822610146A061E5616661606807F0D9
:103610007BF90146A060104807F076F906F04CFCF3
:1036200006F0E6F806F05EFF054629464FF07E50AC
:1036300006F0ACFF616907F0B3F821690646284639
:1036400007F0AEF80146304606F0A2FFE0602046E3
:10365000BDE87040FFF7A0BF000080BF00220270ED
:103660007047012910B5044603D1002303710D20D2
:1036700017E08B1E012B16D804234370052383709B
:103680000623C370D30754BF022301230371012112
:10369000042003F0E5FCA078012103F0E1FCE078D0
:1036A000012103F0DDFCFF2200232272E271A271EE
:1036B00001224FF0FF31637322756375A275637148
:1036C0006372A372E37223732161227010BD032918
:1036D00007D801444B7A23B901234B72437B013352
:1036E00043737047032907D801444B7A022B03D058
:1036F000437B4A720133437370478171704780790D
:103700007047C1717047C079704701727047007A85
:1037100070478171C2710372704703299ABF0918FB
:10372000487A0420704770B51E4603780546144653
:103730001BB3037963B909B906B932B121443144E5
:10374000062391FBF3F1803100E011460D2010E0DB
:10375000022B05D1C943D443F643C9B2E4B2F6B251
:10376000687803F099FCA878214603F095FCE87886
:103770003146BDE8704003F08FBC70BD027D016929
:10378000013AD2B201310346027507D10AB9427B30
:1037900042B918469979DA791B7A09E012B1012207
:1037A000827502E005229A75184600210A460B46EA
:1037B000FFF7B9BF03690133032B08DCC218517A44
:1037C0005A1C11B10361027506E01346F4E74FF08D
:1037D000FF3303610123037500F016B8032910B508
:1037E00010D843185C7A012C00D05AB100225A72CA
:1037F000437B013B437303698B4203D1BDE8104017
:10380000FFF7D8BF10BDFFFF30B5037D85B004467C
:10381000002B4BD003695A1C06D1037A8179C279F7
:10382000FFF781FF142327E003445D7A012D0FD1B8
:103830008179C279037A112938BF4021112A38BF12
:103840004022112B38BF4023FFF76DFF65752FE035
:10385000022D03D18021002208230AE0032D03D189
:10386000002180220B4604E0042D07D160210022B4
:103870008023FFF758FF0123637519E00D4968465F
:1038800005F04CF9684600F0FBFD684605F006F9C6
:103890000949684605F042F9684600F0E1FD6846CE
:1038A00005F0FCF8206900F019FE01E0FFF782FF47
:1038B00005B030BD6EF60000CAF6000038B50378DA
:1038C0000446A3B1437D13B1013B437538BD857DEB
:1038D00015B1013D857538BD4379012B03D1FFF743
:1038E0004DFF657138BDFFF78FFF0123637138BD50
:1038F00010B5044602F0B8FD04F1380001214FF084
:103900007E520023FFF742FE002384F8B03084F893
:10391000BB3084F8A430C4F8C030204610BD90F805
:10392000BB007047007A7047017290F8B30002F054
:1039300005BA406F7047D0F88C00704703460022EC
:1039400080F8B020997902480122FFF747BF00BFF5
:10395000488CFF1F90F8B0007047F8B5044603F09C
:103960007FFC064694F8640003F0B2F9A065E76DA9
:10397000A06D06F0C1FE04F1380501462846FFF7A8
:1039800035FE2846FFF708FE07F05AF8E065E36DBC
:10399000D4F8BC10C4F8BC60DF1B701A236A216E17
:1039A000642241437B43534391FBF2F293FBF2F3D6
:1039B000A26EC3EB0313132101FB0233142293FB0A
:1039C000F2F3A366F8BD806D7047FFFFC26A836A99
:1039D00070B5D31A044642F210750C4805FB03F685
:1039E000FDF700F9A26AE36A96FBF0F055439A42AC
:1039F0002063656305DC9342B4BF194611461A463D
:103A000000E019460A44226670BD00BFD088FF1F3F
:103A100038B5826943690446D31A054803FB01F5AA
:103A2000FDF7E0F8616995FBF0F0084438BD00BF90
:103A3000D088FF1F38B5044605480D46FDF7D2F87B
:103A40006369A269E91A4843D31A90FBF3F038BDC1
:103A5000D088FF1F38B5C36D42F210755D43436BCC
:103A6000ED1A036B95FBF3F590F8253004461BB176
:103A70000748FDF7B7F8451BD4F89000D4F8943008
:103A80008542A8BF28469842A8BF184638BD00BF47
:103A9000D088FF1FD0F89030D0F894209942B8BF5A
:103AA000194690F825309142A8BF114610B504463A
:103AB000C0F898102BB11248FDF794F8D4F898107C
:103AC000411A2046FFF7A4FF94F82530C4F89C0063
:103AD00033B10B48FDF786F8D4F89830C01A01E0EE
:103AE000D4F89800226B636B42F2107102FB003332
:103AF00093FBF1F3C4F8A030012384F8A43010BD87
:103B0000D088FF1F10B50446C0F89C10FFF792FF45
:103B100094F82530C4F898002BB10A48FDF762F8F4
:103B2000D4F89830C01A226B636B42F2107102FB1A
:103B3000003393FBF1F3C4F8A030012384F8A430E0
:103B400010BD00BFD088FF1F38B590F8B0500446B4
:103B5000002D7AD190F8243003B938BD90F8243084
:103B6000002B6DD094F8883093B13848FDF745F8B4
:103B7000374B1A681432904267D884F88850196815
:103B80003248FDF73CF82046BDE8384002F0F2BC70
:103B900094F8A430EBB12D48FDF72FF82C4B1A68A0
:103BA000143290421D4650D894F8B23023B12046CA
:103BB00002F0ECFC002844D02046D4F89C1002F01F
:103BC00005FD29682148FDF71AF8002384F8A43080
:103BD00038BD94F8B230002B37D0E56DD4F8A03062
:103BE0001A48EB1A83EAE375A5EBE375FCF7F7FFD8
:103BF00000280CBF062302239D42204618DD02F058
:103C0000C5FC10BB124D1148FCF7F7FF2B681433AD
:103C100098421AD8D4F89C10204602F0D7FC2046CF
:103C200002F0A8FC29680948BDE83840FCF7E7BF66
:103C300002F0ACFC48B12046BDE8384002F08EBC32
:103C400038BD204602F096FCB6E738BDD088FF1F8D
:103C50004095FF1F90F8A530012B10B5044605D103
:103C6000426FD0F8A8309A4224DC10BD022B29D133
:103C7000626FD4F8A8309A420EDDFFF7EBFED4F85D
:103C8000A830616FC91A0029B8BF4942CB1A0A216E
:103C9000594300EB410110E0FFF7DCFED4F8A830F7
:103CA000616FC91A0029B8BF49425B1A0A2101FB9A
:103CB000030102E0FFF7CEFE01462046BDE81040BA
:103CC000FFF7E8BE10BD90F8B03010B50446D3B988
:103CD00002F05CFCA0B92046FFF7BCFE014620467E
:103CE000FFF796FE0146204602F070FC2046FFF7E3
:103CF000B1FE01462046FFF7CDFE204602F03AFC19
:103D0000012384F8243010BD30B5837985B0044692
:103D1000032B1DD8DFE803F0020D17171A48FCF734
:103D20005EFF40F62C3540F2CB23002808BF1D462D
:103D300019E01548FCF753FF00280CBF4FF47A75C3
:103D40004FF47A650FE01048FCF74CFF05460AE097
:103D50000E49684604F0E2FE684600F091FB6846B2
:103D600004F09CFE0DE0204602F010FC30B9204625
:103D70002946FFF78FFE204602F0FCFB012384F862
:103D8000243005B030BD00BFD088FF1FE3F600002F
:103D9000002280F8242002F0E1BBFFFF38B5044682
:103DA00001230D4680F8B030FFF7F2FFA1790448F7
:103DB0000DB1042200E00222BDE83840FFF792BCBA
:103DC000488CFF1F90F8B01010B5E1B9446F40F671
:103DD000FF72944217D0446F40F26C72944210DD2F
:103DE000D0F8AC20084C1AB92268C0F8AC2010BD3D
:103DF00023689A1AB2F5C87F05D9BDE81040FFF7CD
:103E0000CDBFC0F8AC1010BD4095FF1F13B50446E0
:103E100003220E48A179FFF765FCD4F88C30023BF1
:103E2000C4F88C30D4F88C300193019B012BCCBFAB
:103E3000019B0123C4F88C30D4F88C30092B03DCAF
:103E400020460121FFF7AAFF02B010BD488CFF1FDA
:103E5000F8B5044690F8700002F03AFFA067D4F875
:103E60008060A26FD4F88450676FD4F88000D4F8D3
:103E700084100A235D435E4301447D4302FB0652E6
:103E80004B4392FBF3F36367D4F88050A36FD4F8ED
:103E90008400E66FD4F88010D4F88420704303FBCC
:103EA00005030A4493FBF2F3E367636FB3F5486FCE
:103EB0000ADD204602F052FB012384F888302046B8
:103EC000BDE8F840FFF7A2BFF8BD90F824007047A6
:103ED00080F8A510704790F8A500704740F2DC53B9
:103EE0009942D8BFC0F8A8107047D0F8A800704712
:103EF00038B590F8243004460BB9002038BDC56DA4
:103F0000D0F8A0300B485B1B83EAE375A5EBE375A3
:103F1000FCF765FE00280CBF0C2304239D42ECDD5A
:103F2000E26DD4F8A030606F9A42A8BF00F58050CF
:103F300038BD00BFD088FF1F012380F8B230704722
:103F4000002310B580F8B23090F8243004463BB11D
:103F500002F01CFB20B92046BDE8104002F00ABB6D
:103F600010BD90F8B2007047012380F8B13070475F
:103F7000002380F8B130704710B5044690F8B500C2
:103F8000616901F007FFA16994F8B60001F002FF32
:103F9000A16A94F8B80001F0FDFE94F8B900E16A56
:103FA00001F0F8FE2046BDE81040FFF70FBD90F885
:103FB000B1007047836E002B82B0836E08DD0093E2
:103FC000009B0098002BD8BF404200F5806005E0C0
:103FD0000193019B0198002BD8BF404202B070476B
:103FE000012938B504460D4606D890F8BA0001F00C
:103FF00055FEE571012038BD002038BDC368012B96
:1040000003D049DB032B1EDD46E08379032B1AD84E
:10401000DFE803F002090B1206230377132380F86D
:10402000643012232AE007232DE0032303771723AC
:1040300080F86430162321E004230377152380F8E9
:104040006430142324E08379032B25D8DFE803F0C0
:104050000209101A092303771E2380F864301A23FB
:104060000CE00A2303771B2380F864301C230FE045
:1040700003230377162380F86430152380F870300B
:1040800000230FE020230377112380F864301023EE
:1040900080F87030012305E00023037780F8643056
:1040A00080F8703080F825307047FFFF70B5044607
:1040B00088B01E46012384F8B1309DF8343084F86E
:1040C000B5309DF8383084F8B6309DF83C3084F82F
:1040D000B8309DF840309DF8300084F8B9309DF834
:1040E000443084F8BA30A17184F8B300154601F069
:1040F000C9FDE560207226742046FFF77FFF94F823
:10410000B50001F0C5FD606194F8B60001F0C0FD96
:104110006369A061984205DC9842B4BF02461A4622
:10412000184600E01A46801A206294F8B80001F0A0
:10413000AFFDA06294F8B90001F0AAFDE06294F826
:10414000BA0001F07BFD0025E071C4F890502A48C8
:10415000FCF748FD84F8A550C4F89400C4F8A850B2
:10416000A5662046FFF732FC217F84F8BB5064230C
:10417000C4F88C304B1E302B0AD9E379012B38D18F
:1041800094F8BB30002B34D02046FFF7BDFD30E063
:10419000204602F0DDF994F86400431E302BECD881
:1041A00002F096FD06F0A8FA6E4603460121134A76
:1041B0006846FFF7EBF90FCE04F138050FC596E816
:1041C0000F0085E80F0094F87000431E302BD4D800
:1041D000012384F8BB300523C4F880301423C4F8CD
:1041E000843002F075FDA067A36F6367A36FE36778
:1041F000C3E708B070BD00BFD088FF1F000020419A
:1042000010B50446FFF75FFD2046FFF799FE616990
:104210002046FFF777FC2046FFF796FC41F294100A
:1042200003F03CF8E36DA362A1692046FFF76AFC46
:104230002046FFF789FC41F2941003F02FF8E36D5C
:10424000E3622046BDE81040FFF7C0BB30B54B1E0F
:10425000632B97B004460D4600F2A4800021FFF7BF
:104260009DFD204602F09CF9642003F017F801211F
:10427000207F02F0F5FE227F4C4B53F832300122B2
:1042800083F8802040F2EE2003F008F8227F00231C
:104290000D210DA802F0AAFA642002F0FFFF44F6F7
:1042A0002C410DA802F0E6FA642002F0F7FF01A805
:1042B000002104F033FC0F2D16D80021102205A890
:1042C00004F07CFC1022294609A804F077FC09A917
:1042D00005A804F0B1FC014601A804F04FFC09A8B0
:1042E00004F0DCFB05A809E02946102209A804F027
:1042F00065FC01A809A904F049FC09A804F0CEFB5B
:10430000002101A804F0C7FC0121044601A804F023
:10431000C2FC2334204400F0DF040C210DA802F07D
:1043200013FA23490DA8FCF70AFE22490DA8FCF751
:1043300006FE20490DA8FCF702FE01A90DA804F015
:104340000BFB1C490DA8FCF7FAFD1A490DA8FCF758
:10435000F6FD18490DA8FCF7F2FD16490DA8FCF76B
:10436000EEFD1022002321460DA804F038FB0D219C
:104370000DA802F0E9F90DA802F0C4F940F2DC50F2
:1043800002F08CFF0DA802F095FAC82002F086FF1B
:1043900001A804F083FB084B0D930DA802F08AFAE4
:1043A000012000E0002017B030BD00BFF0F8000091
:1043B0002EF70000DEE60000B0F80000D0F8900014
:1043C0007047D0F894007047D0F898007047806E1E
:1043D000003018BF0120704780790130C0B27047AB
:1043E0004069704780697047007F70478369416109
:1043F000994205DC9942B4BF0A461A46194600E0C4
:104400001A46114401627047436981618B4205DCA1
:104410009942B4BF0A461A460B4600E00A461344C6
:1044200003627047806A7047C06A704790F8640002
:10443000704781627047C162704790F870007047A2
:10444000D0F8C000003018BF01207047D0F8C0007D
:104450007047C0F8C01070470023C0F8C0307047E4
:10446000054B1A6840F6B7339A42014602D9034811
:1044700004F072BA704700BF4095FF1F1097FF1FEE
:1044800008B5084B1A6840F6B7339A42014607D977
:10449000054804F061FA0448BDE8084004F07CBA1D
:1044A00008BD00BF4095FF1F1097FF1F08B5094BBF
:1044B0001A6840F6B7339A42014609D900230648E4
:1044C0000A2204F08CFA0448BDE8084004F064BAFB
:1044D00008BD00BF4095FF1F1097FF1F08B5084B90
:1044E0001A6840F6B7339A42014607D9054804F0E6
:1044F000AEFA0448BDE8084004F04EBA08BD00BF5B
:104500004095FF1F1097FF1F2DE9F047427903796F
:10451000467881F803219D18013D00220C46EDB23A
:1045200081F80521092B00F28A80DFE803F0050AF3
:104530001622313D49586877902323711DB9BDE893
:10454000F087002700E001270122E31995421A7144
:1045500000F070831744FFB200E00027BA48FCF770
:10456000F8FAE319022D187100F064830137FFB2E5
:1045700000E00027B54BC42000FB0630FFF7D2F95E
:10458000E319032D187100F055830137FFB200E0E5
:104590000027AD48FCF7BCFAE319042D187100F0B0
:1045A00049830137FFB200E00027A748FCF7B7FABC
:1045B000E319052D187100F03D830137FFB200E0CB
:1045C0000027A24BC42000FB0630FFF7F7FEE319DB
:1045D000062D187100F02E830137FFB200E000278E
:1045E0009A4BC42000FB0630FFF7E8FEE3190012E7
:1045F000072D187100F01E830137FFB200E000277D
:10460000924BC42000FB0630FFF7DBFEE319082DB8
:10461000187100F00F830137FFB200E000278B4BC9
:10462000C42000FB0630FFF7CCFEE3190012092D71
:10463000187100F0FF820137FFB20A2300E0002763
:104640001A46C3EB070852FA88F80F2A5FFA88F86F
:1046500009D804EB08010020AA42087100F0EA82A0
:104660000132D2B2EDE7102A0DD17748FCF761FA9A
:1046700004EB0803102D187100F0DC8208F101082A
:104680005FFA88F811221346C2EB080753FA87F73E
:10469000162BFFB208D827440021AB42397100F035
:1046A000C9820133DBB2EFE7172B0DD1674BC42072
:1046B00000FB0630FFF790FEE319172D187100F08C
:1046C000B9820137FFB201E0182B0DD15F4BC42036
:1046D00000FB0630FFF7F9FBE319182D187100F005
:1046E000A9820137FFB201E0192B15D15848314694
:1046F000FFF713F804EB070830B155483146FFF7D0
:104700000CF8003018BF0120192D88F8040000F0C3
:1047100091820137FFB21A231946C3EB070851FAF9
:1047200088F81D295FFA88F809D804EB08020020F0
:10473000A942107100F07E820131C9B2EDE7A1F10A
:104740001E03032B3BD8DFE803F00212232E3F4B5E
:10475000C42000FB0630FFF737FE04EB08031E2DD4
:10476000187100F0678208F101085FFA88F8374B8A
:10477000C42000FB0630FFF727FE04EB08030012FD
:104780001F2D187100F0568208F101085FFA88F8B1
:1047900004EB08030022202D1A7100F04B8208F16F
:1047A00001085FFA88F804EB08030022212D1A7132
:1047B00000F0408208F101085FFA88F822210A46D9
:1047C000C1EB080752FA87F7232AFFB208D827441B
:1047D0000023AA423B7100F02D820132D2B2EFE7F2
:1047E000A2F12403052B5DD8DFE803F00312203487
:1047F0003E4D164BC42000FB0630FFF72BF9E319A2
:10480000242D187100F0168201370028FFB205DA56
:104810000E4BC42000FB0630FFF71CF9E319001211
:10482000252D187100F006820137FFB2074BC42016
:1048300000FB0630FFF7BEFBE319262D187100F0D0
:10484000F9810137FFB207E0D088FF1F3889FF1FC9
:10485000488CFF1F4FF0FF30E3190012272D18710D
:1048600000F0E8810137FFB2A14BC42000FB063005
:10487000FFF73EFBE319282D187100F0DB810137AB
:104880000028FFB205DA9A4BC42000FB0630FFF780
:104890002FFBE3190012292D187100F0CB8101378D
:1048A000FFB22A221346C2EB070853FA88F82A2BD4
:1048B0005FFA88F809D804EB08010020AB420871C0
:1048C00000F0B8810133DBB2EDE72B2B02D02C2BAB
:1048D00010D020E08748FCF757F904EB08030A22C0
:1048E00090FBF2F02B2D187100F0A48108F1010863
:1048F0005FFA88F87E4BC42000FB0630FFF7A0FD6E
:1049000004EB08032C2D187100F0948108F10108C4
:104910005FFA88F82D231A46C3EB080952FA89F981
:104920002D2A5FFA89F909D804EB09010020AA426F
:10493000087100F07F810132D2B2EDE72E2A10D14A
:104940006B4BC42000FB0630FFF741FD04EB09036D
:104950002E2D187100F06E8109F101095FFA89F9B5
:104960002F221346C2EB090753FA87F7322BFFB207
:1049700008D827440021AB42397100F05B81013334
:10498000DBB2EFE7332B0DD1594BC42000FB0630CF
:10499000FFF7E7FAE319332D187100F04B81013767
:1049A000FFB234239A46C3EB07085AFA88F8BAF1E3
:1049B000430F5FFA88F80BD804EB08020021AA45E0
:1049C000117100F037810AF1010A5FFA8AFAEAE709
:1049D000474BC42707FB06373846FEF7AAFFAAF164
:1049E0004403042B43D8DFE803F0030D18253200FD
:1049F00004EB0803442D187100F01C8108F1010834
:104A00005FFA88F804EB08030012452D187100F0D6
:104A1000118108F101085FFA88F83846FFF75BFA60
:104A200004EB0803462D187100F0048108F1010819
:104A30005FFA88F83846FFF758FA04EB0803472D69
:104A4000187100F0F78008F101085FFA88F838461D
:104A5000FFF74BFA04EB08030012482D187100F021
:104A6000E98008F101085FFA88F84FF0490AD14659
:104A7000CAEB080659FA86F6B9F1500FF6B20AD811
:104A800026440023A945337100F0D48009F10109BF
:104A90005FFA89F9ECE7B9F1510F13D13846FFF706
:104AA00086FA30B13846FEF73DFF80F0AA000130AB
:104AB000C0B2A319512D187100F0BC800136F6B2B6
:104AC0004FF052093846FFF772FA002800F0A38031
:104AD000A9F152030E2B00F29E80DFE803F00D17C0
:104AE000222C363F48515B646E757E87910000BF73
:104AF0003889FF1FD088FF1F3846FFF771FCA319C4
:104B0000522D187100F096800136F6B23846FFF744
:104B100067FCA3190012532D187100F08B80013629
:104B2000F6B23846FFF75EFCA319542D187100F059
:104B300081800136F6B23846FFF754FCA319001203
:104B4000552D187176D00136F6B23846FFF74CFC79
:104B5000A319562D18716DD00136F6B23846FFF7FD
:104B60006CFCA319572D187164D00136F6B2384683
:104B7000FFF758FCA319582D18715BD00136F6B217
:104B80003846FFF74FFCA3190012592D187151D068
:104B90000136F6B23846FFF747FCA3195A2D1871B3
:104BA00048D00136F6B23846FFF73EFCA319001292
:104BB0005B2D18713ED00136F6B2A31900225C2D90
:104BC0001A7137D00136F6B23846FFF72FFCA31919
:104BD0005D2D18712ED00136F6B23846FEF7F3FE81
:104BE000A3195E2D187125D00136F6B23846FEF7AE
:104BF000EAFEA31900125F2D18711BD00136F6B220
:104C00000D48FBF7BDFFA319602D187112D00136B6
:104C1000F6B24FF061094B46C9EB06021A44FF2B6E
:104C2000D2B207D022440021AB42117102D001332D
:104C3000DBB2F1E7BDE8F087D088FF1F2DE9F04136
:104C40004279037981F803219D18013D00220C4629
:104C5000EDB281F80521092B74D8DFE803F0050ACD
:104C600016222D39454F5965912323711DB9BDE891
:104C7000F081002600E001260122A31995421A7155
:104C800000F04A831644F6B200E00026B748FBF76E
:104C900060FFA319022D187100F03E830136F6B2B1
:104CA00000E00026B24AA31912681A71032D00F021
:104CB00033830136F6B200E00026AC48FBF728FF4C
:104CC000A319042D187100F027830136F6B200E015
:104CD0000026A648FBF723FFA319052D187100F045
:104CE0001B830136F6B200E00026A3190022062D30
:104CF0001A7100F011830136F6B200E00026A31904
:104D00000022072D1A7100F007830136F6B200E089
:104D100000269648FBF766FFA319082D187100F0CE
:104D2000FB820136F6B200E000269048FBF75AFFFE
:104D3000A3190012092D187100F0EE820136F1B2AC
:104D40000A2300E000211A46CE1A52FA86F60F2AEC
:104D5000F6B208D826440020AA42307100F0DC8266
:104D60000132D2B2F0E7102A0AD18048FBF7E1FE07
:104D7000A319102D187100F0CF820136F6B211225E
:104D80001346B71A53FA87F7132BFFB208D82744F4
:104D90000021AB42397100F0BF820133DBB2F0E792
:104DA000142B0AD17148FBF71AFFE319142D18715F
:104DB00000F0B2820137FFB215231A46FE1A52FAEA
:104DC00086F6172AF6B208D826440021AA42317185
:104DD00000F0A2820132D2B2F0E7182A0ED1654863
:104DE000FFF773F810B16448FFF76FF8A319182D97
:104DF000187100F091820136F6B219221346B71AE3
:104E000053FA87F71D2BFFB208D827440021AB4285
:104E1000397100F081820133DBB2F0E7A3F11E02A9
:104E2000032A31D8DFE802F002151F275148FFF7A7
:104E3000CBFA06465048FFF7C7FA0223304490FBEE
:104E4000F3F0E3191E2D187100F066820137FFB2EE
:104E500001E04FF0FF30E31900121F2D187100F030
:104E60005B820137FFB2E3190022202D1A7100F096
:104E700053820137FFB2E3190022212D1A7100F08D
:104E80004B820137FFB222231A46FE1A52FA86F6E7
:104E9000232AF6B208D826440021AA42317100F034
:104EA0003B820132D2B2F0E7A2F12403032B48D8AF
:104EB000DFE803F00216293C2E48FEF7CBFD07463B
:104EC0002D48FEF7C7FD0223384490FBF3F0A319E9
:104ED000242D187100F0208201360028F6B20ADA7B
:104EE0002448FEF7B7FD07462348FEF7B3FD02232B
:104EF000384490FBF3F0A3190012252D187100F02F
:104F00000B820136F6B21B48FFF754F807461A48E1
:104F1000FFF750F80223384490FBF3F0A319262D35
:104F2000187100F0F9810136F6B201E04FF0FF3060
:104F3000A3190012272D187100F0EE810136F6B288
:104F400028221346B71A53FA87F72A2BFFB208D83C
:104F500027440021AB42397100F0DE810133DBB21E
:104F6000F0E72B2B0AD02C2B15D021E0D088FF1F87
:104F7000F094FF1F848BFF1FC08AFF1FB648FBF70A
:104F800003FEE3190A2290FBF2F02B2D187100F0BA
:104F9000C3810137FFB2B14A9269E319003218BFE9
:104FA00001222C2D1A7100F0B7810137FFB22D2399
:104FB0001A46FE1A52FA86F62D2AF6B208D8264468
:104FC0000021AA42317100F0A7810132D2B2F0E78C
:104FD0002E2A10D1A248FFF7FAF918B9A148FFF715
:104FE000F6F900E00120A3192E2D187100F094812C
:104FF0000136F6B22F221346B71A53FA87F7632BFE
:10500000FFB208D827440021AB42397100F08481F7
:105010000133DBB2F0E7652B0DD0662B15D0642B86
:105020001ED19148FEF76BFBE319642D187100F057
:1050300073810137FFB28C48FEF765FBE319652DDC
:10504000187100F069810137FFB28748FEF75FFBF6
:10505000E319662D187100F05F810137FFB26723F5
:105060001A46FE1A52FA86F66D2AF6B208D8264477
:105070000021AA42317100F04F810132D2B2F0E733
:10508000A2F16E03032B2DD8DFE803F0020C1620EB
:105090007648FBF729FAA3196E2D187100F03C81B0
:1050A0000136F6B27148FBF705FAA3196F2D187196
:1050B00000F032810136F6B26C48FBF719FAA319F9
:1050C000702D187100F028810136F6B26748FBF7A1
:1050D0000FFAA3190012712D187100F01D8101360D
:1050E000F6B272221346C2EB060853FA88F8772B01
:1050F0005FFA88F809D804EB08010020AB42087178
:1051000000F00A810133DBB2EDE7782B02D0792B76
:105110000DD030E05048FBF746FD04EB0803782D36
:10512000187100F0F98008F101085FFA88F84A4820
:10513000FBF739FD18B14848FBF73DFDC0B204EB61
:105140000803792D187100F0E78008F10106424844
:10515000F6B2FBF728FD20B13F48FBF72CFDC0F36A
:10516000072026447A2D307100F0D68008F102081D
:105170005FFA88F87B231A46C3EB080752FA87F7D1
:105180007C2AFFB208D827440021AA42397100F0D6
:10519000C3800132D2B2EFE7A2F17D03042B4CD8D9
:1051A000DFE803F0030D1C2C3B002B48FBF7FFFC52
:1051B000E3197D2D187100F0AF800137FFB226484A
:1051C000FBF7F5FC18B12448FBF7FBFCC0B2E31970
:1051D0007E2D187100F0A0800137FFB21E48FBF74A
:1051E000E6FC20B11C48FBF7ECFCC0F30720E319F8
:1051F0007F2D187100F090800137FFB21648FBF741
:10520000D6FC18B11448FBF7E3FCC0B2E319802DBB
:10521000187100F081800137FFB20F48FBF7C7FC1F
:1052200020B10D48FBF7D4FCC0F30720E319812D12
:10523000187171D00137FFB282221346BE1A53FA99
:1052400086F6BD2BF6B213D826440021AB4231714D
:1052500062D00133DBB2F1E7D088FF1FF094FF1F6B
:10526000848BFF1FC08AFF1F488CFF1F9894FF1F6D
:10527000A3F1BE02052A41D8DFE802F0030D172191
:105280002B3526480021FBF7BCFCA319BE2D187155
:1052900042D00136F6B221480121FBF7B2FCA31936
:1052A000BF2D187138D00136F6B21C480221FBF729
:1052B000A8FCA319C02D18712ED00136F6B21748DC
:1052C0000321FBF79EFCA319C12D187124D00136D0
:1052D000F6B212480421FBF794FCA319C22D1871F1
:1052E0001AD00136F6B20D480521FBF78AFCA31946
:1052F000C32D187110D00136F6B2C4231A46F11A24
:105300001144FF2AC9B207D021440020AA420871E3
:1053100002D00132D2B2F2E7BDE8F081D088FF1F9F
:105320002DE9FF4783788B70002381F803310579DD
:1053300090F8038181F80531A844A8F102080646D7
:105340000C4690F801905FFA88F8052D43D8DFE805
:1053500005F0030303052839482358E2C04D477977
:105360002846FEF7DFFA874200F0548205F1C400B8
:10537000FEF7D8FA874200F04D8205F5C470FEF7BB
:10538000D1FA874200F0468205F51370FEF7CAFA9B
:10539000874200F03F82B34B1B689F4240F0488237
:1053A00038E201257319B0481979FBF7B3FBB8F15E
:1053B000040F00F0608294F80531002B40F05B820E
:1053C000013500E001253544A7482979FBF7A9FB01
:1053D000B8F1050F62E00F2D40F21582102D0CD1AF
:1053E0004179022903D8A048FBF7A5FB02E0082376
:1053F00084F80531B8F1100F50E0122D40F203820D
:10540000132D14D1417901290BD8954BC42000FBF1
:105410000930FEF7E5FD38B994F8053143F008038B
:1054200000E0082384F80531B8F1130F36E0172D9A
:1054300040F2E981182D17D1437933B9884BC42044
:1054400000FB0930FEF7A4FC0BE0012B06D1844BD6
:10545000C42000FB0930FEF736FC02E0082381F887
:105460000531B8F1180F19E0192D1AD17C4BC42061
:1054700000FB0930FEF76EFA737920B1002B40F083
:10548000DE81012B02E0012B00F2D98140F0E8819E
:1054900076484946FEF71BF9B8F1190F40F0AD8187
:1054A000E9E11D2D40F2AF81A5F11E03032B3AD88F
:1054B000DFE803F002092D36B8F11E0F437900F042
:1054C000DA81022201E0002301221644C422357948
:1054D00003EB0525624B02FB09394846FEF76EFFD8
:1054E000854205DB4846FEF76CFF854240F3BE81EE
:1054F00094F8053143F0020384F80531B8F11F0F29
:1055000000F0B98194F80531002B40F0B481B8F176
:10551000200F00F0B08194F80531002B40F0AB81F2
:10552000B8F1210FBAE7322D40F26D81332D08D149
:10553000437953B94A4BC42000FB0930FEF700FD04
:1055400061E1452D40F25F810CE0012B06D1444B17
:10555000C42000FB0930FEF7EFFC54E1082381F87A
:10556000053150E1472D1ED0482D2AD0462D42D17D
:10557000417919B1012901D0022906D1384BC42043
:1055800000FB0930FEF7A4FC02E0082384F8053193
:10559000B8F1460F00F06F8194F80531002B40F010
:1055A0006A81022300E00123F218B8F1470F127953
:1055B00000F0618194F80511002940F05C8101330D
:1055C00001E0002201233344197940F2DC5302EB5D
:1055D0000121994206D994F8053143F0080384F873
:1055E000053105E01E4BC42000FB0930FEF776FCB8
:1055F000B8F1480F52E7502D40F20581512DDFF8E8
:1056000060A035D1C42505FB09A547792846FEF7DA
:1056100089F980F0AA00C3B201339F42284602D123
:10562000FEF7A2FC0FE0FEF7C2FC30B12846FEF701
:10563000A3FC2846FEF79CFC05E094F8053143F0F6
:10564000080384F80531B8F1510F00F0148194F883
:105650000531002B40F00F810227522509E000BFE1
:105660003889FF1FF094FF1FD088FF1F488CFF1F51
:105670000127C42303FB09A94846FEF798FC00282C
:1056800000F0BF80A5F152030D2B00F2BA80DFE8D5
:1056900003F007153644B8B866758A97ACB8BABA3D
:1056A000F319B8F1520F1B7900F0E58094F8052149
:1056B000002A40F0E0800137FFB200E00023F21939
:1056C0004846117903EB0121FEF790FE4846FEF7AC
:1056D00087FE01464846FEF7ADF901464846FEF70B
:1056E000D9F94846FEF730FAB8F1530F00F0C380FD
:1056F00094F80531002B40F0BE800137FFB2F3195A
:10570000B8F1540F1B7900F0B68094F80521002AF7
:1057100040F0B1800137FFB200E00023F2194846A3
:10572000117903EB0121FEF76FFE4846FEF75AFEA2
:1057300001464846FEF77EF901464846FEF7AAF9BB
:105740004846FEF701FAB8F1550F00F0948094F83E
:105750000531002B40F08F800137FFB25625F31939
:1057600045451B7900F0878094F80521002A40F018
:10577000828001350137EDB2FFB200E00023F2195B
:105780004846117903EB0121FEF753FE4846FEF728
:105790001DF945456FD094F80531002B6BD10135CB
:1057A0000137EDB2FFB2F31945451B7963D094F888
:1057B0000521002A5FD101350137EDB2FFB200E0CB
:1057C0000023F2194846117903EB0121FEF733FE5D
:1057D0004846FEF7FBF845454DD094F80531002BBF
:1057E00049D101350137EDB2FFB23E44337913B1EF
:1057F0004846FEF705FD454550E694F8053113B1DE
:1058000039E0FF2D37D094F8053143F0480384F890
:10581000053130E094F8053143F0080384F8053190
:10582000B8F1030F27D094F8053123BB0225B9E561
:10583000C42000FB09507179FEF776F8F0E794F880
:1058400005310E4943F0080384F80531684603F03A
:1058500065F96846FEF714FE684603F01FF91BE67B
:10586000074849460022FDF7B9FF15E64846294694
:10587000FEF710F942E604B0BDE8F08730F700000B
:10588000488CFF1FF8B5002381F8033181F80531FA
:1058900090F8036103791E44023E05460C46F6B2B9
:1058A000052B3DD8DFE803F0030303052434482328
:1058B0009BE14779B548FEF735F8874200F09B81B8
:1058C000B348FEF72FF8874200F09581B148FEF704
:1058D00029F8874200F08F81AF48FEF723F887420E
:1058E00000F08981AD4B1A68974240F0918182E1C6
:1058F0000127EB19AA481979FBF70CF9042E00F0DF
:10590000968194F80531002B40F09181013700E039
:1059100001272F44A2483979FBF703F9052E5CE1F2
:105920000F2B40F25E81102B0BD14179022903D855
:105930009B48FBF700F902E0082384F80531102E9C
:105940004BE1132B40F24D81142B0CD1417909B15D
:10595000012903D19248FBF761F902E0082384F89A
:105960000531142E39E1172B40F23B81182B16D14B
:10597000437933B98848FEF70BFA8648FEF708FAF0
:105980000BE0012B06D18448FEF79DF98148FEF714
:105990009AF902E0082384F80531182E1DE11D2B29
:1059A00040F21F81A3F11E02032A3CD8DFE802F077
:1059B000020831391E2E437900F03981022201E0BC
:1059C00000230122154474482D7903EB0525FEF7C9
:1059D000F5FC85420FDB7048FEF7F3FC85420ADCDC
:1059E0006C48FEF7EBFC854205DB6A48FEF7E9FCF4
:1059F000854240F3138194F8053143F0020384F8A3
:105A000005311F2E00F0138194F80531002B40F072
:105A10000E81202E00F00B8194F80531002B40F010
:105A20000681212ED9E0632B40F2DB80652B11D05B
:105A3000662B1FD0642B25D15A486979FDF75DFE8E
:105A4000642E00F0F48094F80531002B40F0EF80D4
:105A5000022700E00127EB1952481979FDF751FEA2
:105A6000652E00F0E48094F80531002B40F0DF80D3
:105A7000013700E001272F444A483979FDF745FEF8
:105A8000662EAAE06D2B40F2AC80702B1CD0712BDF
:105A900027D06F2B30D143791BB94348FAF716FD55
:105AA00008E0012B03D14048FAF706FD02E0082385
:105AB00084F805316F2E00F0BA8094F80531002B80
:105AC00040F0B580022300E00123EA18702E12791D
:105AD00000F0AD8094F80511002940F0A880013352
:105AE00001E0002201232B442F48197902EB012108
:105AF000FAF7CAFE712E70E0BD2B72D9A3F1BE0277
:105B0000052A75D8DFE802F00312213152612448DA
:105B10006A790021FBF77BF8BE2E00F0888094F8AC
:105B20000531002B40F08380022700E00127EB19AC
:105B30001B481A790121FBF76AF8BF2E77D094F839
:105B40000531002B73D1013700E00127EB19144810
:105B50001A790221FBF75BF8C02E68D094F8053162
:105B6000002B64D10137FFB200E00127EB190C488C
:105B70001A790321FBF74BF8C12E58D094F8053160
:105B8000002B54D10137FFB211E000BF3889FF1F4D
:105B9000FC89FF1FC08AFF1F848BFF1FF094FF1F2B
:105BA000D088FF1F488CFF1F9894FF1F0127EB1917
:105BB0001F481A790421FBF72AF8C22E37D094F82F
:105BC0000531A3BB0137FFB200E001273D4418486F
:105BD0002A790521FBF71BF8C32E28D094F805314C
:105BE0002BBB94F8053143F0480384F80531F8BD28
:105BF000FF2BF6D1F8BD94F8053143F0080384F883
:105C00000531032E13D094F8053183B9022770E6CD
:105C100069791960092000F091F8F2E729460548F2
:105C2000FDF738FF04482946FDF734FFE9E6F8BDE3
:105C3000D088FF1F848BFF1FC08AFF1F0F281FB54E
:105C400004460FD801F034F90028FBD072B63A2090
:105C500001F01AF962B60123A340DBB218402041DB
:105C6000C0B20AE00649684602F058FF6846FEF7EF
:105C700007FC684602F012FF002004B010BD00BF10
:105C80004EF7000008B572B601F0EAF862B608BD3A
:105C900008B572B601F0F8F862B608BDF0B5244D4B
:105CA0002B68642B85B004460F462E460DDD214936
:105CB000684602F033FF6846FEF7D2FB684602F002
:105CC000EDFE2868FEF70AFC2FE00F2823D801F02C
:105CD000EFF80028FBD072B63A2001F0D5F862B692
:105CE000012317F0010F03FA04F40BBF20EA0404A8
:105CF000E4B204F0FF04044301F0DAF80028FBD01A
:105D000072B63A20A1B201F0F5F862B633680233F8
:105D1000336001200AE00849684602F0FFFE684649
:105D2000FEF7AEFB684602F0B9FE002005B0F0BDFC
:105D30009888FF1FA5F70000FAF70000F0B5134C94
:105D40002368642B85B006460F4625460EDD1049B4
:105D5000684602F0E3FE6846FEF782FB684602F002
:105D60009DFE2068FEF7BAFB00200DE001F0A0F8D0
:105D70000028FBD072B63046394601F0A1F862B671
:105D80002B6801332B60012005B0F0BD9888FF1F00
:105D9000A5F70000F0B5134C2368642B85B00646C8
:105DA0000F4625460EDD1049684602F0B7FE6846EC
:105DB000FEF756FB684602F071FE2068FEF78EFB88
:105DC00000200DE001F074F80028FBD072B63046D8
:105DD000B9B201F08FF862B62B6802332B60012054
:105DE00005B0F0BD9888FF1FA5F7000008B590B179
:105DF00016210920FFF7A2FF18210720FFF79EFFB9
:105E00001A210820FFF79AFF1C212E20FFF796FF8A
:105E10002F201E2111E015210920FFF78FFF1721E8
:105E20000720FFF78BFF19210820FFF787FF1B21B1
:105E30002E20FFF783FF2F201D21BDE80840FFF72C
:105E40007DBF08B54FF448710A20FFF7A3FF40F665
:105E500098010C20FFF79EFF4FF496610E20FFF78C
:105E600099FF40F272611020FFF794FF4FF44871E0
:105E70001220FFF78FFF40F698011420FFF78AFFEA
:105E800040F2CF311620FFF785FF40F69801182029
:105E9000FFF780FF4FF448611A20FFF77BFF4FF4B4
:105EA000C8711C20FFF776FF40F6C4111F20FFF7D2
:105EB00071FF40F20E612120FFF76CFF4FF4486143
:105EC0002420FFF767FF4FF4C8712620FFF762FF19
:105ED0004FF448612920FFF75DFF4FF4C8712B2074
:105EE000FFF758FF00200146FFF7D8FE00210120F0
:105EF000FFF7D4FE00210220FFF7D0FE002103208F
:105F0000FFF7CCFE05200121BDE80840FFF7C6BE23
:105F100010B5084C084B2278C42000FB0230FDF776
:105F200097FF23780133DBB2032B88BF0023237054
:105F300010BD00BF9E88FF1F3889FF1F0148FDF775
:105F4000BDBC00BF488CFF1F10B51E4C2368042B3E
:105F5000C4BF002323602368042B2ED8DFE803F09E
:105F6000030A151D2A001848FAF721FE10B1164839
:105F7000FAF766FE1448FAF716FEF0B1124801214E
:105F8000FAF790FE1048012111E00F48FAF70FFED2
:105F900098B10D48FAF76DFE0FE00B48FAF703FED3
:105FA00058B109480021FAF77DFE07480021FAF7A9
:105FB00097FE02E00448FAF734FE236801332360B9
:105FC00010BD00BFA088FF1FD088FF1F70B50D4C0B
:105FD0000D4D2378032B84BF002323702078C42623
:105FE00006FB0050FDF7EEFE207806FB0050FDF7A3
:105FF00031FEFFF7A9FFFFF7A1FF237801332370DC
:1060000070BD00BF9C88FF1F3889FF1F70B50B4C07
:106010000B4D2378032B84BF002323702078C426E4
:1060200006FB0050FDF799FC207806FB0050FDF7B9
:106030008BFD23780133237070BD00BF9D88FF1F47
:106040003889FF1F10B5044602F064FC204610BDDD
:1060500010B504460430FAF79DFC204610BDFFFF42
:1060600010B5094C04F5137000F01EFA04F5C47065
:1060700000F01AFA04F1C40000F016FA2046BDE858
:10608000104000F011BA00BF3889FF1F064B10B551
:10609000541E9C4206D830235A43013ABDE81040B2
:1060A00002F022BC002010BD57555505054B417329
:1060B0001B782BB1037B03F1604303F56443197034
:1060C000704700BFFC96FF1F30B501218BB00D203B
:1060D00000F0C6FF7A48FAF732FD04467848FAF72E
:1060E00033FD214602467748FDF7BBFA80210A4678
:1060F0000B467448FDF70DFB80210A460B4671489C
:10610000FDF711FB642001F0C9F800F0EBFB0C2057
:1061100000F08AFD012000F0B1FD002000F060FDDC
:106120006748FAF70CFD04466548FAF70DFD4FF095
:106130001A0E03460A2107200C228DE80740002191
:106140001C220591049260482246FDF7AFFF5C488F
:10615000FAF7F5FC04465A48FAF7F6FC4FF01F0C24
:1061600003460E21082010228DE80710012121226C
:106170000591049255482246FDF798FF5048FAF7DA
:10618000DEFC04464E48FAF7DFFC4FF0140C4FF0EB
:10619000240E2E2112228DE80650022126220346CB
:1061A000059104924A482246FDF780FF4448FAF7D9
:1061B000C6FC04464248FAF7C7FC162203464FF0D5
:1061C000180C2F204FF0290E8DE8055003212B22AB
:1061D0000492404805912246FDF768FF3848FAF7D7
:1061E000CFFC38B13648FAF7CBFC31288CBF0025FC
:1061F000012500E00546002433482044FDF78FFBCD
:1062000040B3C434B4F5447FF6D11DB33248802185
:10621000FFF74CFF192231492F48FFF737FF304B6A
:10622000402118702F48FFF741FF41F288322E4974
:106230002C48FFF72BFF2D4B802118702C48FFF7BF
:1062400035FF2B482B494CF25032FFF71FFF2A4BEA
:10625000187010E0294906A802F060FC06A8FEF7B5
:106260000FF906A802F01AFC1D4A002313701F4AFA
:106270001370214A13701248FAF74FFC430803F1D8
:10628000376303F5D833B3FBF0F001F06BF80C483B
:10629000FAF786FC01F00AF90948FAF73EFC1849BA
:1062A00002461848FCF74CFC17481849FAF748FA18
:1062B000082104480A460B46FDF72BFA0BB030BD07
:1062C000D088FF1F488CFF1F3889FF1FFC89FF1FE4
:1062D000C08AFF1F848BFF1F2489FF1F115F0000EE
:1062E0002089FF1FA888FF1F0D6000002189FF1F64
:1062F000BC88FF1FCD5F0000A488FF1F52F800007C
:10630000C896FF1FA48CFF1F9894FF1FE896FF1FDD
:1063100010B500240C48FCF7A1FF0C48FCF77CF9F1
:106320000B48FCF779F9002C4FF0200301DA094AF9
:1063300000E0094A013413604FF6E8539C42C8BF9D
:106340006FF00904E6E700BFA48CFF1F608CFF1FFD
:106350005494FF1F84F00F4088F00F40F8B5304C84
:10636000304E314D2046FDF7C3FA04F1C400FDF76D
:10637000BFFA04F5C470FDF7BBFA04F513702B4C9B
:10638000FDF7B6FA22462A49002004F07FFB29488F
:10639000FDF764F9304628494FF4E132FAF7F7FD8A
:1063A0003046264E2946224604F070FB30462449EA
:1063B0004FF4E132FAF7EBFD2946224D22463046F2
:1063C00004F064FB2846FAF7B5FC22461E4928462D
:1063D0001E4D04F05BFB1E48FAF75CF82846FCF7FC
:1063E00067FB224628461B491B4D04F04FFB1B4808
:1063F00000278026294622460770467304F046FB94
:106400001748294622460770467304F03FFB15489B
:106410004673077029462246BDE8F84004F036BBB3
:106420003889FF1F608CFF1F516000006087FF1FCD
:1064300061600000488CFF1F1097FF1F5494FF1FDE
:10644000E896FF1FD088FF1F030B0000A48CFF1FDE
:106450009894FF1F1D2B0000456000002489FF1F3A
:10646000A888FF1FBC88FF1F30B50D4C0023218872
:1064700003710C2201230B4207D10A4A19432180E0
:10648000118821EA0303138030BD05795B000135D3
:10649000013A05719BB2EED1FF23037130BD00BFFD
:1064A0001495FF1F1095FF1F044B0279012101FA7B
:1064B00002F2198821EA02021A8070471495FF1F20
:1064C000F8B51E4603790B2B0446154634D8CFB2D7
:1064D0003846012100F0C4FD2379184AD754184AE0
:1064E00044F2506122F81310164B1A6805EB45056B
:1064F00006EB4606AD00B60012F4800225806680E9
:1065000016D1196841F480011960A3F59033383B26
:106510004FF6FF7119605A609A6042F6A27243F812
:10652000042C02F5803243F8042C074B20221A7009
:10653000064B4FF480721A602079F8BD2E95FF1F2C
:106540001695FF1F3C80044048E400E008E100E0AD
:106550004FF408724FF41663FFF7B2BF044B027991
:10656000012101FA02F2198821EA02021A80704719
:106570001095FF1F044B0279012101FA02F21988DC
:106580000A431A80704700BF1095FF1F034B027922
:106590001B8843FA02F000F0010070471095FF1FBE
:1065A00003790B2B0CD8012202FA03F3054A118858
:1065B00021EA030313801BB9034B4FF480721A6066
:1065C000704700BF1095FF1F88E100E00C2359437E
:1065D0000388994203DB43889942B8BF0B4602798E
:1065E0000B2A9CBF014921F8123070471695FF1FF6
:1065F00070B52E4A2E4D118895F90030194111F0D1
:10660000010F144606D02B4A0021D05C00F008FD93
:106610000C232B702088284C2178CBB25AB20B2A3D
:106620001FDC40FA02F60131F607C9B2F5D5237036
:10663000204B0121985C00F0F3FC23781F4A2B705B
:1066400059B2013332F811101D4A10680844106025
:106650001C4A10680144116042F6A37142F80C1CF8
:1066600022E0174A23701168C1F56A3303F5C0733D
:10667000B3F5966F05DB4EF660208342A8BF034654
:1066800001E04FF49663194411600E490868034411
:106690000B600D4B42F6A371196012680B4B9A42C6
:1066A00003D9074A00231360237070BD1095FF1FA4
:1066B0006487FF1F2E95FF1F1295FF1F1695FF1F62
:1066C0000C95FF1F0C600340006003407FA903008E
:1066D0000B4A10B514680C1B044442F224739C420C
:1066E00008D9A1F51C53103B62B61468241A9C42C9
:1066F000FBD372B613681B1A8B42FBD310BD00BFCD
:10670000041000E0006908B510B103685B699847A0
:1067100008BD006908B510B103689B68984708BDBB
:10672000006908B518B103681B69984708BD4FF0A8
:10673000FF3008BD006908B518B10368DB689847E9
:1067400008BD4FF0FF3008BD2DE9F04704468946EB
:1067500000F086FD236933B11A681846126849466D
:106760009047BDE8F0876069002837D01C4A11685F
:1067700041F0807111601B4A116841F00101116004
:10678000656972B6DFF860A0A269DAF8006013707C
:1067900030462946FFF79CFF08274FF0010818EA0A
:1067A000090FA3690CBF002201221A7063691D44FE
:1067B00030462946FFF78CFF4FEA4808013F5FFA51
:1067C00088F8ECD1A36901221A7062B663691D448E
:1067D000DAF800309B1BAB42FAD30120BDE8F0870A
:1067E000FCED00E0001000E0041000E0F8B51646F3
:1067F0004FF47A7200238260194A037104460373CE
:10680000026080F820300D4619B9012E0ED1154BCB
:1068100004E0092904D10A2E08D1134B23611DE09D
:10682000072903D1082E01D1104BF7E70027304686
:106830000121276100F014FC2846022100F010FC21
:106840000B4B84F8216084F8225053F83620A26163
:1068500053F83530676103F50073E3612046F8BDF6
:10686000B0F80000C896FF1FD896FF1FE896FF1FDC
:10687000F0F8000008B5036923B11A681846926958
:10688000904708BD4B0803F1B76303F55843B3FBCA
:10689000F1F34361054B1A6842F080721A60044BB1
:1068A0001A6842F001021A6008BD00BFFCED00E06A
:1068B000001000E038B50569044635B12B6828465C
:1068C0001B6A98470023236109E090F821002946BC
:1068D00000F0C6FB94F82200294600F0C1FB00231B
:1068E000636138BD38B50920FFF7CCF9064C0025A7
:1068F000206006486560FAF775F92573A060656148
:106900002561A56138BD00BFF094FF1FD088FF1F2F
:10691000844641EA000313F003036DD1403A41D3AA
:1069200051F8043B40F8043B51F8043B40F8043B69
:1069300051F8043B40F8043B51F8043B40F8043B59
:1069400051F8043B40F8043B51F8043B40F8043B49
:1069500051F8043B40F8043B51F8043B40F8043B39
:1069600051F8043B40F8043B51F8043B40F8043B29
:1069700051F8043B40F8043B51F8043B40F8043B19
:1069800051F8043B40F8043B51F8043B40F8043B09
:1069900051F8043B40F8043B51F8043B40F8043BF9
:1069A000403ABDD2303211D351F8043B40F8043B99
:1069B00051F8043B40F8043B51F8043B40F8043BD9
:1069C00051F8043B40F8043B103AEDD20C3205D3A9
:1069D00051F8043B40F8043B043AF9D2043208D0A1
:1069E000D2071CBF11F8013B00F8013B01D30B8813
:1069F00003806046704700BF082A13D38B078DD0F1
:106A000010F003038AD0C3F10403D21ADB071CBFC2
:106A100011F8013B00F8013B80D331F8023B20F82C
:106A2000023B7BE7043AD9D3013A11F8013B00F865
:106A3000013BF9D20B7803704B7843708B788370ED
:106A400060467047F0B5304B1B681B06FBD42F4BDC
:106A50001B6813F08002F6D172B62D4B197800290D
:106A600050D02C4908684F688E68CD680C6938444E
:106A7000143130440968284420440844C0F34E00CF
:106A8000254940F400400860C86A0F6B4E6B8D6B5F
:106A9000CC6B3844403130440968284420440844D1
:106AA000C0F34E001D4940F40040086001F1081198
:106AB000143151F8140C51F8107C51F80C6C51F849
:106AC000085C51F8044C0968384430442844204498
:106AD0000844C0F34E00124940F400400860C86A00
:106AE0000F6B4E6B8D6BCC6B384440313044096872
:106AF000284420440844C0F34E000A4940F40040B2
:106B000008601A7062B6F0BD24B0034024B00B4098
:106B10003B95FF1F38B003402CB0034030B003401A
:106B20002CB00B4030B00B4010B5204B2048214911
:106B300060221A70E1225A701F4B204A1C78204BA9
:106B4000082C01D1012402E00A2C03D1392404606D
:106B5000132005E00C2C0CBF35243D2404601220CA
:106B6000086014601860174B17491B78174A03B167
:106B700001230B601360164B164A1978164B012936
:106B800001D880210BE0042901D8842107E00829DD
:106B900001D8852103E0102994BF86218721116047
:106BA00019600E4B01221A7010BD00BF0040074053
:106BB00008B003400CB003406587FF1F08B00B40CE
:106BC0000CB00B403E95FF1F20B0034020B00B409F
:106BD0006687FF1F24B0034024B00B403B95FF1F86
:106BE0000E4B1A7860B1BAB9012119700C4B1B78A1
:106BF00023B10C4B1A6003F500231A60FFF794BF12
:106C000052B11870064B1B78002BF7D0054B18605B
:106C100003F500231860F1E7704700BF3E95FF1FA2
:106C20003B95FF1F24B003400C2804D9102828BF2F
:106C30001020102307E00A2804D8092834BF0823AD
:106C40000A2300E00C23094AD9B2081A1070084A36
:106C50001078834208D0074B11701B7813B1064B94
:106C600000221A60FFF760BF704700BF3A95FF1F10
:106C70006587FF1F3B95FF1F24B0034010B5114BE4
:106C80001B7804460BB1FFF7DDFE012C0E4A01D83C
:106C9000002302E0042C02D8042313600EE0082C29
:106CA00003D805231360082308E0102C03D806231B
:106CB0001360102302E0072313602023034A13709C
:106CC00010BD00BF3B95FF1F24B003406687FF1F28
:106CD0000D2838B50FD9172801D80E380AE0A0F1D1
:106CE0001A03052B01D8093804E0A0F12203062B72
:106CF00047D81838C0B2244B1C5C244B1B780BB10E
:106D0000FFF7A0FE210614D472B6214B214D1C6062
:106D100001232B7062B672B61D4B1B681A0601D593
:106D20001D4B1FE02B78002BEFD062B601F0E0FF87
:106D3000F1E772B6194B1A4D1A6814F0400F14BFE0
:106D400022F0100242F010021A60164B04F03F02CB
:106D50001A6001232B7062B672B6124B1B681B06B9
:106D600008D5114B186800232B7062B60F4B1B78A7
:106D7000184138BD2B78002BDCD062B601F0B8FF8B
:106D8000EAE7002038BD00BFC8F800003B95FF1FB0
:106D900000B003403D95FF1F10B003400CB00B4006
:106DA0003C95FF1F00B00B4010B00B403A95FF1F01
:106DB000084B1A6842F480521A60074B1A78074B46
:106DC0000AB1802200E0C0221A70054B80F30C004B
:106DD000188070472C8004403E95FF1F21C00C4056
:106DE00000C00C40024B1B78DB07FBD5704700BF8F
:106DF000010002407FB5174B6A4603F110056E464D
:106E000018685968144603C40833AB422246F7D1C8
:106E1000114B1A7812F0020F1D4612D080229A717F
:106E200033229A7203225A7272B60C4C46F0010653
:106E30002046B04762B6237813F0700301D0237068
:106E400006E044F621632A78D20701D4013BFAD147
:106E500004B070BDE0F800000100024000000240F4
:106E6000B0F5006F10B5044609D2064B1B78DB075E
:106E700001D4FFF7BFFF04F1A054207810BD00201B
:106E800010BD00BF0100024040F2FE73984210B5F1
:106E9000044609D8054B1B78DB0701D4FFF7AAFF8E
:106EA00004F1A054208810BD002010BD0100024054
:106EB000024B187800F00100704700BF010002404B
:106EC000B0F5006F38B504460D460FD2084B1B785D
:106ED000DB0701D4FFF78EFF04F1A0542378AB4207
:106EE00004D02570BDE83840FFF77CBF38BD00BF37
:106EF0000100024038B540F2FE73984204460D4648
:106F00001ED8104B1B78DB0701D4FFF773FF14F07A
:106F1000010F04F1A05404D12388AB4210D0258086
:106F20000AE02378AB4202D02570FFF75BFF63785D
:106F30002D0AAB4204D06570BDE83840FFF752BF60
:106F400038BD00BF01000240024B1A6801321A60CE
:106F5000704700BF4095FF1F08B50B4C23685803CE
:106F600001D500F0E5FD2368590501D500F04EFC80
:106F700023681A0501D502F043F92368DB04ECD538
:106F800002F094FBE9E700BF3480044008B5FFF746
:106F9000E3FFFFFF014B10221A80704700200540DD
:106FA0007047FFFF024A1368184410601846704784
:106FB0006887FF1F002070474FF0FF3070474FF089
:106FC000FF307047EFF313839BB9EFF3108098B94C
:106FD000EFF3058323B10F2B04D9084A985C01E035
:106FE0004FF48070EFF311833BB1834238BF1846F2
:106FF00070474FF0FF30704718467047F0E300E0ED
:10700000044B054900221A600A60044A10601022ED
:107010001A60704714D0034004D0034000D00340EE
:10702000212810B518D80D4A52F8303093F8804214
:107030003CB1012211B183F8802010BD83F80021FA
:1070400010BD02EBC00043681A6811B142F00302A0
:1070500001E022F002021A6010BD00BFF0F800004B
:10706000212816D80B4A02EBC00301295B6852F8AD
:10707000302004D182F880124FF4A27208E0002080
:1070800082F8800211B94FF4807201E040F20312DD
:107090001A607047F0F80000282838B5604A0446A6
:1070A0000B4611D112780B2A04D8C2F10C0201FA56
:1070B00002F304E00C2A1CBF0C3A41FA02F3184612
:1070C000BDE83840FFF774BE11780125002B05FAA2
:1070D00001F2D8BF002102DD934205D32946FFF714
:1070E0009FFF2046294697E00338C2B2012A01D803
:1070F0004C4A06E0202C01D0192C01D14A4A00E06C
:107100004A4A126802FB0332CA401D287BD8DFE8D6
:1071100000F0575F4E337A7A212A7A7A7A7A7A7A2D
:107120007A7A7A3C450F187A707A7A7A7A7A7A671C
:107130003F4B1A6003F5973340F2444203F5FA736C
:107140005FE03C4B1A6003F5973340F2444203F58D
:10715000F87356E0384B1A6003F5973340F2444217
:1071600003F5F6734DE0354B1A6003F5973340F2A3
:10717000444203F5F47344E0314B1A6003F59F3346
:1071800040F2444203F5F0733BE02E4B1A6003F5E6
:107190009F3340F2444203F5EE7332E02A4B1A600B
:1071A00003F59F3340F2444203F5EC7329E0274B8B
:1071B0001A6003F59F3340F2444203F5EA7320E07E
:1071C000234B1A6003F580334FF45172203318E0DB
:1071D000204B1A6003F580334FF451721C3310E0DA
:1071E0001D4B1A60A3F5DB234FF45172A3F5F9632D
:1071F00007E01A4B1A60A3F5DB234FF45172A3F298
:10720000CC731A6038BD7F2B2046D4BF00210121EA
:10721000FFF706FF20460121BDE83840FFF720BFF9
:107220006C87FF1F0890034008800B4008800340D4
:1072300010800340188003402080034028800340D2
:107240003080034038800340408003404880034042
:10725000109003401890034010800B4018800B40A2
:1072600072B60B4B0B491A680B4B1B68096862B668
:10727000490102D5322A88BF0133C2F5BB326021F1
:10728000FF32B2FBF1F24FF47A7000FB032070473B
:1072900018E000E004ED00E04095FF1F38B504461B
:1072A000FFF7DEFF054624B938BD013C0AD005F5DD
:1072B0007A75FFF7D5FF401BB0F57A7FF5D201F064
:1072C00017FDF6E738BDFFFF1F4B4FF4000210B566
:1072D0001A604FF080721A604FF000721A604FF01F
:1072E00080621A604FF000621A60184B184A194CFD
:1072F00000204BF6FF7118605960282313609360DB
:107300001361936113629362136393630922226092
:1073100004F58054043420606160A360236144F864
:10732000042C04F5FE2420600B4801600B490B601F
:107330008B600B4B1A60FFF7F7FBFA20FFF7AEFFED
:10734000BDE8104000F0F2BE08E100E00480034018
:107350000C8003400080034008800B400C800B40F1
:1073600000800B40194B1A6842F480621A60184A78
:1073700000231370174A1370174A1370174A1370BB
:10738000174A1370174B40F213321A604FF45172C0
:107390005A60154BC0F344321A70C0F347125A704A
:1073A0000221042200F01F0098729A70D9745A7555
:1073B00088221A743C22DA700C4B40226FF44A7116
:1073C0001A700B444FF400521A6070473480044026
:1073D000CA95FF1F4995FF1FD095FF1FCB95FF1F33
:1073E0004895FF1F40A0044000A006402DE400E0A7
:1073F000134A937800F0030103F0EC030B434107B9
:1074000048BF43F01003937000F00F03042B0C49A6
:1074100003D18B7943F040038B715379C20603F09B
:10742000EF03074A48BF43F0100353719379810675
:1074300003F0EF0348BF43F010039371704700BFA0
:1074400000A0064008B5114B1B685B0500D408BDC1
:107450000F4B1A7802F0FF0312B101F049FCF7E775
:107460000C4A4FF4005111600B4A0C49D37040F2A2
:1074700003120A604A600A4A13700A4A13700A4BE0
:107480001B680BB101221A7008BD00BF3480044094
:107490004895FF1F84E100E000A0064040A00440A2
:1074A000CA95FF1F4995FF1F4495FF1F38B5044635
:1074B0000D4B1B7803F0FF05002BF9D1204601216D
:1074C000FFF7CEFD20462946FFF7AAFD074B53F8EC
:1074D0003420074B1A60074BA4229A709A7902F065
:1074E000DF029A7138BD00BF4895FF1FF0F8000019
:1074F000CC95FF1F00A006400D4A38B5146814F45F
:1075000080624FF0000410D021280A4D0AD80A4AA0
:10751000012152F830302B60FFF7A2FD2B681C7060
:10752000012038BD2C60204638BD104638BD00BF54
:10753000348004404495FF1FF0F800000E4B1B6898
:1075400013F4806316D012280C4B03D140F20231A1
:107550000B4A04E0142809D10A4A40F202311160B2
:107560005A7B42F001025A73012070475A7B02F0A5
:10757000FE025A73002070473480044000A0064089
:107580000CA0044014C00440F8B51F4B1B685A05FA
:10759000064638D51D4B1B6823B11D4A917941F031
:1075A0002001917101221A701A4B1C781444402C4E
:1075B0001F4628BF0024184D2B78A34218D1FFF78F
:1075C00001FD40280FDC124A13791B06F3D52B78F6
:1075D00012490133402B28BF0023C95CDBB2C9B27A
:1075E000D1712B70E7E7FF28E5DD01F081FBE2E7D1
:1075F0000A4BF6B21E550A4B01221A70044BE4B234
:10760000BC223C70DA70F8BD34800440CC95FF1F7A
:1076100000A00640D095FF1FCB95FF1F4A95FF1F86
:107620004895FF1F294B1B685A052DE9F04707466F
:107630008A4649D5264B1B6823B1264A917941F0E9
:107640002001917101221A703D4607EB0A039D4209
:1076500037D2DFF89080204E98F8004096F80090DE
:107660000134402C28BF00245FFA89F9A1451DD1BF
:10767000184BBC22DA70FFF7A5FC40280FDC154A36
:1076800013791B060FD5337814490133402B28BFDB
:107690000023C95CDBB2C9B2D171337003E0FF28AB
:1076A00001DD01F025FB33784B45E4D00B4B15F899
:1076B000012B1A550A4B0122E4B21A7088F80040D7
:1076C000C3E7044BBC22DA70BDE8F0873480044085
:1076D000CC95FF1F00A00640CB95FF1F4A95FF1FCA
:1076E0004895FF1FD095FF1F08B5034B1B7813B1BA
:1076F00001F0FEFAF9E708BD4895FF1F064A074B5F
:107700001B781078DBB2C0B283422CBF3F3000F14F
:10771000FF30C01A704700BFCB95FF1FD095FF1FE9
:10772000054B1878054B1B78C0B2DBB2984238BFC6
:107730004030C01A704700BFCA95FF1F4995FF1F10
:1077400010B5104B10491A780B78D2B2DBB29A42BE
:1077500014D00133402B28BF00230C48DCB2C05C9E
:107760000C700B490968C0B251B19A4238BF40321F
:10777000D31A1A2B04DC00230B7010BD4FF0FF301E
:1077800010BD00BFCA95FF1F4995FF1F8A95FF1FB7
:107790004495FF1F084B1A78084B1B78DBB29A42BE
:1077A00007D00133402B28BF0023054AD05CC0B26C
:1077B00070474FF0FF307047CA95FF1F4995FF1F74
:1077C0008A95FF1F0C4B1B685B0514D50B4BDA78B1
:1077D00002F0CB02DA7040225A74DA7842F03402B6
:1077E000DA70074B1A78074BD2B21A70064B1B6837
:1077F0000BB100221A7070473480044000A006408C
:107800004995FF1FCA95FF1F4495FF1F30B5394B9F
:107810001A7912F0300F31D072B69A7D02F0FF0063
:1078200022B9DA7940225A7462B627E062B6324A47
:10783000324913780978DBB2C9B214462D4AD5799A
:107840005A1C402A28BF00228A42EDB202D02C4B9B
:107850009D541346421E12F0FF00EFD1DAB222709F
:10786000284A126852B18B4236BFC1F14001C1EBC8
:1078700003035B18272BC4BF012313701D4BD9785A
:10788000C9B20D0620D51B791C061DD51E4B1F4AFB
:107890001D781378EDB2DBB21046AB420CD0154A1E
:1078A0000133402B14791A4C28BF0023E45CE4B266
:1078B000D471127D072AF0D9DBB203700D4B1A790F
:1078C000100644BF7C22DA70490612D5094B1A799A
:1078D00052060ED50F4A002111700F4A12681AB1D4
:1078E000997901F0DF01997100231370014B3C225B
:1078F000DA7030BD00A00640CA95FF1F4995FF1FF2
:107900008A95FF1F4495FF1FD095FF1FCB95FF1F42
:107910004A95FF1F4895FF1FCC95FF1F21282BD8A4
:10792000164B1B5CFF2B27D0154A02EBC000002131
:1079300042681160134A106840F020001060124A3B
:1079400001201160114998400860114841F8040C69
:10795000104911604FF4A07101397FF4FDAF116837
:107960008905FCD42022013A7FF4FDAF0A4A1BB2FC
:1079700032F8130080B270470020704700FA000010
:10798000F0F80000388004400050044008500440E3
:107990000000020380014A0000510440F0B50C4B86
:1079A0000C4C1A7842F0020504EBC50682F0010285
:1079B000706009481A700678002E0CBF8827C82707
:1079C00086F0010647EA0141067044F83510F0BD23
:1079D0003C96FF1F0080FF1FB496FF1F431E032B22
:1079E00010B510D872B6094A52F8230048B1416860
:1079F00042F82310064A018832F81340611A22F82F
:107A0000131062B610BD002010BD00BF2C96FF1FE2
:107A10001C98FF1F013803280AD872B6054B53F88B
:107A20002030002013B101305B68FBE762B670477D
:107A3000002070478096FF1F10B572B60123174AC9
:107A40001A4412F8012C12071CD59900144A52F856
:107A500031402CB902EB431308305860114B09E058
:107A600041F0010152F8314064B902EBC103083022
:107A700058600D4B42F831300C4B1A78013A1A70AD
:107A800062B610BD0133052BD9D162B6074B002277
:107A90001A70BDE8104000F0A7BB00BF58FB000003
:107AA0000080FF1F88004000C8004000AA96FF1F0A
:107AB000431E032B30B532D8194A400140F0100064
:107AC000104472B6174CE25C032A09D8DFE802F0D2
:107AD000160218050830022213E00830042210E0D4
:107AE0001148124A50F8234014B940F8231002E01C
:107AF00052F82300416042F823100FE0032200E017
:107B00000522E25410F0080F01F108030A884360CF
:107B10000CBF8823C82343EA0243036062B630BD2A
:107B20000080FF1FE895FF1F8096FF1F9096FF1FA4
:107B30002DE9F84FAB4F3C78E4B214F0040F3D460A
:107B400019D0A94B1B78A3B1A84A117801F0FF0303
:107B500021B1013BDBB2137003B900BEA44A117816
:107B600001F0FF0329B1013BDBB213700BB900F048
:107B70004FFC04233B7004F0080303F0FF02002BCA
:107B800000F067829B4B9C4C1A78D2B215094FEAE1
:107B9000920840F0E48104EBC803596854F8383087
:107BA000C3F38303013B0C2B00F2D681DFE813F013
:107BB00095019501D401D401D401D401D401D4019B
:107BC000B001D401D401D4010D008C4D0A684B687A
:107BD0008B486B6001218B4B44F838302A60DFF80A
:107BE0005082017092B240F2816000238242C8F854
:107BF00000302361A36117D8B2F5D06F80F01E81E9
:107C0000B2F5817F00F0CF8006D8802A00F0BA80DC
:107C1000822A00F0BB8031E140F202339A4200F048
:107C2000D180B2F5A06F1CE042F22100824200F048
:107C300051810ED8B2F5086F00F09E80B2F5106F3A
:107C400040F01C81684B6C4EAA781A7006F18009CE
:107C50000AE042F221218A4200F0088142F22133F7
:107C60009A4200F00F8109E1336A1B0603D5706A5E
:107C7000083800F0B9FA08364E45F5D10026B1466D
:107C8000DFF8B0A156F80A0028B1D0F804B000F02F
:107C9000ABFA5846F8E74AF806005B4BDFF898A1C4
:107CA000F05056F80A0028B1D0F804B000F09CFA61
:107CB0005846F8E7554B4AF80600F050544B23F865
:107CC0001900544B19F80320023A032A08D8DFE8B8
:107CD00002F002040204002200E0012203F809205D
:107CE00009F10109B9F1040F06F10406C8D14A4BA4
:107CF00000221A7001269A46484A494B32443344BE
:107D000012F8012C9B0012F0080F1A704FEA860936
:107D100025D000F04BFA38B104EB46130830586018
:107D2000404B44F8393006E09AF8003044F8390006
:107D300001338AF8003000F039FA49F0010338B114
:107D400004EBC302083050602E4A44F8332006E0AA
:107D500044F833009AF8003001338AF8003049F0D3
:107D60000202013649F003090023052E44F832309F
:107D700044F83930C0D186E01B4B2B4C1B78237064
:107D80000B4683E0284C237063707EE0AA88042AA7
:107D900074D8254C920023706370244B9B5C9E0723
:107DA00073D5217071E0AA8802F07F02042A65DC95
:107DB0006B88002B62D191001C4A0A44117821F093
:107DC000020159E0AA8802F07F02042A56DC6B887F
:107DD000002B53D19100154A0A44117841F0020159
:107DE0004AE000BF80200740B396FF1F3D96FF1F6B
:107DF000B596FF1F902007400080FF1FA096FF1F31
:107E0000B496FF1FC8004000D895FF1F9096FF1F33
:107E10001C98FF1FE895FF1FAA96FF1F58FB000044
:107E200030C8011088004000AB96FF1FC0200740FB
:107E3000D495FF1F2C96FF1F8096FF1F6A88A98884
:107E40009F4B53F8084CA3F10C00BCB133F80C6CF9
:107E5000964209D133F80A6C8E4205D1120A032AE0
:107E60000CBF2378038911E00C33EAE7954A1168C7
:107E7000954A1160A978954A117004E0944B0F223D
:107E80001A7027E000231C4600E00223EE88B3426C
:107E900038BF1E46402E34BF354640252046294671
:107EA000FFF77CFD761B2C4403D1402D12D13546C3
:107EB00003E0402E34BF3546402520462946FFF7D3
:107EC0006DFD761B2C4401D1402D03D1814AC8F8A9
:107ED000004016800122804B3DE0804B1A8842F220
:107EE00021039A4210D100237D4AC85C9854013383
:107EF000072BF9D11368862B02D17A4B0F221A7007
:107F000000200146FFF74AFD774B44F8383023E064
:107F1000764E3568B5B1DFF8BC81B8F80090B9F19C
:107F2000400F34BF4C46402428462146FFF736FD1B
:107F3000C4EB09039BB2A8F800300BB9402C00D168
:107F40002B193360654B1A88B2F5A06F04D100225B
:107F50005A709A78664B1A7001225F4B6CE004EB02
:107F6000C806013D736802F00802A3F10800EDB2F3
:107F700002F0FF01002A36D000F036F95D485E4B72
:107F800050F82520EAB1516840F8251002F10801A7
:107F90007160595D03290BD8DFE801F0020406087F
:107FA000032104E0022102E0052100E004215955EB
:107FB00016F0080F12880CBF8823C82343EA024337
:107FC00042E05A5D032A07D8DFE802F0404002048D
:107FD000002206E0012204E016F0080F0CBF022286
:107FE00003225A5532E054F83820120C23F8082C9A
:107FF00022B3DFF834E123F8061C43F8041C5EF8D2
:1080000025303E4913B94EF8250002E051F82530DD
:1080100058603B4B41F8250033F815100A4423F80B
:10802000152000F0C3F810B10830706006E0354B41
:1080300044F838001A7801321A7007E02A4B324AA5
:1080400016F0080F08BF134644F8383008233B7079
:1080500070E5E0071FD520492B482C4C02230B70FC
:108060002B4B1A702B4B186098602B48D8601A6104
:108070009A615C60164B0D2018702848FF2303702E
:108080002B700274264A1370264B9F221A7001230C
:108090000B70BDE8F88F210604D50D4B0D221A7028
:1080A00080232B70A20705D51C4B1A78D2B21A7008
:1080B00002232B70E30644BF10232B70BDE8F88F1A
:1080C00068FB00004095FF1F2C98FF1FC496FF1F00
:1080D000C0200740A896FF1F94200740A096FF1FCE
:1080E0002498FF1F3D96FF1FC8004000D495FF1F36
:1080F000982007408096FF1FE895FF1FD895FF1F27
:108100001C98FF1FAA96FF1F88004000EC95FF1FD8
:108110003C96FF1F0080FF1F4096FF1F88200740EE
:108120008C200740842007402C96FF1F08B501F0E3
:1081300025FB00221A4B0021D15098180832882ABA
:108140004160F7D1174A106840F48020106002F5B2
:1081500028326832C3F307201070C3F307401B0EA8
:1081600010751376FF2302F81C3C02F8143C02F849
:108170008C3C012302F8083C82F8641002F8183C99
:10818000094B70226FF450711A700B444FF4007257
:108190001A6003F1C04303F5C82310221A7008BD0A
:1081A0000080FF1F3480044049E400E072B60C4AAE
:1081B0001168B1FA81F30B2B02D962B60020704727
:1081C0004FF00040D84021EA0001116062B6054935
:1081D00048225343C8180022CA504260704700BF6B
:1081E0007087FF1F0084FF1F0C4B4822C31AB3FB8C
:1081F000F2F30B2B11D80A4A127822B1094A1278ED
:108200000AB1FFF719BC72B6074A4FF0004121FAD4
:1082100003F311681943116062B670470084FF1FB1
:10822000AA96FF1FB396FF1F7087FF1F10B5104C53
:1082300023686BB120684288531C0244147A028878
:10824000934212D3FFF7D0FF094B00221A600DE0D2
:10825000084B1B7813B94FF0FF3010BD0320FFF718
:10826000BDFB20600028E5D1F5E74380204610BD26
:10827000C096FF1FB396FF1F10B50B4C236813B1B8
:1082800023686BB902E0094B1B7813B94FF0FF303C
:1082900010BD0320FFF7A2FB20600028F0D1F5E716
:1082A0005A881344187A10BDC096FF1FB396FF1F5B
:1082B000044B9888044B1B681BB11A885B88D31A3F
:1082C000184470471C98FF1FC096FF1F2DE9F84304
:1082D0002D4E012307460C463370002C4FD02B4DFA
:1082E0002B68A9462BBB4AF2F928294B1B7803F0CF
:1082F000FF020BB9327015E00420FFF78BFB072853
:1083000008D801233370FFF751FFC9F8000080B986
:108310001D4B1870B8F101081E4B01D01A782AB114
:1083200001221A704FF0FF30BDE8F88300F0E0FC46
:10833000DBE72968174A488800231370C0F1400220
:10834000944238BF224600F1080C10448C44488007
:10835000A41A934204D0F85C0CF803000133F8E748
:108360001F444B883F2B06D940230B800420FFF786
:108370009FFB00232B60084B05221A70ADE7347079
:108380002046BDE8F88300BFB696FF1FB896FF1FD2
:10839000B396FF1FBC96FF1FB596FF1F07B502AB34
:1083A000012103F8010D1846FFF790FF03B05DF8B7
:1083B00004FBFFFF2DE9F041114B1B78F3B1114E87
:1083C000114B3468114D01271F7098464CB100279E
:1083D00063882F70042023802146FFF769FB3760F4
:1083E00009E0FFF7E3FE014620B104202C70FFF7FF
:1083F0005FFB00E02F70002388F80030BDE8F081BB
:10840000B396FF1FB896FF1FB696FF1FB596FF1FC6
:1084100038B50E4B1B7803F0FF05ABB90C4C216847
:1084200031B14B880B800420FFF742FB256038BD3B
:10843000FFF7BCFE014620B10420BDE83840FFF73D
:1084400037BB044B01221A7038BD00BFB696FF1F20
:10845000B896FF1FB596FF1F08B50368C9B21B6821
:10846000984708BD08B50368C9B21B68984708BD9E
:1084700008B50368C9B21B68984708BD08B503680A
:10848000C9B21B68984708BD4B0803F1376000F577
:10849000D830B0FBF1F0FEF765BF10B54B0803F123
:1084A000376000F5D8301446B0FBF1F0FEF75AFF04
:1084B0002046BDE81040FEF79BBFFEF7C3BF08464D
:1084C000FEF7F4BF08B50846FFF716F8003018BFEE
:1084D000012008BD08B50846FFF730F8003018BF86
:1084E000012008BDFFF71CB9FFF754B9FFF728B901
:1084F000FFF7FAB8FFF766B9FFF700B908B5084605
:10850000FFF742F8012008BD08B50846FFF73CF820
:10851000012008BD10B5084614461146FFF782F841
:10852000204610BD38B508460D4602F03AFC044618
:1085300021462846FFF776F8204638BD7047FFFFF2
:10854000044B00221A714FF47A711A73024A99602F
:108550001A607047C896FF1F30FA000008B503681C
:10856000C9B21B68984708BD08B50368C9B21B6843
:10857000984708BD08B50368C9B21B68984708BD8D
:1085800008B50368C9B21B68984708BD4B0803F1DA
:10859000376000F5D830B0FBF1F000F0F7BB10B554
:1085A0004B0803F1376000F5D8301446B0FBF1F00A
:1085B00000F0ECFB2046BDE8104000F02DBC00F0C0
:1085C00055BC084600F086BC08B5084600F09EFC85
:1085D000003018BF012008BD08B5084600F0B8FCFF
:1085E000003018BF012008BD00F094BD00F0CCBDE4
:1085F00000F0A0BD00F072BD00F0DEBD00F078BD5F
:1086000008B5084600F0C2FC012008BD08B50846C0
:1086100000F0BCFC012008BD10B508461446114608
:1086200000F0FEFC204610BD38B508460D4602F0AD
:10863000B8FB04462146284600F0F2FC204638BD2F
:108640007047FFFF044B00221A714FF47A711A73BE
:10865000024A99601A607047D896FF1F88FA000096
:1086600008B50368C9B21B68984708BD08B5036818
:10867000C9B21B68984708BD08B50368C9B21B6832
:10868000984708BD08B50368C9B21B68984708BD7C
:108690004B0803F1B76000F55840B0FBF1F000F073
:1086A00033BE10B54B0803F1B76000F558401446CF
:1086B000B0FBF1F000F028FE2046BDE8104000F0CD
:1086C00065BE00F08DBE084600F0BEBE08B5084687
:1086D00000F0D6FE003018BF012008BD08B50846DE
:1086E00000F0F0FE003018BF012008BD00F07ABF96
:1086F00000F0B2BF00F086BF00F058BF00F0C4BF6A
:1087000000F05EBF08B5084600F0FAFE012008BD83
:1087100008B5084600F0F4FE012008BD10B5084673
:108720001446114600F036FF204610BD38B5084605
:108730000D4602F036FB04462146284600F02AFF8B
:10874000204638BD7047FFFF044B00221A714FF4DA
:108750007A711A73024A99601A607047E896FF1F8F
:10876000E0FA000008B5034B01221A60024B1B68B7
:10877000984708BD0C7103400097FF1F08B5034BD5
:1087800001221A60024B5B68984708BD1C710340C8
:108790000097FF1F08B5034B01221A60024B9B682C
:1087A000984708BD2C7103400097FF1F08B5034B85
:1087B00001221A60024BDB68984708BD3C710340F8
:1087C0000097FF1F054B1A6842F400021A60044B21
:1087D00000221A60034B01221A7070473C8004404B
:1087E00000700340FC96FF1F064B01221A6003F540
:1087F00088333C331A6822F400021A60024B0022CC
:108800001A70704700700340FC96FF1FF0B5457862
:10881000134C144F2B011A194260134A9E1886609C
:10882000066947F8256000259D501951032199508C
:108830004378427B4433DBB2037303F1604303F5B7
:10884000644301211A70027B53119B0003F16043C2
:1088500003F5614302F01F0201FA02F21A60F0BD53
:10886000007103400097FF1F08710340F8B50C4BDF
:108870001B7806460F460BB9FFF7A4FF0024094DED
:10888000625DE3B23AB9304673703946FFF7BEFF16
:1088900001202855F8BD0134042CF0D10020F8BD8A
:1088A000FC96FF1FF896FF1F8268002310B5136027
:1088B000027B0121541102F01F0201FA02F2084961
:1088C00041F82420074A41785354D15C31B901332F
:1088D000042BFAD1BDE81040FFF786BF10BD00BFE2
:1088E00080E100E0F896FF1F037870B504460D465E
:1088F00016461BB1FFF7D8FF0023237025612046E1
:108900003146FFF7B3FF10B10123237000E0207060
:10891000207870BD037810B504460BB1FFF7C4FF93
:108920000023237010BD08B5FDF7CEFBFDF7F0FC6A
:1089300000F0DEF9FAE7F8B506460C468F18002578
:10894000BC4207D0336814F8011B1B6830469847B7
:108950000544F5E72846F8BD2DE9F04100258C686F
:108960008AB0074688462E4694B12B46404601A958
:10897000212200F092F93B68202C34BF22462022AD
:108980005B68384601A91544A41A98470644EBE7EA
:1089900030460AB0BDE8F08107B5064B1B88ADF83C
:1089A0000430036801A95B680222984703B05DF8B0
:1089B00004FB00BF30FB000008B503685B68984704
:1089C000002008BD0EB403B503AA52F8041B01929F
:1089D00002F02EFC02B05DF804EB03B0704770B5F6
:1089E00005468AB022B90368C9B21B6898472CE0D3
:1089F000012A08BF0A2221B930228DF8252021241E
:108A000013E02124B1FBF2F002FB1011C9B20929D5
:108A10000AAE94BF303137312644C9B206F8241C5F
:108A2000014610B1013CE4B2ECE733B1013CE4B2E1
:108A30000AAB23442D2203F8242C2B6801A95B6880
:108A400028462144C4F1220298470AB070BD00298B
:108A5000BABF49422D2300230A22FFF7C0BFFFF708
:108A600027BCFFF7E3BBFFF707BCFFF7A3BC084633
:108A7000FFF794BC08461146FFF728BC7047FFFF7C
:108A8000044B00221A714FF47A711A73024A9960EA
:108A90001A6070471097FF1F40FB000010B5044696
:108AA000006802F04FF8204610BD38B504460D4668
:108AB0000068013102F018F910B184E821000120AA
:108AC00038BD43688B4210B5044606D2FFF7EDFF70
:108AD00020B1A3680BB922681370012010BDF8B54E
:108AE00004460F46154622B9036803B11A700023E5
:108AF0000BE01146FFF7E5FF064640B9206810B1CC
:108B000002F020F8266000236360A36004E0A56003
:108B10002068394602F03DF92046F8BD38B50023FB
:108B2000044603604360836003730D4639B1084611
:108B300002F037F9294602462046FFF7D0FF2046CB
:108B400038BD38B5054600680C4660B16A688B6868
:108B50009A4206D3096802F01CF9A368AB600023AF
:108B60000AE001F0EFFF23682B6063686B60A36885
:108B7000AB60002323606360A36038BD81420B4675
:108B800003D009689A68FFF7AABF7047884210B5FA
:108B9000044601D0FFF7D5FF204610BD38B5054685
:108BA0000C4641B1084602F0FCF821460246284630
:108BB000FFF795FF00E0A960284638BD10B50023F7
:108BC00086B004460360436083600373084601A9CE
:108BD00000F0CCF8204601A9FFF7E0FF204606B0E0
:108BE00010BD07B500238DF80410012201A98DF8EE
:108BF0000530FFF774FF03B05DF804FB10B50023E8
:108C000004460360436083600373FFF7EAFF204676
:108C100010BD70B504460E4685685AB11544294604
:108C2000FFF74FFF30B12068A3683146184402F0C7
:108C3000B0F8A560204670BD0B4609689A68FFF73A
:108C4000E8BF13B500238DF80410012201A90446E2
:108C50008DF80530FFF7DDFF204602B010BD8268B9
:108C600008B50B4612B919B9012008BD11B903683E
:108C7000187802E0006802F082F8D0F1010038BFF5
:108C8000002008BD8368994203D2006810B1405C9F
:108C9000704700207047FFF7F5BF38B50C469AB112
:108CA00091B181688B4202D30023237038BDC91A69
:108CB000551E8D4228BF0D4601682A46194420469C
:108CC00002F08EF80023635538BD38B504680546B8
:108CD0003CB114F8010B20B102F06EFA04F8010C5B
:108CE000F7E7284638BD006808B101F0D8BE7047E4
:108CF00010B50E4C2378BBB901232370FFF7D8FAC7
:108D000008B1FFF7BBFEFEF70BFD08B1FFF716FC3D
:108D100000F000FA08B1FFF793FC00F063FC08B123
:108D2000FFF710FD0023237010BD00BF2097FF1F29
:108D300010B50023B0FBF2F402FB1400092894BF25
:108D400030303730C0B2C85420460CB10133F1E79F
:108D5000CA18547022469A4206DA885CCC5C8C545D
:108D6000C8540132013BF6E7084610BD031E10B59A
:108D70000C4603DBBDE81040FFF7DABF2D2001F8F9
:108D8000010B5842FFF7D4FF204610BD194B1A685B
:108D900042F400621A60184A00231370174A1370D5
:108DA000174A1370174A1370174A1370174B40F283
:108DB00013321A604FF451725A60154BC0F34432AB
:108DC0001A70C0F347125A7000F01F0004220221EB
:108DD00098729A70D9745A7588221A743C22DA7083
:108DE0000C4B40221A70A3F22B334FF400421A604E
:108DF000704700BF348004409297FF1F2997FF1FE0
:108E00009897FF1F9397FF1F2897FF1F0CB00440F0
:108E100000B006402FE400E0134A937800F003010D
:108E200003F0EC030B43410748BF43F0100393707A
:108E300000F00F03042B0C4903D18B7943F040035E
:108E40008B715379C20603F0EF03074A48BF43F022
:108E5000100353719379810603F0EF0348BF43F089
:108E600010039371704700BF00B0064008B5114B66
:108E70001B681B0500D408BD0F4B1A7802F0FF03D6
:108E800012B1FFF735FFF7E70C4A4FF400411160CC
:108E90000B4A0C49D37040F203120A604A600A4A36
:108EA00013700A4A13700A4B1B680BB101221A7027
:108EB00008BD00BF348004402897FF1F84E100E014
:108EC00000B006400CB004409297FF1F2997FF1F87
:108ED0002497FF1F38B50446094B1B7803F0FF05A4
:108EE000002BF9D120460121FEF7BAF82046294689
:108EF000FEF796F8034B53F83420034B1A6038BD45
:108F00002897FF1FF0F800009497FF1F0D4A38B50F
:108F1000146814F400624FF0000410D021280A4DA8
:108F20000AD80A4A012152F830302B60FEF798F82F
:108F30002B681C70012038BD2C60204638BD1046BF
:108F400038BD00BF348004402497FF1FF0F80000B4
:108F50000B4B1B6813F4006310D01728094B09D181
:108F6000094A40F2023111605A7B42F001025A7301
:108F7000012070475A7B02F0FE025A7300207047AE
:108F80003480044000B0064008B00440F8B51D4BE2
:108F90001B681A05064633D51B4B1B680BB1012213
:108FA0001A701A4B1C780134282C1F4628BF002445
:108FB000174D2B78A34218D1FEF704F840280FDC98
:108FC000144A13791B06F3D52B7813490133282B48
:108FD00028BF0023C95CDBB2C9B2D1712B70E7E7AF
:108FE000FF28E5DDFFF784FEE2E70B4BF6B21E55E6
:108FF0000A4B01221A70074BE4B2BC223C70DA70B3
:10900000F8BD00BF348004409497FF1F9897FF1F5E
:109010009397FF1F00B006402A97FF1F2897FF1F56
:10902000274B1B681A052DE9F04707468A4644D5A9
:10903000244B1B680BB101221A703D4607EB0A0353
:109040009D4237D2DFF890801F4E98F8004096F886
:1090500000900134282C28BF00245FFA89F9A1452B
:109060001DD11A4BBC22DA70FDF7ACFF40280FDC93
:10907000164A13791B060FD5337815490133282B6F
:1090800028BF0023C95CDBB2C9B2D171337003E0E1
:10909000FF2801DDFFF72CFE33784B45E4D00C4B65
:1090A00015F8012B1A550B4B0122E4B21A7088F8FF
:1090B0000040C3E7054BBC22DA70BDE8F08700BF73
:1090C000348004409497FF1F9397FF1F00B0064021
:1090D0002A97FF1F2897FF1F9897FF1F08B5034B7C
:1090E0001B7813B1FFF704FEF9E708BD2897FF1FAF
:1090F000064A074B1B781078DBB2C0B283422CBF04
:10910000273000F1FF30C01A704700BF9397FF1F50
:109110009897FF1F054B1878054B1B78C0B2DBB240
:10912000984238BF4030C01A704700BF9297FF1F67
:109130002997FF1F10B5104B10491A780B78D2B23F
:10914000DBB29A4214D00133402B28BF00230C48D5
:10915000DCB2C05C0C700B490968C0B251B19A42D4
:1091600038BF4032D31A1A2B04DC00230B7010BD19
:109170004FF0FF3010BD00BF9297FF1F2997FF1FD0
:109180005297FF1F2497FF1F084B1A78084B1B7834
:10919000DBB29A4207D00133402B28BF0023054A97
:1091A000D05CC0B270474FF0FF3070479297FF1FFE
:1091B0002997FF1F5297FF1F0C4B1B681B0514D5E7
:1091C0000B4BDA7802F0CB02DA7040225A74DA786C
:1091D00042F03402DA70074B1A78074BD2B21A7099
:1091E000064B1B680BB100221A7070473480044094
:1091F00000B006402997FF1F9297FF1F2497FF1F7B
:1092000030B5374B1A7912F0300F31D072B69A7DE3
:1092100002F0FF0022B9DA7940225A7462B627E0E0
:1092200062B6304A304913780978DBB2C9B21446C5
:109230002B4AD5795A1C402A28BF00228A42EDB217
:1092400002D02A4B9D541346421E12F0FF00EFD16C
:10925000DAB22270264A126852B18B4236BFC1F18F
:109260004001C1EB03035B18272BC4BF012313701C
:109270001B4BD978C9B20C0620D51B7918061DD511
:109280001C4B1D4A1D781378EDB2DBB21046AB4281
:109290000CD0134A0133282B1479184C28BF002313
:1092A000E45CE4B2D471127D072AF0D9DBB203701A
:1092B0000B4B1A79120644BF7C22DA704B060ED58E
:1092C000074B1A7912F0400F194608D00C4B0022B8
:1092D0001A700C4B1B6803B11A703C23CB7030BD65
:1092E00000B006409297FF1F2997FF1F5297FF1F5C
:1092F0002497FF1F9897FF1F9397FF1F2A97FF1F21
:109300002897FF1F9497FF1F174B1A6842F480524B
:109310001A60164A00231370154A1370154A137009
:10932000154A1370154A1370154A40F21331116033
:109330004FF451715160134AC0F344311170C0F3BE
:10934000471100F01F0051709072937013742C231A
:10935000D3700D4B40226FF44B711A700B444FF4D5
:1093600000321A60704700BF348004400A98FF1F23
:10937000A197FF1F1098FF1F0B98FF1FA097FF1FBB
:1093800008C0044000C0064031E400E0134A93786E
:1093900000F0030103F0EC030B43410748BF43F027
:1093A0001003937000F00F03042B0C4903D18B7949
:1093B00043F040038B715379C20603F0EF03074A71
:1093C00048BF43F0100353719379810603F0EF0314
:1093D00048BF43F010039371704700BF00C00640C0
:1093E00008B5114B1B68DB0400D408BD0F4B1A787D
:1093F00002F0FF0312B1FFF77BFCF7E70C4A4FF4D2
:10940000003111600B4A0C49D37040F203120A601C
:109410004A600A4A13700A4A13700A4B1B680BB160
:1094200001221A7008BD00BF34800440A097FF1FBE
:1094300084E100E000C0064008C004400A98FF1F15
:10944000A197FF1F9C97FF1F38B50446094B1B7857
:1094500003F0FF05002BF9D120460121FDF700FEA6
:1094600020462946FDF7DCFD034B53F83420034B1F
:109470001A6038BDA097FF1FF0F800000C98FF1F7E
:109480000D4A38B5146814F480524FF0000410D01F
:1094900021280A4D0AD80A4A012152F830302B609F
:1094A000FDF7DEFD2B681C70012038BD2C602046C6
:1094B00038BD104638BD00BF348004409C97FF1F64
:1094C000F0F800000B4B1B6813F4805310D00E28EB
:1094D000094B09D1094A40F2023111605A7B42F02E
:1094E00001025A73012070475A7B02F0FE025A7340
:1094F000002070473480044000C0064004C004408F
:10950000F8B51D4B1B68DA04064633D51B4B1B68A8
:109510000BB101221A701A4B1C780134282C1F46FB
:1095200028BF0024174D2B78A34218D1FDF74AFD20
:1095300040280FDC144A13791B06F3D52B78134906
:109540000133282B28BF0023C95CDBB2C9B2D1711B
:109550002B70E7E7FF28E5DDFFF7CAFBE2E70B4BDF
:10956000F6B21E550A4B01221A70074BE4B2AC2228
:109570003C70DA70F8BD00BF348004400C98FF1FC7
:109580001098FF1F0B98FF1F00C00640A297FF1FF7
:10959000A097FF1F38B504464518AC4204D014F814
:1095A000010BFFF7ADFFF8E738BDFFFF08B5034B30
:1095B0001B7813B1FFF79CFBF9E708BDA097FF1FCD
:1095C000064A074B1B781078DBB2C0B283422CBF2F
:1095D000273000F1FF30C01A704700BF0B98FF1F03
:1095E0001098FF1F054B1878054B1B78C0B2DBB2F3
:1095F000984238BF4030C01A704700BF0A98FF1F1A
:10960000A197FF1F10B5104B10491A780B78D2B2F2
:10961000DBB29A4214D00133402B28BF00230C4800
:10962000DCB2C05C0C700B490968C0B251B19A42FF
:1096300038BF4032D31A1A2B04DC00230B7010BD44
:109640004FF0FF3010BD00BF0A98FF1FA197FF1F0A
:10965000CA97FF1F9C97FF1F084B1A78084B1B786F
:10966000DBB29A4207D00133402B28BF0023054AC2
:10967000D05CC0B270474FF0FF3070470A98FF1FB0
:10968000A197FF1FCA97FF1F054B1A78054BD2B24F
:109690001A70054B1B680BB100221A70704700BF8F
:1096A000A197FF1F0A98FF1F9C97FF1F10B5294B1A
:1096B0001A79920620D5284AD87913782749013398
:1096C000402B097828BF00238B42C0B203D0244925
:1096D000C854D9B21170234A116869B1224A12786C
:1096E000D2B2934236BFC2F14002C2EB03039B18D1
:1096F000272BC4BF01230B70164AD178C9B20C06C0
:1097000016D51379180613D5184B17481C7803780B
:10971000DBB29C4202D16C23D37009E00133282BC9
:1097200028BF0023124CE45CDBB2E4B2D4710370B6
:109730004B060ED5074B1A7912F0400F194608D088
:109740000C4B00221A700C4B1B6803B11A702C23AF
:10975000CB7010BD00C006400A98FF1FA197FF1FE5
:10976000CA97FF1F9C97FF1F0B98FF1F1098FF1FA2
:10977000A297FF1FA097FF1F0C98FF1F1FB572B67F
:10978000154B70221A70154A412111700F2102F8F1
:10979000011C80221A701A781206FCD5104B18682A
:1097A00062B6104B984298BF0A2301AC98BF584349
:1097B00021460A22FFF7BCFA0023E15C0A4A29B1DC
:1097C00002EB430001330A2B4180F6D101335B00E9
:1097D000137004B010BD00BF00000240070002403B
:1097E000080002407F969800FC87FF1FFFFFFFFFE5
:1097F0002DE9F043DFF8EC808BB004460D4600F015
:1098000073F898F90030013306460F4638D02046E9
:10981000294600F0E5F9002832D0204629462AA33F
:10982000D3E9002300F02CFE814600282DD12046EC
:10983000294627A3D3E9002300F004FE00B398F9DA
:1098400000102548CDF8209004260022002302298C
:10985000CDE90445CDE9024500960190CDE9062306
:109860002CD0684600F0C2F940B3089B1BB101F050
:1098700035F9089B0360DDE906010BB0BDE8F08314
:10988000304639460BB0BDE8F083134B98F8001012
:10989000019303220023CDE90445CDE9024500925E
:1098A000089329B90D4B4FF06042CDE90623D8E764
:1098B0000B4B00220229CDE90623D2D101F00EF98B
:1098C00022230360D1E700BFEF39FAFE422E864023
:1098D00051302DD5104987C0B0FB0000FFFFEF4786
:1098E0000000F07F1288FF1F2DE9F04FDFF8E4C27F
:1098F00021F00047674583B004460D4602460B46FB
:109900004FEAD1760DD9DFF8D0C2674526D9C1F329
:10991000130707431DD1002E40F0158103B0BDE8A9
:10992000F08FA54B9F4200F2CF80A44B9F4200F2E4
:10993000E1808BA3D3E9002300F060F90022A04B63
:1099400000F09EFD002800F008819D4B204629462E
:10995000002200F053F903B0BDE8F08F82A3D3E9F1
:10996000002300F08DFD002840F0C78020462946E6
:109970007FA3D3E9002300F065FD002840F0E380D9
:109980007DA3D3E900232046294600F0E9FA8D4B58
:1099900003EBC606D6E9002300F030F900F07AFDAB
:1099A000804600F077FA76A3D3E9002306460F46F7
:1099B00000F0D6FA02460B462046294600F01CF974
:1099C00071A3D3E90023CDE900013046394600F008
:1099D000C7FA82468B46DDE9000152465B4600F03D
:1099E0000BF904460D4622462B462046294600F038
:1099F000B7FA67A3D3E9002306460F4600F0B0FA92
:109A000065A3D3E9002300F0F7F832463B4600F0A7
:109A1000A7FA63A3D3E9002300F0F0F832463B46EF
:109A200000F09EFA60A3D3E9002300F0E5F8324687
:109A30003B4600F095FA5EA3D3E9002300F0DEF880
:109A400032463B4600F08CFA02460B462046294639
:109A500000F0D2F806460F462046294632463B46DD
:109A6000B8F1000F51D000F07BFA324604460D46A3
:109A70003B4600204FF0804100F0BEF802460B4606
:109A80002046294600F096FB02460B4650465946B2
:109A900000F0B2F8DDE9002300F0AEF80B46024614
:109AA0004749002000F0A8F86FF47F7398454FDA1B
:109AB00008F57A7801EB085100224FF0B87300F0F6
:109AC0004FFA03B0BDE8F08F3F4B9F423FF658AFCF
:109AD0003E4BF4002344D3E9002300F08DF83C4BC7
:109AE000C6F101081C44CDE90001D4E900ABC6EB86
:109AF000080870E74FF0000875E719A1D1E90001E7
:109B000002460B4600F02CFA08E700F029FA002282
:109B100080468946304639464FF0804300F06CF865
:109B200002460B464046494600F044FB22462B467F
:109B300000F062F802460B460020214900F05CF874
:109B400003B0BDE8F08F0020002103B0BDE8F08F26
:109B500001EB085103B0BDE8F08F804643E700BF3A
:109B60009C7500883CE4377EEF39FAFE422E864031
:109B700051302DD5104987C0FE822B654715F73F20
:109B80000000E0FE422EE63F763C7935EF39EA3DB3
:109B9000D0A4BE726937663EF16BD2C541BDBB3EF3
:109BA0002CDE25AF6A56113F93BDBE166CC1663FD1
:109BB0003E5555555555C53F422ED63FFFFF2F3ECA
:109BC0000000F03FB8FB0000B1A2F03FD8FB00005E
:109BD000C8FB0000412E8640FFFFEF7FAFF30080FF
:109BE00041F0004101F58010C00F70470020704720
:109BF00081F0004102E000BF83F0004330B54FEA3E
:109C000041044FEA430594EA050F08BF90EA020FAA
:109C10001FBF54EA000C55EA020C7FEA645C7FEA3D
:109C2000655C00F0E2804FEA5454D4EB5555B8BF60
:109C30006D420CDD2C4480EA020281EA030382EAD1
:109C4000000083EA010180EA020281EA0303362D63
:109C500088BF30BD11F0004F4FEA01314FF4801C36
:109C60004CEA113102D0404261EB410113F0004F48
:109C70004FEA03334CEA133302D0524263EB4303FF
:109C800094EA050F00F0A780A4F10104D5F1200E9D
:109C90000DDB02FA0EFC22FA05F2801841F10001F8
:109CA00003FA0EF2801843FA05F359410EE0A5F1CC
:109CB00020050EF1200E012A03FA0EFC28BF4CF0FD
:109CC000020C43FA05F3C01851EBE37101F00045B3
:109CD00007D54FF0000EDCF1000C7EEB00006EEBC0
:109CE0000101B1F5801F1BD3B1F5001F0CD349084A
:109CF0005FEA30004FEA3C0C04F101044FEA4452A1
:109D000012F5800F80F09A80BCF1004F08BF5FEA27
:109D1000500C50F1000041EB045141EA050130BD07
:109D20005FEA4C0C404141EB010111F4801FA4F1AA
:109D30000104E9D191F0000F04BF01460020B1FAFF
:109D400081F308BF2033A3F10B03B3F120020CDA37
:109D50000C3208DD02F1140CC2F10C0201FA0CF015
:109D600021FA02F10CE002F11402D8BFC2F1200C7A
:109D700001FA02F120FA0CFCDCBF41EA0C01904030
:109D8000E41AA2BF01EB0451294330BD6FEA040479
:109D90001F3C1CDA0C340EDC04F11404C4F1200264
:109DA00020FA04F001FA02F340EA030021FA04F376
:109DB00045EA030130BDC4F10C04C4F1200220FACD
:109DC00002F001FA04F340EA0300294630BD21FA0B
:109DD00004F0294630BD94F0000F83F4801306BFD1
:109DE00081F480110134013D4EE77FEA645C18BFC5
:109DF0007FEA655C29D094EA050F08BF90EA020F5C
:109E000005D054EA000C04BF1946104630BD91EA53
:109E1000030F1EBF0021002030BD5FEA545C05D156
:109E20004000494128BF41F0004130BD14F5800495
:109E30003CBF01F5801130BD01F0004545F0FE4109
:109E400041F470014FF0000030BD7FEA645C1ABF3E
:109E5000194610467FEA655C1CBF0B46024650EA75
:109E6000013406BF52EA033591EA030F41F40021A1
:109E700030BD00BF90F0000F04BF0021704730B527
:109E80004FF4806404F132044FF000054FF00001FC
:109E900050E700BF90F0000F04BF0021704730B5BD
:109EA0004FF4806404F1320410F0004548BF404292
:109EB0004FF000013EE700BF42004FEAE2014FEAE7
:109EC00031014FEA02701FBF12F07F4393F07F4FC2
:109ED00081F06051704792F0000F14BF93F07F4FF4
:109EE000704730B54FF4607401F0004521F0004137
:109EF00020E700BF50EA010208BF704730B54FF0BD
:109F000000050AE050EA010208BF704730B511F0C1
:109F1000004502D5404261EB41014FF4806404F1F9
:109F200032045FEA915C3FF4DCAE4FF003025FEA7B
:109F3000DC0C18BF03325FEADC0C18BF033202EB03
:109F4000DC02C2F1200300FA03FC20FA02F001FA5D
:109F500003FE40EA0E0021FA02F11444C1E600BFFC
:109F600070B54FF0FF0C4CF4E06C1CEA11541DBFAF
:109F70001CEA135594EA0C0F95EA0C0F00F0DEF87A
:109F80002C4481EA030621EA4C5123EA4C5350EA5F
:109F9000013518BF52EA033541F4801143F48013B0
:109FA00038D0A0FB02CE4FF00005E1FB02E506F041
:109FB0000042E0FB03E54FF00006E1FB03569CF096
:109FC000000F18BF4EF0010EA4F1FF04B6F5007F9C
:109FD00064F5407404D25FEA4E0E6D4146EB06060E
:109FE00042EAC62141EA55514FEAC52040EA5E5097
:109FF0004FEACE2EB4F1FD0C88BFBCF5E06F1ED841
:10A00000BEF1004F08BF5FEA500E50F1000041EB77
:10A01000045170BD06F0004646EA010140EA020024
:10A0200081EA0301B4EB5C04C2BFD4EB0C0541EA46
:10A03000045170BD41F480114FF0000E013C00F35B
:10A04000AB8014F1360FDEBF002001F0004170BD7F
:10A05000C4F10004203C35DA0C341BDC04F1140498
:10A06000C4F1200500FA05F320FA04F001FA05F224
:10A0700040EA020001F0004221F0004110EBD370F1
:10A0800021FA04F642EB06015EEA430E08BF20EA1D
:10A09000D37070BDC4F10C04C4F1200500FA04F3C0
:10A0A00020FA05F001FA04F240EA020001F0004152
:10A0B00010EBD37041F100015EEA430E08BF20EAC5
:10A0C000D37070BDC4F1200500FA05F24EEA020E0D
:10A0D00020FA04F301FA05F243EA020321FA04F03C
:10A0E00001F0004121FA04F220EA020000EBD370F3
:10A0F0005EEA430E08BF20EAD37070BD94F0000FF3
:10A100000FD101F00046400041EB010111F4801F26
:10A1100008BF013CF7D041EA060195F0000F18BFD7
:10A12000704703F00046520043EB030313F4801F13
:10A1300008BF013DF7D043EA0603704794EA0C0FCD
:10A140000CEA135518BF95EA0C0F0CD050EA4106E3
:10A1500018BF52EA4306D1D181EA030101F0004160
:10A160004FF0000070BD50EA410606BF1046194688
:10A1700052EA430619D094EA0C0F02D150EA013694
:10A1800013D195EA0C0F05D152EA03361CBF1046D5
:10A1900019460AD181EA030101F0004141F0FE4174
:10A1A00041F470014FF0000070BD41F0FE4141F4F8
:10A1B000780170BD70B54FF0FF0C4CF4E06C1CEAF8
:10A1C00011541DBF1CEA135594EA0C0F95EA0C0FAD
:10A1D00000F0A7F8A4EB050481EA030E52EA033568
:10A1E0004FEA013100F088804FEA03334FF0805589
:10A1F00045EA131343EA12634FEA022245EA1115B6
:10A2000045EA10654FEA00260EF000419D4208BF66
:10A21000964244F1FD0404F5407402D25B084FEA13
:10A220003202B61A65EB03055B084FEA32024FF4BF
:10A2300080104FF4002CB6EB020E75EB030E22BF1C
:10A24000B61A754640EA0C005B084FEA3202B6EBDC
:10A25000020E75EB030E22BFB61A754640EA5C008B
:10A260005B084FEA3202B6EB020E75EB030E22BF1B
:10A27000B61A754640EA9C005B084FEA3202B6EB1C
:10A28000020E75EB030E22BFB61A754640EADC00DB
:10A2900055EA060E18D04FEA051545EA16754FEA3D
:10A2A00006164FEAC30343EA52734FEAC2025FEA5B
:10A2B0001C1CC0D111F4801F0BD141EA00014FF0EA
:10A2C00000004FF0004CB6E711F4801F04BF0143BB
:10A2D0000020B4F1FD0C88BFBCF5E06F3FF6AFAED7
:10A2E000B5EB030C04BFB6EB020C5FEA500C50F167
:10A2F000000041EB045170BD0EF0004E4EEA1131EA
:10A3000014EB5C04C2BFD4EB0C0541EA045170BDF0
:10A3100041F480114FF0000E013C90E645EA060E34
:10A320008DE60CEA135594EA0C0F08BF95EA0C0F62
:10A330003FF43BAF94EA0C0F0AD150EA01347FF4AA
:10A3400034AF95EA0C0F7FF425AF104619462CE781
:10A3500095EA0C0F06D152EA03353FF4FDAE1046E4
:10A36000194622E750EA410618BF52EA43067FF435
:10A37000C5AE50EA41047FF40DAF52EA43057FF4C5
:10A38000EBAE12E74FF0FF3C06E000BF4FF0010CD0
:10A3900002E000BF4FF0010C4DF804CD4FEA410C34
:10A3A0007FEA6C5C4FEA430C18BF7FEA6C5C1BD001
:10A3B00001B050EA410C0CBF52EA430C91EA030F82
:10A3C00002BF90EA020F0020704710F1000F91EADF
:10A3D000030F58BF994208BF90422CBFD8176FEAAD
:10A3E000E37040F0010070474FEA410C7FEA6C5C7B
:10A3F00002D150EA013C07D14FEA430C7FEA6C5C82
:10A40000D6D152EA033CD3D05DF8040B704700BFAD
:10A410008446104662468C461946634600E000BFFB
:10A4200001B5FFF7B7FF002848BF10F1000F01BDCD
:10A430004DF808EDFFF7F4FF0CBF012000205DF898
:10A4400008FB00BF4DF808EDFFF7EAFF34BF01201D
:10A4500000205DF808FB00BF4DF808EDFFF7E0FFB6
:10A4600094BF012000205DF808FB00BF4DF808ED07
:10A47000FFF7CEFF94BF012000205DF808FB00BF6E
:10A480004DF808EDFFF7C4FF34BF012000205DF850
:10A4900008FB00BF4FEA410212F5001215D211D598
:10A4A0006FF47873B3EB625212D94FEAC12343F0D1
:10A4B000004343EA505311F0004F23FA02F018BF53
:10A4C000404270474FF00000704750EA013005D11C
:10A4D00011F0004008BF6FF0004070474FF00000DF
:10A4E000704700BF4FEA4102B2F1E04324BFB3F529
:10A4F000001CDCF1FE5C0DD901F0004C4FEAC002FB
:10A500004CEA5070B2F1004F40EB830008BF20F0DE
:10A510000100704711F0804F21D113F13872BCBF98
:10A5200001F00040704741F480114FEA5252C2F1ED
:10A530001802C2F1200C10FA0CF320FA02F018BF36
:10A5400040F001004FEAC1234FEAD32303FA0CFC89
:10A5500040EA0C0023FA02F34FEA4303CCE77FEA18
:10A56000625307D150EA01331EBF4FF0FE4040F462
:10A570004000704701F0004040F0FE4040F4000011
:10A58000704700BF80F0004002E000BF81F0004152
:10A5900042001FBF5FEA410392EA030F7FEA226C89
:10A5A0007FEA236C6AD04FEA1262D2EB1363C1BF19
:10A5B000D218414048404140B8BF5B42192B88BF88
:10A5C000704710F0004F40F4000020F07F4018BFAB
:10A5D000404211F0004F41F4000121F07F4118BFCB
:10A5E000494292EA030F3FD0A2F1010241FA03FC73
:10A5F00010EB0C00C3F1200301FA03F100F000435B
:10A6000002D5494260EB4000B0F5000F13D3B0F122
:10A61000807F06D340084FEA310102F10102FE2A91
:10A6200051D2B1F1004F40EBC25008BF20F0010001
:10A6300040EA03007047490040EB000010F4000FAF
:10A64000A2F10102EDD1B0FA80FCACF1080CB2EB42
:10A650000C0200FA0CF0AABF00EBC25052421843A1
:10A66000BCBFD0401843704792F0000F81F4000146
:10A6700006BF80F400000132013BB5E74FEA410319
:10A680007FEA226C18BF7FEA236C21D092EA030F85
:10A6900004D092F0000F08BF0846704790EA010FFF
:10A6A0001CBF0020704712F07F4F04D1400028BF2C
:10A6B00040F00040704712F100723CBF00F500000E
:10A6C000704700F0004343F0FE4040F40000704744
:10A6D0007FEA226216BF08467FEA236301464202F0
:10A6E00006BF5FEA412390EA010F40F48000704703
:10A6F0004FF0000304E000BF10F0004348BF4042A9
:10A700005FEA000C08BF704743F0964301464FF0E4
:10A7100000001CE050EA010208BF70474FF0000340
:10A720000AE000BF50EA010208BF704711F0004381
:10A7300002D5404261EB41015FEA010C02BF844651
:10A740000146002043F0B64308BFA3F18053A3F5B0
:10A750000003BCFA8CF2083AA3EBC25310DB01FAF7
:10A7600002FC634400FA02FCC2F12002BCF1004F7B
:10A7700020FA02F243EB020008BF20F0010070470C
:10A7800002F1200201FA02FCC2F1200250EA4C0060
:10A7900021FA02F243EB020008BF20EADC707047A6
:10A7A0004FF0FF0C1CEAD0521EBF1CEAD15392EAB4
:10A7B0000C0F93EA0C0F6FD01A4480EA010C400290
:10A7C00018BF5FEA41211ED04FF0006343EA5010EA
:10A7D00043EA5111A0FB01310CF00040B1F5000F2C
:10A7E0003EBF490041EAD3715B0040EA010062F1DB
:10A7F0007F02FD2A1DD8B3F1004F40EBC25008BFC5
:10A8000020F00100704790F0000F0CF0004C08BFE2
:10A8100049024CEA502040EA51207F3AC2BFD2F1AF
:10A82000FF0340EAC250704740F400004FF00003BD
:10A83000013A5DDC12F1190FDCBF00F000407047F7
:10A84000C2F10002410021FA02F1C2F1200200FA35
:10A8500002FC5FEA310040F1000053EA4C0308BFFC
:10A8600020EADC70704792F0000F00F0004C02BF4D
:10A87000400010F4000F013AF9D040EA0C0093F0C8
:10A88000000F01F0004C02BF490011F4000F013B22
:10A89000F9D041EA0C018FE70CEAD15392EA0C0F90
:10A8A00018BF93EA0C0F0AD030F0004C18BF31F0FB
:10A8B000004CD8D180EA010000F00040704790F0D1
:10A8C000000F17BF90F0004F084691F0000F91F075
:10A8D000004F14D092EA0C0F01D142020FD193EA3B
:10A8E0000C0F03D14B0218BF084608D180EA0100C3
:10A8F00000F0004040F0FE4040F40000704740F09F
:10A90000FE4040F4400070474FF0FF0C1CEAD0526C
:10A910001EBF1CEAD15392EA0C0F93EA0C0F69D0C8
:10A92000A2EB030280EA010C49024FEA402037D033
:10A930004FF0805343EA111143EA10130CF000402A
:10A940008B4238BF5B0042F17D024FF4000C8B421A
:10A9500024BF5B1A40EA0C00B3EB510F24BFA3EBFA
:10A96000510340EA5C00B3EB910F24BFA3EB9103CA
:10A9700040EA9C00B3EBD10F24BFA3EBD10340EA24
:10A98000DC001B0118BF5FEA1C1CE0D1FD2A3FF66A
:10A9900050AF8B4240EBC25008BF20F0010070471F
:10A9A0000CF0004C4CEA50207F32C2BFD2F1FF03C2
:10A9B00040EAC250704740F400004FF00003013AF3
:10A9C00037E792F0000F00F0004C02BF400010F497
:10A9D000000F013AF9D040EA0C0093F0000F01F0AB
:10A9E000004C02BF490011F4000F013BF9D041EACD
:10A9F0000C0195E70CEAD15392EA0C0F08D1420200
:10AA00007FF47DAF93EA0C0F7FF470AF084676E7D2
:10AA100093EA0C0F04D14B023FF44CAF08466EE7AB
:10AA200030F0004C18BF31F0004CCAD130F0004279
:10AA30007FF45CAF31F000437FF43CAF5FE700BFD1
:10AA40004FEA4002B2F1FE4F0FD34FF09E03B3EB3B
:10AA500012620DD94FEA002343F0004310F0004F7B
:10AA600023FA02F018BF404270474FF000007047D1
:10AA700012F1610F01D1420205D110F0004008BF70
:10AA80006FF0004070474FF00000704703460846E3
:10AA9000194600F013B800210A2200F035BA00214F
:10AAA0000A2200F031BAFFFF0A460349034608684C
:10AAB000194600F072B800BF7488FF1F70B5064CCD
:10AAC00006460D4613462CB131462A460220AFF306
:10AAD000008070BD204670BD00000000014B18686A
:10AAE000704700BF7488FF1F70B50E4B0E4DED1AF6
:10AAF000AD1000241E46AC4204D056F824209047E6
:10AB00000134F8E705F03EF9084D094BED1AAD1098
:10AB100000241E46AC4204D056F82420904701344D
:10AB2000F8E770BD90FD000090FD0000A8FD00005A
:10AB300090FD0000024B0146186800F081B800BF8C
:10AB40007488FF1F024B0146186800F035B800BF3B
:10AB50007488FF1F814270B501D300230EE08C186A
:10AB6000A042FAD28518134613F1FF3305D35142A0
:10AB700066182944F65CCE54F6E770BD934203D0C4
:10AB8000CC5CC4540133F9E770BD024403469342E0
:10AB900002D003F8011BFAE7704738B502FB01F455
:10ABA000214600F04DF8054618B100212246FFF776
:10ABB000ECFF284638BDFFFF30B500293CD051F8E6
:10ABC000042C0B1F1D49002AB8BF9B180A680C46AD
:10ABD00012B95A600B6030BD93420DD219685818F3
:10ABE000904203D15A581144426819605A60236058
:10ABF00030BD994203D80A4651680029F9D114683A
:10AC000015199D420AD11B682344D018884213604D
:10AC100012D10868034413604B680CE002D90C237E
:10AC2000036030BD18681C188C4203D10C68496859
:10AC3000204418605960536030BD00BF1898FF1F52
:10AC400070B5CD1C25F0030508350C2D38BF0C253B
:10AC5000002D06463FDB8D423DD3214B1C68184634
:10AC60002146A1B10B685B1B0ED40B2B03D90B60E3
:10AC7000CC18CD501FE08C4202D1626802601AE00D
:10AC80004B6863600C4616E00C464968E9E7154CD2
:10AC900023681BB9304600F031F820602946304661
:10ACA00000F02CF8431C014615D0C41C24F003040A
:10ACB00084420AD1256004F10B00231D20F0070017
:10ACC000C31A0BD05A42E25070BD3046611A00F0F0
:10ACD00015F80130EED10C233360002070BD00BFA9
:10ACE0001898FF1F1498FF1F0A4603490346086877
:10ACF000194600F010BD00BF7488FF1F38B5064C20
:10AD00000023054608462360FCF74CF9431C02D19A
:10AD1000236803B12B6038BD3098FF1F0EB400B517
:10AD20009CB04FF40271ADF814106FF00041049123
:10AD300007914FF6FF711DABADF81610084953F897
:10AD4000042B029006900868019302A900F046F9CE
:10AD5000029B00221A701CB05DF804EB03B0704730
:10AD60007488FF1FC9B2024610F8013B1BB18B4229
:10AD7000F9D1104670470029FBD01846704710F8EB
:10AD8000012B11F8013B012A28BF9A42F7D0D01AB3
:10AD90007047034611F8012B03F8012B002AF9D163
:10ADA0007047034613F8012B002AFBD1181A01380B
:10ADB000704770B592B10B4605461C7810F8016BD0
:10ADC000B44201F1010101D1012A03D128781B7895
:10ADD000C01A70BD013A002CEDD1F7E7104670BDE6
:10ADE00010B5034632B111F8014B03F8014B013A9B
:10ADF000002CF7D11A44934203D0002103F8011B21
:10AE0000F9E710BD84463F482DE9F04FD0F80080A7
:10AE10000E46344614F8015B08EB0500407800F05C
:10AE2000080000F0FF0708B12646F2E72D2D03D1F8
:10AE3000B41C7578012703E02B2D04BF7578B41C72
:10AE400033F010000DD1302D08D1207800F0DF0054
:10AE5000582851D165781023023402E0002B08BF36
:10AE60000A23002F0CBF6FF0004A4FF0004ABAFBD4
:10AE7000F3F9002603FB19AA304608EB050B9BF8F3
:10AE800001B01BF0040F01D0303D0BE01BF0030BB1
:10AE90001BD0BBF1010F14BF4FF0570B4FF0370B16
:10AEA000CBEB05059D4210DAB6F1FF3F0AD04845CD
:10AEB00006D801D1554503DC03FB0050012601E013
:10AEC0004FF0FF3614F8015BD7E7731C0CD1002F4D
:10AED0004FF022030CBF6FF000404FF00040CCF861
:10AEE00000302AB9BDE8F08F07B1404242B106B147
:10AEF000611E1160BDE8F08F002B08BF0823B0E78A
:10AF0000BDE8F08F7888FF1F30B51346044A054628
:10AF10000C46106829462246BDE83040FFF772BF54
:10AF20007488FF1F2DE9F0478D68AB4281460C46BF
:10AF300092461F4643D38B8913F4906F3DD0266809
:10AF40000969C1EB06086669022206EB460696FB14
:10AF5000F2F608F101023A44964238BF16465B0504
:10AF60000FD53146FFF76CFE054698B12169424680
:10AF7000FBF7CEFCA38923F4906343F08003A38105
:10AF800013E0324600F0C7FB054670B94846216918
:10AF9000FFF712FE0C23C9F80030A38943F04003E9
:10AFA000A3814FF0FF30BDE8F0872561666145441D
:10AFB000C8EB06062560A6603D46AF4200D23D467E
:10AFC0002A4620685146FFF7C5FDA3685B1BA360B6
:10AFD00023681D4425600020BDE8F0872DE9F0437B
:10AFE0009DB0074603938B891C060D4616460CD56B
:10AFF0000B6953B94021FFF723FE2860286110B97F
:10B000000C233B60C8E040236B610023099320239D
:10B010008DF8293030238DF82A3033461C4613F83A
:10B02000012B1AB9B4EB06090FD002E0252AF5D19D
:10B03000F8E73846294632464B46FFF773FF0130A2
:10B0400000F0A580099B4B4409932378002B00F066
:10B050009E8000234FF0FF320493079305920693DE
:10B060008DF853301A9304F101094C464D4E217866
:10B070003046052200F040FB09F10109049B28B18C
:10B08000861B0120B04003430493EEE7D90644BF7A
:10B0900020228DF853201A0744BF2B228DF853200D
:10B0A00022782A2A02D0079B21460EE0039A111D1E
:10B0B00012680391002A01DB079204E0524243F038
:10B0C00002030792049301340AE00C46013122780E
:10B0D000303A092A03D80A2000FB0323F5E7079337
:10B0E00023782E2B1AD163782A2B0AD1039B1A1DA1
:10B0F0001B680392002B04F10204B8BF4FF0FF332A
:10B100000BE0611C00230C4601312278303A092AF9
:10B1100003D80A2000FB0323F5E70593224E21788C
:10B120003046032200F0E8FA30B1861B049B402031
:10B13000B04003430493013421781C488DF8281053
:10B140000622661C00F0D8FA88B1194B33B9039B6C
:10B15000073323F007030833039314E003AB009392
:10B16000384604A92A46134BAFF3008007E003AB2F
:10B170000093384604A92A460E4B00F0D9F8B0F1E6
:10B18000FF3F804603D0099B4344099345E7AB89C1
:10B190005B0601D4099801E04FF0FF301DB0BDE817
:10B1A000F08300BFF0FB0000F6FB0000FAFB00009C
:10B1B0000000000025AF0000044B1B6803445B78CF
:10B1C00003F00303012B08BF203070477888FF1F6E
:10B1D0002DE9F041ADF5047D1D464FF400730F4697
:10B1E00090460393044618B183690BB900F01AFA2C
:10B1F00004AE00952046314603AA434600F0F4FA17
:10B20000054670B1204639462A46039B00F0A4F952
:10B21000B542039003D020462946FFF7CDFC0398A2
:10B2200001E04FF0FF300DF5047DBDE8F081FFFF38
:10B2300030B51346044A05460C4610682946224696
:10B24000BDE83040FFF7C4BF7488FF1F2DE9F84305
:10B2500015461F468A680B69DDF820809A42A8BF10
:10B2600013462B6091F8432006460C460AB1013381
:10B270002B602368990602D52B6802332B60236864
:10B2800013F006091DD094F843302268003318BF2C
:10B29000012392061FD5E1185A1C302081F8430083
:10B2A000224494F8451082F84310023313E03046EC
:10B2B000394604F119020123C047013007D009F1D2
:10B2C0000109E2682B68D31A9945F0DBDBE74FF000
:10B2D000FF30BDE8F8833046394604F14302C047E9
:10B2E0000130F4D023682A68E16803F00603042BD8
:10B2F00008BFC2EB01052369A2680CBF25EAE5750A
:10B3000000259A42C4BFC3EB0203ED184FF00009B9
:10B31000A9450ADA3046394604F11A020123C0472A
:10B320000130D4D009F10109F2E70020BDE8F8832B
:10B330002DE9FF470E7E0C9D6E2E80460C469146F1
:10B340009A4601F1430000F0A58011D8632E22D067
:10B3500009D8002E00F0AF80582E40F0BF8081F851
:10B3600045607B4A4FE0642E1ED0692E1CD0B5E0AC
:10B37000732E00F0A48009D86F2E2BD0702E40F0D1
:10B38000AD800B6843F020030B6038E0752E21D0B0
:10B39000782E34D0A2E02B681A1D1B682A6001F1B8
:10B3A000420781F842309DE022682B6812F0800F3E
:10B3B00003D01A1D2A601D6805E05106F9D51A1D33
:10B3C0002A60B3F90050002D39DA2D236D4284F83C
:10B3D000433034E022682B6812F0800F03D01A1D2E
:10B3E0002A601D6804E05206F9D51A1D2A601D88DE
:10B3F000237E574A6F2B14BF0A2308231BE07823B0
:10B40000544A84F845302368296813F0800F01F10D
:10B4100004062E6001D00D6802E05F06FBD50D88A2
:10B42000DE0744BF43F0200323601DB9236823F0E7
:10B43000200323601023002184F8431001E0444AD4
:10B440000A236668A660002E03DB216821F0040150
:10B45000216005B96EB104F14201B5FBF3F603FBBF
:10B4600016550F46555D01F801593546002EF4D1A9
:10B4700000E00746082B0AD12368DD0707D562687C
:10B4800023699A4203DC302307F8013C013FC01BCB
:10B4900020612CE009682B68626911F0800F04D0EC
:10B4A000191D29601B681A6005E04906F8D5191DA9
:10B4B00029601B681A8000232361074617E02B6868
:10B4C0001A1D2A601F683846FFF76BFC636820610D
:10B4D000984288BF23612369636005E004F1420755
:10B4E00084F8426001232361002384F84330CDF8BF
:10B4F00000A04046214603AA4B46FFF7A7FE0130B5
:10B5000002D14FF0FF301FE0404649463A462369DA
:10B51000D0470130F5D023689B0705D4E068039B32
:10B520009842B8BF18460FE00025E268039BD31A83
:10B530009D42F3DA4046494604F119020123D047FF
:10B540000130DED00135F0E704B0BDE8F08700BF80
:10B5500001FC000012FC000038B5074C0546002035
:10B560002060084611461A46FDF726FA431C02D110
:10B57000236803B12B6038BD3098FF1FF8B507462C
:10B5800000F1480494B1A5686668013E0CD4AB890B
:10B59000012B07D9B5F90E30013303D038462946BF
:10B5A00000F0E4F96835F0E72468EBE7F8BDFFFF49
:10B5B000002310B5044603604360836081814366C5
:10B5C000C28103614361836119465C300822FFF741
:10B5D000DCFA054B6362054BA362054BE362054B46
:10B5E0002462236310BD00BF63B7000085B700006D
:10B5F000BDB70000E1B7000070B54B1E68255D4384
:10B600000E4605F17401FFF71BFB044640B1002113
:10B6100080E842000C30A06005F16802FFF7B5FA3F
:10B62000204670BD836910B5044633BB8364C36490
:10B630000365124B124A1B688262984204BF0123C1
:10B64000836100F01FF86060204600F01BF8A060E6
:10B65000204600F017F80421E06000226068FFF740
:10B66000A7FFA06809210122FFF7A2FFE0681221CD
:10B670000222FFF79DFF0123A36110BDECFB000038
:10B680007DB50000F8B51B4B1E68B369074613B9BA
:10B690003046FFF7C7FF4836B4687368013B04D4EF
:10B6A000B4F90C5075B16834F8E733682BB93846F3
:10B6B0000421FFF7A1FF306008B13668ECE70C23E6
:10B6C0003B60F8BD4FF6FF73E3810123A3816566FC
:10B6D0002560A560656025616561A56104F15C0078
:10B6E00029460822FFF751FA6563A563A564E5645E
:10B6F0002046F8BDECFB000010B5C9B202449042F0
:10B70000034606D01C788C4200F10100F7D11846A0
:10B7100010BD002010BDF8B5064614460D4621B9EF
:10B720001146BDE8F840FFF78BBA1AB9FFF744FAA3
:10B730002046F8BD00F056F9A0420ED23046214610
:10B74000FFF77EFA074650B129462246FBF7E0F89C
:10B7500030462946FFF730FA01E02846F8BD384662
:10B76000F8BD10B50C46B1F90E1000F045F90028EF
:10B7700003DB636D0344636510BDA38923F4805329
:10B78000A38110BD2DE9F0411D468B89DB050746DD
:10B790000C46164605D5B1F90E100022022300F022
:10B7A0000FF9A389B4F90E1023F48053A38138460E
:10B7B00032462B46BDE8F041FFF7CEBE10B50C4631
:10B7C000B1F90E1000F0FCF8431CA38903D123F457
:10B7D0008053A38110BD43F48053A381606510BDE5
:10B7E000B1F90E1000F02EB830B515469BB01468B4
:10B7F00029B124B14FF4C162ADF80C2005E04FF43B
:10B8000022720024ADF80C202146002C00910491F6
:10B8100003DA8B230360002012E04FF6FF72ADF8CD
:10B820000E2069461A461E9B02940594FFF7D6FB2C
:10B83000031E4FF0000003DB2B60009B1870049880
:10B840001BB030BD38B5064C0023054608462360C2
:10B85000FBF7B2FB431C02D1236803B12B6038BD58
:10B860003098FF1F8A892DE9F041054610070C46E4
:10B8700057D44B68002B02DC0B6C002B18DDE66AFA
:10B88000B6B102F48052002392B22F682B600AB145
:10B89000626D10E0216A28460123B047411C024630
:10B8A00009D12B683BB11D2B01D0162B46D12F603F
:10B8B0000020BDE8F081A3895B0705D56368D21A33
:10B8C000636B0BB1236CD21AE66A216A2846002307
:10B8D000B047461CA28905D12B681BB11D2B01D096
:10B8E000162B19D100236360D1042369236004D58A
:10B8F000421C01D12B6803B96065616B2F60002980
:10B90000D6D004F14403994202D02846FFF754F9F7
:10B9100000206063BDE8F08142F04002A281BDE8F2
:10B92000F0810E69002EC3D00B680E60C6EB0308D1
:10B9300093070CBF4B6900238B6012E0A38943F08F
:10B940004003A3814FF0FF30BDE8F081A76A216A70
:10B95000284632464346B8470028EFDD0644C0EB90
:10B960000808B8F1000FF1DCA2E7FFFF38B50B695A
:10B9700005460C46DBB118B183690BB9FFF752FEDF
:10B980000C4B9C4201D16C6808E00B4B9C4201D1EE
:10B99000AC6803E0094B9C4208BFEC68B4F90C307A
:10B9A0002BB128462146BDE83840FFF75BBF002099
:10B9B00038BD00BF24FD000044FD000064FD000010
:10B9C00038B5074C054600202060084611461A4647
:10B9D000FBF7F5FA431C02D1236803B12B6038BD95
:10B9E0003098FF1F51F8040C002802DA04390B5874
:10B9F000184404387047FFFF38B5074C054600204F
:10BA00002060084611461A46FBF7D4FA431C02D1BF
:10BA1000236803B12B6038BD3098FF1F5B42542070
:10BA20004E4F542050524553454E545D00415400F2
:10BA30004F4B0041542B4E414D453F0041542B503C
:10BA40005357443F00556E61626C6520746F2069E6
:10BA50006E697469616C697A65204254206D6F6407
:10BA6000756C65206265636175736520626F6172D4
:10BA700064206D6F64656C20697320756E737570DA
:10BA8000706F727465642E20426F617264204D6F16
:10BA900064656C3A0041542B4E414D453D25730081
:10BAA0000D0A0041542B505357443D253034690052
:10BAB00043616C6C6F63206661696C203200417475
:10BAC00074656D7074656420746F205045454B201B
:10BAD0006F7574736964652062756666657221208E
:10BAE0005065656B696E6720706F736974696F6EFE
:10BAF0003A2000417474656D7074656420746F2021
:10BB0000676574204152524956414C2054494D4575
:10BB100020666F7220612062797465206F7574737E
:10BB20006964652062756666657221205472796960
:10BB30006E6720746F206765742074696D65206678
:10BB40006F7220706F736974696F6E3A2000417470
:10BB500074656D7074656420746F207075726765AC
:10BB6000206D6F7265207468616E20746865206353
:10BB70006F6E74656E7473206F66207468652062E2
:10BB800075666665722120547269656420746F2041
:10BB900070757267653A200044756D70696E672034
:10BBA00043697263756C61722042756666657200E6
:10BBB0004275666665722073697A652069733A20FA
:10BBC0000043616C6C6F63206661696C00FFFFFF6E
:10BBD000000000000100000002000000030000005F
:10BBE000040000000600000007000000080000003C
:10BBF000090000000A0000000B0000000C0000001B
:10BC00000D0000000E0000000F00000010000000FA
:10BC100011000000120000001300000014000000DA
:10BC200015000000160000001800000019000000B8
:10BC30001A0000001B0000001C0000001D00000096
:10BC40001E0000001F000000200000002100000076
:10BC50002200000023000000240000002500000056
:10BC60002600000027000000280000002900000036
:10BC70002A0000002B0000002C0000002D00000016
:10BC80002E0000002F0000003000000031000000F6
:10BC900032000000330000003400000035000000D6
:10BCA00036000000370000003800000039000000B6
:10BCB0003A0000003B0000003C0000003D00000096
:10BCC0003E0000003F000000400000004100000076
:10BCD0004200000043000000440000004400000057
:10BCE000450000004600000047000000480000003A
:10BCF000490000004A0000004B0000004C0000001A
:10BD00004D0000004E0000004F00000050000000F9
:10BD100051000000520000005300000054000000D9
:10BD200055000000560000005700000058000000B9
:10BD300058000000590000005A0000005B0000009D
:10BD40005C0000005D0000005E0000005F0000007D
:10BD5000600000006100000062000000630000005D
:10BD6000640000006500000066000000660000003E
:10BD70006700000068000000690000006A00000021
:10BD80006B0000006C0000006D0000006E00000001
:10BD90006F000000700000007100000072000000E1
:10BDA00072000000730000007400000075000000C5
:10BDB00076000000770000007800000079000000A5
:10BDC0007A0000007B0000007C0000007C00000086
:10BDD0007D0000007E0000007F0000008000000069
:10BDE0008100000082000000830000008400000049
:10BDF000850000008600000086000000870000002B
:10BE000088000000890000008A0000008B0000000C
:10BE10008C0000008D0000008E0000008F000000EC
:10BE20008F000000900000009100000092000000D0
:10BE300093000000940000009500000096000000B0
:10BE40009700000097000000980000009900000093
:10BE50009A0000009B0000009C0000009D00000074
:10BE60009E0000009F0000009F000000A000000056
:10BE7000A1000000A2000000A3000000A400000038
:10BE8000A5000000A6000000A7000000A700000019
:10BE9000A8000000A9000000AA000000AB000000FC
:10BEA000AC000000AD000000AE000000AF000000DC
:10BEB000AF000000B0000000B1000000B2000000C0
:10BEC000B3000000B4000000B5000000B6000000A0
:10BED000B6000000B7000000B8000000B900000084
:10BEE000BA000000BB000000BC000000BD00000064
:10BEF000BE000000BE000000BF000000C000000047
:10BF0000C1000000C2000000C3000000C400000027
:10BF1000C5000000C5000000C6000000C70000000A
:10BF2000C8000000C9000000CA000000CB000000EB
:10BF3000CC000000CD000000CD000000CE000000CD
:10BF4000CF000000D0000000D1000000D2000000AF
:10BF5000D3000000D4000000D4000000D500000091
:10BF6000D6000000D7000000D8000000D900000073
:10BF7000DA000000DB000000DC000000DC00000054
:10BF8000DD000000DE000000DF000000E000000037
:10BF9000E1000000E2000000E3000000E400000017
:10BFA000E4000000E5000000E6000000E7000000FB
:10BFB000E8000000E9000000EA000000EB000000DB
:10BFC000EB000000EC000000ED000000EE000000BF
:10BFD000EF000000F0000000F1000000F20000009F
:10BFE000F3000000F3000000F4000000F500000082
:10BFF000F6000000F7000000F8000000F900000063
:10C00000FA000000FB000000FC000000FC00000043
:10C01000FD000000FE000000FF0000000001000025
:10C020000101000002010000030100000401000002
:10C0300004010000050100000601000007010000E6
:10C0400008010000090100000A0100000B010000C6
:10C050000C0100000D0100000D0100000E010000A8
:10C060000F0100001001000011010000120100008A
:10C07000130100001401000015010000160100006A
:10C08000170100001701000018010000190100004D
:10C090001A0100001B0100001C0100001D0100002E
:10C0A0001E0100001F01000020010000210100000E
:10C0B00021010000220100002301000024010000F2
:10C0C00025010000260100002701000028010000D2
:10C0D000290100002A0100002B0100002C010000B2
:10C0E0002D0100002D0100002E0100002F01000095
:10C0F0003001000031010000320100003301000076
:10C100003401000035010000360100003701000055
:10C1100038010000390100003A0100003B01000035
:10C120003B0100003C0100003D0100003E01000019
:10C130003F010000400100004101000042010000F9
:10C1400043010000440100004501000046010000D9
:10C150004701000048010000490100004A010000B9
:10C160004B0100004C0100004D0100004E01000099
:10C170004F0100004F01000050010000510100007C
:10C18000520100005301000054010000550100005D
:10C19000560100005701000058010000590100003D
:10C1A0005A0100005B0100005C0100005D0100001D
:10C1B0005E0100005F0100006001000061010000FD
:10C1C00062010000630100006401000065010000DD
:10C1D00066010000670100006801000069010000BD
:10C1E0006A0100006B0100006C0100006D0100009D
:10C1F0006E0100006F01000070010000710100007D
:10C20000720100007301000074010000750100005C
:10C21000760100007701000078010000790100003C
:10C220007A0100007B0100007C0100007D0100001C
:10C230007E0100007F0100008001000081010000FC
:10C2400082010000830100008401000085010000DC
:10C250008601000088010000890100008A010000B9
:10C260008B0100008C0100008D0100008E01000098
:10C270008F01000090010000910100009201000078
:10C280009301000094010000950100009601000058
:10C2900097010000980100009A0100009B01000036
:10C2A0009C0100009D0100009E0100009F01000014
:10C2B000A0010000A1010000A2010000A3010000F4
:10C2C000A4010000A6010000A7010000A8010000D1
:10C2D000A9010000AA010000AB010000AC010000B0
:10C2E000AD010000AE010000B0010000B10100008E
:10C2F000B2010000B3010000B4010000B50100006C
:10C30000B6010000B7010000B9010000BA01000049
:10C31000BB010000BC010000BD010000BE01000027
:10C32000C0010000C1010000C2010000C301000003
:10C33000C4010000C5010000C7010000C8010000E1
:10C34000C9010000CA010000CB010000CC010000BF
:10C35000CE010000CF010000D0010000D10100009B
:10C36000D2010000D4010000D5010000D601000078
:10C37000D7010000D8010000DA010000DB01000055
:10C38000DC010000DD010000DF010000E001000031
:10C39000E1010000E2010000E4010000E50100000D
:10C3A000E6010000E7010000E9010000EA010000E9
:10C3B000EB010000EC010000EE010000EF010000C5
:10C3C000F0010000F2010000F3010000F4010000A0
:10C3D000F5010000F7010000F8010000F90100007C
:10C3E000FB010000FC010000FD010000FF01000056
:10C3F000000200000102000003020000040200002D
:10C400000502000007020000080200000902000007
:10C410000B0200000C0200000D0200000F020000E1
:10C4200010020000120200001302000014020000BB
:10C430001602000017020000190200001A02000094
:10C440001B0200001D0200001E020000200200006E
:10C450002102000023020000240200002602000046
:10C4600027020000280200002A0200002B02000020
:10C470002D0200002E0200003002000031020000F8
:10C4800033020000340200003602000037020000D0
:10C49000390200003A0200003C0200003E020000A7
:10C4A0003F0200004102000042020000440200007E
:10C4B0004502000047020000490200004A02000055
:10C4C0004C0200004D0200004F020000510200002B
:10C4D0005202000054020000560200005702000001
:10C4E000590200005B0200005C0200005E020000D6
:10C4F00060020000610200006302000065020000AB
:10C5000066020000680200006A0200006C0200007F
:10C510006D0200006F020000710200007302000053
:10C520007402000076020000780200007A02000027
:10C530007C0200007E0200007F02000081020000F9
:10C5400083020000850200008702000089020000CB
:10C550008B0200008D0200008E020000900200009D
:10C56000920200009402000096020000980200006F
:10C570009A0200009C0200009E020000A00200003F
:10C58000A2020000A4020000A6020000A80200000F
:10C59000AB020000AD020000AF020000B1020000DB
:10C5A000B3020000B5020000B7020000B9020000AB
:10C5B000BC020000BE020000C0020000C202000077
:10C5C000C4020000C7020000C9020000CB02000044
:10C5D000CE020000D0020000D2020000D50200000E
:10C5E000D7020000D9020000DC020000DE020000D9
:10C5F000E1020000E3020000E5020000E8020000A2
:10C60000EA020000ED020000F0020000F202000069
:10C61000F5020000F7020000FA020000FC02000030
:10C62000FF020000020300000503000007030000F2
:10C630000A0300000D0300001003000012030000B5
:10C6400015030000180300001B0300001E03000078
:10C650002103000024030000270300002A03000038
:10C660002D030000300300003303000036030000F8
:10C67000390300003D0300004003000043030000B5
:10C68000460300004A0300004D0300005003000071
:10C6900054030000570300005B0300005E0300002A
:10C6A0006203000065030000690300006D030000E1
:10C6B0007103000074030000780300007C03000095
:10C6C0008003000084030000880300008C03000046
:10C6D0009003000094030000980300009D030000F5
:10C6E000A1030000A5030000AA030000AE030000A0
:10C6F000B3030000B8030000BC030000C103000046
:10C70000C6030000CB030000D0030000D5030000E7
:10C71000DA030000DF030000E5030000EA03000085
:10C72000EF030000F5030000FB030000000400001D
:10C73000060400000C0400001204000019040000AC
:10C740001F040000250400002C0400003304000036
:10C750003A04000040040000480400004F040000B8
:10C76000560400005E040000660400006E04000031
:10C77000760400007E04000087040000900400009E
:10C7800099040000A2040000AC040000B6040000FC
:10C79000C0040000CA040000D5040000E00400004A
:10C7A000EC040000F804000004050000110500007E
:10C7B0001E0500002C0500003A0500004905000098
:10C7C00059050000690500007A0500008C0500008D
:10C7D0009F050000B3050000C8050000DE0500004D
:10C7E0000A4C697374696E672048616E6420436FF8
:10C7F0006E66696775726174696F6E20616E642020
:10C80000496E7465726E616C205374617475733A0D
:10C8100000094163747561746F722031205B20459B
:10C820006C626F772F577269737420726F746174C2
:10C83000696F6E205D2049443A2000205B204F56EE
:10C8400045524C4F41442064657465637465643A95
:10C85000206163747561746F722064697361626CC6
:10C860006564205D00204865616C746820496E64D1
:10C8700065783A2025690A00094163747561746F0F
:10C88000722032205B20577269737420466C657881
:10C89000696F6E205D2049443A2000094163747538
:10C8A00061746F722033205B205468756D6220665E
:10C8B000696E67657220205D2049443A2000094175
:10C8C00063747561746F722034205B20496E6465F7
:10C8D000782066696E67657273205D2049443A204E
:10C8E00000095B2048616E64205669727475616C42
:10C8F000206163747561746F72283529205D204949
:10C90000443A20000A0944796E616D6978656C20AB
:10C91000496E7465726661636520636F6D6D756ED7
:10C9200069636174696F6E2073657474696E67738F
:10C930003A20000A094261756420726174652042E0
:10C9400050533A20000952657475726E2064656C0C
:10C9500061792074696D653A2000205B00206D6963
:10C9600063726F736563735D0009537461747573EB
:10C970002072657475726E206C6576656C3A200065
:10C980000A09436F6E74726F6C20426F617264208B
:10C99000496E666F726D6174696F6E3A000A094282
:10C9A0006F617264206D6F64656C206E723A200056
:10C9B00009426F61726420485720636F6E66696731
:10C9C00020636F64653A200009426F6172642053EE
:10C9D0002F4E3A2000094669726D776172652056C4
:10C9E000657273696F6E3A20000A54686973207526
:10C9F0006E697420697320636F6E6669677572650E
:10CA00006420696E2074686520307E0020706F732A
:10CA10006974696F6E2072616E67652E00412042F5
:10CA20006C7565746F6F746820636F6D6D756E697A
:10CA3000636174696F6E73206D6F64756C652069D6
:10CA4000732070726573656E742E2028757365206F
:10CA5000276274692720666F72206D6F7265206986
:10CA60006E666F726D6174696F6E29004E6F204241
:10CA70006C7565746F6F746820636F6D6D756E692A
:10CA8000636174696F6E73206D6F64756C65206986
:10CA90006E7374616C6C65642E2028757365202735
:10CAA0006274692720666F72206D6F726520696EEF
:10CAB000666F726D6174696F6E29000A5345454453
:10CAC00020524F424F54494353202D2048616E64F9
:10CAD0002044483444205B46572076657273696F62
:10CAE0006E200009686C70202D2074686973206DB9
:10CAF0006573736167650009646964202D204C6962
:10CB000073742048616E6420436F6E666967757246
:10CB10006174696F6E20616E6420496E7465726E17
:10CB2000616C2053746174757300096F7065202DFA
:10CB3000204F70656E2048616E6420636F6D706C6D
:10CB40006574656C792E0009636C6F202D20436C31
:10CB50006F73652048616E6420636F6D706C6574DF
:10CB6000656C792E0009706F73205B416374756189
:10CB7000746F725F6E7220312D345D205B706F7345
:10CB80006974696F6E5D202D207365742061637414
:10CB90007561746F7220706F736974696F6E0009CC
:10CBA000727374205B4163747561746F725F6E722F
:10CBB00020312D345D202D207265736574206163F2
:10CBC000747561746F722028636C65617220657280
:10CBD000726F72732C2064697361626C6520746F6C
:10CBE000727175652C20706F776572207361766540
:10CBF00020616E6420666F72636520636F6E74726D
:10CC00006F6C206D6F64657329000A097265652079
:10CC10005B6F7074696F6E5F6E725D202D20416472
:10CC200076616E63656420436F6E666967757261D5
:10CC300074696F6E20436F6D6D616E64732E0009B1
:10CC4000097265652030202D20646F6573206E6F3A
:10CC50007468696E6720286F6E6C792064697370E0
:10CC60006C6179732061206D65737361676529005C
:10CC700009097265652031202D2052657365747332
:10CC8000207468652044796E616D6978656C204216
:10CC900061756420526174652C2052657475726EE2
:10CCA0002044656C61792054696D6520616E642053
:10CCB0005374617475732052657475726E204C657F
:10CCC00076656C20746F2064656661756C74732082
:10CCD00028314D6270732C20323530205B35303076
:10CCE000206D6963726F735D2C2032205B616C77FD
:10CCF0006179732072657475726E5D29000909721D
:10CD000065652032202D2052657365747320746828
:10CD1000652044796E616D6978656C206163747516
:10CD200061746F722049447320746F20646566617A
:10CD3000756C747320666F72204C454654204841D0
:10CD40004E44202849442032322F32342F32362F9D
:10CD500032382F3330290009097265652033202DC0
:10CD600020526573657473207468652044796E6120
:10CD70006D6978656C206163747561746F722049A8
:10CD8000447320746F2064656661756C74732066EB
:10CD90006F722052494748542048414E4420284948
:10CDA000442032312F32332F32342F32372F323961
:10CDB000290009097265652034205B736574746904
:10CDC0006E675D202D204368616E6765732074680F
:10CDD000652044796E616D6978656C204261756487
:10CDE000205261746520746F206120757365722014
:10CDF00073656C65637465642053657474696E67EC
:10CE00002E20287469703A2056616C756573206114
:10CE10007265207468652073616D65206F6E65733F
:10CE2000207573656420696E207468652044796E8E
:10CE3000616D6978656C2077697A6172642900098F
:10CE400009202020202020202020202020202020F9
:10CE500020202028636F6D6D6F6E20536574746998
:10CE60006E6773206172653A2033343D3537363052
:10CE7000306270732C20313D314D6269742F732CF8
:10CE8000203235323D334D627073290009097265D5
:10CE9000652035205B302F315D202D20436F6E667D
:10CEA000696775726520313032332F34303935205F
:10CEB000706F736974696F6E207265736F6C7574CF
:10CEC000696F6E202820302D3E313032333B2031C7
:10CED0002D3E343039352029000A09627469202D2D
:10CEE0002053686F777320426C7565746F6F746838
:10CEF000204D6F64756C6520496E666F726D61744C
:10CF0000696F6E2028696620696E7374616C6C6548
:10CF10006429000962776E205B6E616D655D202D6E
:10CF2000204368616E67652074686520426C756592
:10CF3000746F6F7468204D6F64756C652042726FFA
:10CF4000616463617374696E67204E616D65000989
:10CF5000627770205B636F64655D202D204368619C
:10CF60006E67652074686520426C7565746F6F74B8
:10CF700068204D6F64756C652050616972696E67D9
:10CF800020436F64650A0009707772202D20466F78
:10CF90007263652061207265626F6F742028506F24
:10CFA000776572206379636C6573207468652061AE
:10CFB00063747561746F722050535520616E6420E4
:10CFC0007265626F6F747320746865206D61696E3D
:10CFD00020626F617264292E0A0041637475617466
:10CFE0006F72206E756D62657273206172653A2092
:10CFF000313D577269737420526F746174696F6E3A
:10D000003B20323D577269737420466C6578696FB6
:10D010006E3B20333D5468756D623B20343D496E54
:10D020006465782066696E67657273004164766135
:10D030006E636564204D616E6167656D656E742019
:10D04000436F6E736F6C6520636F6D6D616E64739B
:10D050003A002B2B2B205741524E494E47202B2B69
:10D060002B2055736520746865736520636F6D6D43
:10D07000616E647320776974682063617574696F89
:10D080006E2E20496E636F727265637420757361D2
:10D090006765206D617920726573756C7420696EA7
:10D0A000207468652068616E64206265636F6D69D5
:10D0B0006E67206D6973636F6E666967757265640C
:10D0C00020616E64206D617920766F696420796FCC
:10D0D00075722057617272616E74792E0009446511
:10D0E0006D6F6E7374726174696F6E20616E64200F
:10D0F000546573742046756E6374696F6E730009AE
:10D1000064666F205B64656D6F206E722E20312D1A
:10D11000335D205B20666F72636520312D323030C5
:10D120003020205D202D20666F72636520636F6E56
:10D1300074726F6C2064656D6F6E73747261746964
:10D140006F6E730009646666205B534552564F5FED
:10D150006E7220312D345D202D2064656D6F6E73ED
:10D160007472617465207265616C2074696D6520EC
:10D17000466F7263652052656164696E6700096479
:10D180007066205B534552564F5F6E7220312D34CE
:10D190005D202D2064656D6F6E73747261746520FF
:10D1A0007265616C2074696D6520506F7369746974
:10D1B0006F6E20466565646261636B000A09496EA3
:10D1C000697469616C697A6174696F6E20616E64FB
:10D1D00020416476616E636564204D616E616765B0
:10D1E0006D656E742046756E6374696F6E730009A9
:10D1F000746D72202D20446973706C617920737492
:10D2000061747573206F6620496E7465726E616C0F
:10D210002054696D6572730009656563205B534531
:10D2200052564F5F6E7220312D345D202D2044699F
:10D2300073706C617920454550524F4D20636F6E7D
:10D2400066696775726174696F6E20666F722061BE
:10D2500063747561746F72202848572050696E732B
:10D260002C2072616E6765732C202E2E2E290009EA
:10D270006163747561746F72206E756D626572732F
:10D28000206172653A20313D577269737420526F84
:10D29000746174696F6E3B20323D577269737420FC
:10D2A000466C6578696F6E3B20333D5468756D62DE
:10D2B0003B20343D496E6465786573000A096361FB
:10D2C00070205B6163747561746F72206E722031BF
:10D2D0002D345D202D2043616C696272617465207C
:10D2E0006163747561746F7220506F736974696FD4
:10D2F0006E2053656E736F722028706572666F7250
:10D300006D7320612066756C6C2073776565702085
:10D31000616E642073746F7265732063616C6962FF
:10D32000726174696F6E20726573756C74732069B5
:10D330006E20454550524F4D29000A09696E6520FF
:10D340005B6F7074696F6E5F6E725D205B76616C8F
:10D3500075655D202D2050726F6772616D2F496E6B
:10D36000697469616C697A6520454550524F4D007A
:10D3700009696E652031205B616E792076616C757C
:10D38000655D2020202020202D20496E6974696170
:10D390006C697A6520454550524F4D20666F72206A
:10D3A0007468652066697273742074696D652028DD
:10D3B000736574732050574D2072616E6765732CCE
:10D3C00020657463290009696E652032205B426F15
:10D3D000617264204D6F64656C5D202D205265671D
:10D3E000697374657220426F617264204D6F646569
:10D3F0006C0009696E652033205B426F61726420A6
:10D40000485720636F6E66696775726174696F6EE5
:10D410005D202D20526567697374657220426F61CB
:10D42000726420485720636F6E6669677572617415
:10D43000696F6E0009696E652034205B532F4E20A2
:10D44000594541522020205D202D205965617220D0
:10D450006F66206D616E75666163747572696E6763
:10D4600020283220646967697473290009696E6530
:10D470002035205B532F4E204D4F4E544820205DC9
:10D48000202D204D6F6E7468206F66206D616E7563
:10D49000666163747572696E6720283220646967FB
:10D4A000697473290009696E652036205B532F4E1D
:10D4B00020554E49545F4E525D202D20556E6974A3
:10D4C000206E756D626572206F662070726573657F
:10D4D0006E74206D6F6E74680009696E6520372068
:10D4E0002D20496E697469616C697A65732074686E
:10D4F0006520426C7565746F6F7468204D6F64753C
:10D500006C65206E616D6520616E6420426175649A
:10D510002052617465000A09626170205B415420E9
:10D52000636F6D6D616E64205D202D20426C7565AA
:10D53000746F6F7468204D6F64756C652041542062
:10D54000636F6D6D616E6420706173737468726F68
:10D550007567682066756E6374696F6E20286261F6
:10D56000636B646F6F7229000A09737370205B61CB
:10D5700063747561746F725F6E725D205B7370654A
:10D5800065642070657263656E745D202D20436F45
:10D590006E666967757265204163747561746F7238
:10D5A0002069735F6D6F76696E672073706565645F
:10D5B0002028666F72206163747561746F727320C6
:10D5C00077697468206F726967696E616C2066772D
:10D5D0002900466F722068656C70206F6E20626152
:10D5E00073696320636F6D6D616E64732C20706C62
:10D5F0006561736520747970652027686C70272ECB
:10D6000000506172616D65746572206F7574206F72
:10D61000662072616E67652E204163636570746178
:10D62000626C652072616E676520697320307E329E
:10D630003030302E000A44656D6F6E737472617401
:10D64000696E6720466F72636520436F6E74726FF8
:10D650006C3A2069735F6D6F76696E6720756E74C2
:10D66000696C20666F7263652000206973206465B1
:10D670007465637465642E0054696D656F757420FC
:10D68000646574656374696E67206D6F74696F6E2D
:10D690002E2044656D6F6E7374726174696F6E20B5
:10D6A00061626F727465642E004D6F76656D656E94
:10D6B000742073746F7070656420616E6420706F85
:10D6C000736974696F6E2068656C642E004F7065B5
:10D6D0006E696E672048616E64206E6F772E004819
:10D6E0006F6C64696E6720506F736974696F6E2E1A
:10D6F00000506172616D65746572206F7574206F82
:10D70000662072616E67652E204163636570746187
:10D71000626C652072616E676520697320317E32AC
:10D720003030302E000A44656D6F6E737472617410
:10D73000696E6720466F72636520436F6E74726F07
:10D740006C20436F6D706C69616E63653A2044793B
:10D750006E616D6963616C6C792041646A75737484
:10D76000696E6720746F206D6565742064657369E8
:10D7700072656420666F7263652E200048616E6476
:10D780002077696C6C206E6F772064796E616D69AB
:10D7900063616C6C792061646A7573742074686568
:10D7A000206772697020746F206D61696E746169A1
:10D7B0006E20746865206465736972656420666FA5
:10D7C0007263652E0055736520277273742720637A
:10D7D0006F6D6D616E6420746F207465726D696E1B
:10D7E0006174652074686973206D6F64652E0049EB
:10D7F0006E76616C6964206E756D62657220666F0D
:10D800007220666F7263652064656D6F6E737472EB
:10D810006174696F6E2E2056616C6964206E756D3F
:10D82000626572732061726520312D332E00454E82
:10D8300041424C45440044495341424C4544202810
:10D84000706F737369626C7920736F6D65204857D0
:10D850002070696E732061726520696E636F7272E9
:10D860006563746C7920636F6E6669677572656451
:10D8700029000A446973706C6179696E672073745A
:10D8800061747573206F6620496E7465726E616C89
:10D890002054696D6572733A000943757272656E42
:10D8A00074205369676E616C2046696C7465726997
:10D8B0006E673A20000954696D657220666F7220A8
:10D8C000543D32306D733A20000954696D65722001
:10D8D000666F7220543D3230306D733A20005468C8
:10D8E000652070696E7320666F722074686973209A
:10D8F0006163747561746F722061726520636F6E0D
:10D90000736964657265642076616C696420616E18
:10D910006420636F72726563746C7920636F6E66E6
:10D920006967757265642E20436F6E6669726D203B
:10D930007468652070696E7320666F72206F7468FA
:10D940006572206163747561746F727320616E64B7
:10D95000207468652054656D7065726174757265B8
:10D960002070696E2E005468652070696E732066A1
:10D970006F722074686973206163747561746F726B
:10D980007320617265204E4F5420434F52524543DD
:10D99000544C5920636F6E666967757265642E20FA
:10D9A000546869732077696C6C20726573756C7448
:10D9B00020696E2074696D657273206265696E6797
:10D9C0002064697361626C65642028747279202711
:10D9D000746D722720636F6D6D616E6429000A4457
:10D9E0006973706C6179696E6720636F6E666967D1
:10D9F00075726174696F6E206F6620485720706978
:10DA00006E7320666F72206163747561746F72202B
:10DA1000000950574D2050696E3A200009504F546C
:10DA20002050696E3A20000943757272656E742049
:10DA300050696E3A20000A0954656D706572617410
:10DA40007572652050696E2028636F6D6D6F6E2052
:10DA5000746F20616C6C206163747561746F727394
:10DA6000293A20000A0950574D204D696E3A20008E
:10DA70000950574D204D61783A20000A09504F5403
:10DA8000204D696E3A200009504F54204D61783A7C
:10DA900020000943757272656E74206D656173753F
:10DAA00072656D656E743A20000A416476616E633A
:10DAB000656420436F6E66696775726174696F6E25
:10DAC00020436F6D6D616E6473200009546F206D8B
:10DAD000616B6520616E20616476616E63656420B0
:10DAE000636F6E66696775726174696F6E2C2074FE
:10DAF000686520706172616D65746572206F662063
:10DB00002772656527206D757374206265207769BB
:10DB10007468696E2074686520616C6C6F776564E9
:10DB20002072616E67652E00095479706520276840
:10DB30006C702720666F72206D6F726520696E664B
:10DB40006F726D6174696F6E206265666F726520B9
:10DB5000636F6E74696E75696E672E000952657326
:10DB60006574204261756420526174652C20526591
:10DB70007475726E2044656C61792054696D6520FE
:10DB8000616E64205374617475732052657475728C
:10DB90006E204C6576656C20746F206465666175D7
:10DBA0006C742073657474696E67732E0009506C11
:10DBB0006561736520506F776572204379636C658A
:10DBC000207468652068616E64202874727920274B
:10DBD0007077722720636F6D6D616E642920616EAE
:10DBE0006420757365207468652027646964272044
:10DBF0006F6E207468697320636F6E736F6C65203D
:10DC0000746F20636F6E6669726D20746865206E34
:10DC100065772073657474696E67732E00095265A9
:10DC200073657420494473206F6E20616C6C20749E
:10DC300068652034206163747561746F727320614C
:10DC40006E6420746865205669727475616C206119
:10DC500063747561746F7220666F72207468697383
:10DC60002068616E642E00094944732077696C6CEA
:10DC700020636F6E6669677572656420666F7220D7
:10DC800061204C4546542068616E643A2049442026
:10DC9000323220285669727475616C206163747524
:10DCA00061746F722920616E642032342F32362FF6
:10DCB00032382F33302028506879736963616C20C3
:10DCC0006163747561746F7273290009434155541F
:10DCD000494F4E2120496620796F7520686176652D
:10DCE000206F746865722064657669636573206966
:10DCF0006E7374616C6C6564206F6E20746865204F
:10DD00006D61696E2073797374656D207573696ECA
:10DD1000672074686573652073616D65204944737D
:10DD20002C20706C6561736520757365207468655F
:10DD3000205553423244796E616D6978656C20617B
:10DD40006E642044796E616D6978656C2057697ADC
:10DD500061726420746F2072656D617020746865F3
:10DD60002049447320746F20796F75722064657345
:10DD7000697265642073657474696E67732E000937
:10DD8000506C6561736520506F77657220437963CD
:10DD90006C65207468652068616E642028747279EF
:10DDA00020277077722720636F6D6D616E64292064
:10DDB000616E6420757365207468652027646964EA
:10DDC0002720636F6D6D616E6420746F20636F6ECA
:10DDD0006669726D20746865206E657720494473AA
:10DDE0002068617665206265656E2E00094944737E
:10DDF0002077696C6C20636F6E6669677572656405
:10DE000020666F7220612052494748542068616E35
:10DE1000643A204944203231202856697274756171
:10DE20006C206163747561746F722920616E642067
:10DE300032332F32352F32372F323920285068793C
:10DE4000736963616C206163747561746F727329A7
:10DE500000094368616E67652074686520426175DA
:10DE600064205261746520746F206120757365723F
:10DE70002073656C65637465642073657474696E82
:10DE8000672E0009506C65617365206E6F74653A8A
:10DE90002074686973206F7074696F6E20636861A5
:10DEA0006E676573207468652042617564205261F5
:10DEB0007465206F6E207468652044796E616D69A9
:10DEC00078656C20706F727420696E74657266611B
:10DED00063652E2042617564207261746520666FEF
:10DEE0007220555342206F72206F746865722069EA
:10DEF0006E746572666163657320617265206E6F12
:10DF0000742061666665637465642E0009546865F3
:10DF10002076616C756573206F6620746869732064
:10DF200073657474696E672061726520746865201A
:10DF300073616D65207573656420696E2044796E28
:10DF4000616D6978656C2057697A6172642E20531F
:10DF5000656520526F626F74697320646F63756DBD
:10DF6000656E746174696F6E2C20696E20706172C9
:10DF7000746963756C6172204261756420726174AA
:10DF80006520706172616D6574657220666F7220C4
:10DF90004D582073657269657320746F20636F6ECE
:10DFA0006669726D20746865206D65616E696E6763
:10DFB000206F66207468652076616C75652E000997
:10DFC0004261756420726174652073657474696E52
:10DFD000672077696C6C206265206368616E676595
:10DFE0006420746F3A20000A09596F752073686FB6
:10DFF000756C6420706F776572206379636C65203F
:10E0000074686520626F61726420746F20656E6150
:10E01000626C6520746865206E6577207365747422
:10E02000696E672E202874727920277077722720F6
:10E03000636F6D6D616E64290009496620796F75A3
:10E0400020656E636F756E74657220636F6D6D759C
:10E050006E69636174696F6E206572726F7273208E
:10E0600061667465722074686973206368616E67A5
:10E07000652C207573652027726565203127207413
:10E080006F20726573746F726520746865206261B9
:10E090007564207261746520746F207468652064F3
:10E0A000656661756C742073657474696E672E00A3
:10E0B00009436F6E66696775726520506F73697486
:10E0C000696F6E205265736F6C7574696F6E20286E
:10E0D000302D3E313032333B20312D3E3430393516
:10E0E000290009506F736974696F6E207265736FD0
:10E0F0006C7574696F6E2077696C6C206265206343
:10E100006F6E6669677572656420746F2031306266
:10E1100069742028307E31303233292E20546869CA
:10E12000732077696C6C206265636F6D6520616335
:10E1300074697665206166746572207265626F6FBE
:10E1400074696E67207468652068616E642E0009CA
:10E15000506F736974696F6E207265736F6C75743C
:10E16000696F6E2077696C6C20626520736574201E
:10E17000746F2031326269742028307E3430393532
:10E18000292E20546869732077696C6C206265635E
:10E190006F6D652061637469766520616674657270
:10E1A000207265626F6F74696E672074686520689D
:10E1B000616E642E0009496E76616C69642070613D
:10E1C00072616D6574657220666F7220706F73691D
:10E1D00074696F6E207265736F6C7574696F6E2EE3
:10E1E000204D7573742062652027302720666F727A
:10E1F0002031303233206F722027312720666F7232
:10E2000020343039352E000A09494D504F525441BF
:10E210004E543A20596F75206D757374206E6F7768
:10E2200020706F776572206379636C652074686510
:10E230002068616E6420746F20656E61626C652079
:10E24000746865206E65772073657474696E672ED7
:10E250000009496E76616C696420706172616D6558
:10E260007465722E0009547970652027686C7027D8
:10E2700020666F72206D6F726520696E666F726DB9
:10E280006174696F6E2E000A50726F6772616D2F34
:10E29000496E697469616C697A6520454550524FD1
:10E2A0004D0009496E76616C696420706172616D20
:10E2B000657465722E20557365202761687027206C
:10E2C000666F72206D6F726520696E666F726D6128
:10E2D00074696F6E2E0009496E697469616C697AA0
:10E2E000696E6720454550524F4D2077697468200C
:10E2F00066697273742072756E2076616C756573D1
:10E30000202870776D2072616E6765732C206574AC
:10E310006329000946696E652074756E696E672011
:10E320006F66207468652050574D2072616E676576
:10E3300020616E64206F7468657220706172616D17
:10E3400065746572732063616E20626520646F6E10
:10E3500065207573696E672044796E616D697865B3
:10E360006C2057697A6172642062792073657474D5
:10E37000696E672074686520626F61726420746FD3
:10E380002063616C6962726174696F6E206D6F6485
:10E39000652E000953657474696E67204861726464
:10E3A0007761726520426F617264204D6F64656CA5
:10E3B0000009426F617264204D6F64656C2077695B
:10E3C0006C6C2062652073657420746F3A200009BC
:10E3D00053657474696E6720486172647761726511
:10E3E00020426F61726420485720436F6E666967F0
:10E3F00000094552524F523A205265766973696F4F
:10E400006E206D7573742062652061206E756D627B
:10E410006572206265747765656E20302D32353502
:10E420000009426F61726420485720636F6E66690D
:10E43000672077696C6C2062652073657420746F47
:10E440003A20000953657474696E672053657269D8
:10E45000616C204E756D626572202D2059454152C8
:10E4600000094552524F523A2059454152206D758C
:10E4700073742062652061203220646967697420AA
:10E480006E756D6265722028692E652E20313620EA
:10E49000666F722032303136290009536572696126
:10E4A0006C204E756D626572205945415220776926
:10E4B0006C6C2062652073657420746F3A200009CB
:10E4C00053657474696E672053657269616C204E80
:10E4D000756D626572202D204D4F4E5448000945E0
:10E4E00052524F523A204D4F4E5448206D7573741E
:10E4F00020626520612076616C6964203220646945
:10E50000676974206E756D6265722028692E652EAC
:10E5100020313120666F72204E6F76656D626572B4
:10E5200029000953657269616C204E756D626572D0
:10E53000204D4F4E54482077696C6C2062652073E3
:10E54000657420746F3A20000953657474696E67AE
:10E550002053657269616C204E756D626572202D65
:10E5600020554E4954204E5220696E207468652013
:10E57000596561722F4D6F6E7468207370656369A1
:10E580006669656400094552524F523A20554E491A
:10E5900054204E52206D6178696D756D2076616CE6
:10E5A0007565206973203235352E0009536572690F
:10E5B000616C204E756D62657220554E4954204E37
:10E5C000522077696C6C2062652073657420746FCB
:10E5D0003A200009496E697469616C697A696E67ED
:10E5E0002074686520426C7565746F6F7468204D87
:10E5F0006F64756C65204E616D6520616E642042AC
:10E60000617564205261746500534545445F255827
:10E61000255825580009426C7565746F6F74682021
:10E620004E616D652077696C6C206265207365743E
:10E6300020746F20002E2E2E20446F6E652E002E2B
:10E640002E2E204641494C20286D6179626520427A
:10E6500054206D6F64756C65206E6F7420646574F2
:10E6600065637465643F207472792027627469273A
:10E6700020636F6D6D616E6429000A0942617564E3
:10E6800020526174652077696C6C20626520736527
:10E690007420746F20313535203230306270732C25
:10E6A00020384E312E0A0953656E64696E672070FA
:10E6B0006173737468726F75676820636F6D6D61E5
:10E6C0006E642E205265706C793A0A090041542B11
:10E6D000554152543D3131353230302C302C3000E0
:10E6E000095479706520276168702720666F722051
:10E6F0006D6F726520696E666F726D6174696F6EA1
:10E700002E000A4966206368616E6765732077652D
:10E710007265207375636365737366756C2C207006
:10E720006C6561736520504F574552204359434CE7
:10E73000452074686520626F61726400466F7220C4
:10E740006E6578742073746570732C20796F7520F2
:10E750006D61792077616E7420746F207573652008
:10E7600074686520277265652720636F6D6D616E23
:10E770006420746F207365742049447320616E6453
:10E780002042617564205261746520666F72207446
:10E79000686520626F61726420616E642066696ED4
:10E7A000616C6C792072756E20612053656C6620F7
:10E7B00043616C6962726174696F6E20746F20636B
:10E7C0006F6D706C65746520746865207365742D59
:10E7D00075702070726F6365647572652E00496E86
:10E7E00076616C6964206163747561746F72206E08
:10E7F000756D6265720043616C6962726174696E05
:10E8000067206163747561746F72206E756D6265E7
:10E81000723A2000546865206163747561746F7288
:10E820002077696C6C206E6F7720706572666F72EE
:10E830006D20612066756C6C2073776565702E2085
:10E840004D616B6520737572652074686520616326
:10E85000747561746F72206973206E6F74206F62BB
:10E86000737472756374656420616E642077616986
:10E870007420756E74696C207468652070726F63A3
:10E880006573732066696E69736865732E005468DA
:10E890006520756E6974206D6179207365656D20E2
:10E8A000756E726573706F6E7369766520647572CC
:10E8B000696E67207468652063616C696272617457
:10E8C000696F6E2070726F6365647572652E205477
:10E8D000686973206973206E6F726D616C2E000A17
:10E8E00043616C6962726174696F6E20636F6D70F1
:10E8F0006C6574652E20526573756C74732073613A
:10E9000076656420746F20454550524F4D2E005956
:10E910006F75206D61792077616E7420746F20723D
:10E920006570656174207468652070726F636564DA
:10E9300075726520666F72206F74686572206163FE
:10E94000747561746F72732E00506572666F726DAC
:10E95000696E672066756C6C2072616E6765205306
:10E9600077656570206F6E206163747561746F7276
:10E97000206E756D6265723A200054686520756E70
:10E980006974206D6179207365656D20756E72659F
:10E9900073706F6E7369766520647572696E672037
:10E9A0007468652073776565702070726F63656445
:10E9B0007572652E2054686973206973206E6F72BA
:10E9C0006D616C2E00537765657020636F6D706CA0
:10E9D0006574652E004F4E004F4646000A426C7526
:10E9E00065746F6F7468204D6F64756C6520496E37
:10E9F000666F726D6174696F6E0009426C75657443
:10EA00006F6F7468204D6F64756C653A2050524585
:10EA100053454E54000942726F6164636173742000
:10EA20006E616D653A20000950616972696E6720F8
:10EA3000636F64653A2025303469200A0009506FFD
:10EA4000776572207374617475733A200009426CA3
:10EA50007565746F6F7468204D6F64756C653A20CE
:10EA60004E4F542050524553454E542F4E4F542034
:10EA70004445544543544544000A4368616E676504
:10EA800020426C7565746F6F7468204D6F64756C8F
:10EA9000652042726F616463617374204E616D65BD
:10EAA00000094E6F20426C7565746F6F7468206D3D
:10EAB0006F64756C652070726573656E742F646524
:10EAC0007465637465642E0009496E76616C6964CF
:10EAD000206E616D6521204E616D65206D757374CA
:10EAE000206265206120737472696E672077697493
:10EAF00068206D696E696D756D203120616E6420CE
:10EB00006D6178696D756D20323020636861726166
:10EB1000637465727300094D6F64756C6520427291
:10EB20006F6463617374206E616D652077696C6CCE
:10EB3000206265206368616E67656420746F3A20A7
:10EB4000000A094E616D65206368616E6765642027
:10EB50007375636365737366756C792E000A09417A
:10EB60006E206572726F722077617320656E636FBD
:10EB7000756E7465726564207768696C6520617470
:10EB800074656D7074696E6720746F206368616E60
:10EB9000676520746865206E616D652E000A4368A4
:10EBA000616E676520426C7565746F6F7468204D87
:10EBB0006F64756C652050616972696E6720436F80
:10EBC00064650009496E76616C6964205061697200
:10EBD000696E6720636F6465212050616972696E98
:10EBE0006720636F6465206D757374206861766556
:10EBF0002034206469676974732E00094D6F647551
:10EC00006C652050616972696E6720436F6465208E
:10EC100077696C6C206265206368616E676564204B
:10EC2000746F3A2025303469000A095061697269AD
:10EC30006E6720636F6465206368616E676564203A
:10EC40007375636365737366756C792E000A094189
:10EC50006E206572726F722077617320656E636FCC
:10EC6000756E7465726564207768696C652061747F
:10EC700074656D7074696E6720746F206368616E6F
:10EC80006765207468652070616972696E672063CA
:10EC90006F64652E000A426C7565746F6F7468202E
:10ECA0004D6F64756C6520415420506173737468B6
:10ECB000726F756768204D6F6465000954686973E9
:10ECC0002066756E6374696F6E206C65747320794D
:10ECD0006F75207061737320636F6D6D616E647307
:10ECE000206469726563746C7920746F2074686540
:10ECF00020426C7565746F6F7468206D6F64756CFD
:10ED00006520696E20415420636F6E666967757275
:10ED10006174696F6E206D6F64652E0009436F6DBD
:10ED20006D616E64206170706561727320746F2014
:10ED3000626520656D7074792E0009426C7565748A
:10ED40006F6F7468204D6F64756C65207265706CB0
:10ED5000793A0A09000A5365742061637475617415
:10ED60006F72205370656564000944656661756C57
:10ED70007420737065656473206172653A20416325
:10ED8000747561746F7220313D34352C20323D34FE
:10ED9000352C20333D31352C20343D31352E000AC1
:10EDA00009537065656420706172616D6574657288
:10EDB000206973206F7574206F662072616E6765BD
:10EDC0002E2041636365707461626C652072616EB0
:10EDD000676520697320317E3130302E000A095377
:10EDE000706565642077696C6C206265207365745A
:10EDF000206F6E206163747561746F7220256920C5
:10EE0000746F2025692025202E0A000A09546865A0
:10EE10002068616E642077696C6C207265626F6F28
:10EE200074206F6E63652074686520737065656417
:10EE300020636F6E66696775726174696F6E2069B1
:10EE40007320636F6D706C6574652E0A09496620C6
:10EE5000796F752061726520636F6E6E656374658E
:10EE6000642076696120426C7565746F6F746820E8
:10EE7000796F752077696C6C206E65656420746F9E
:10EE80002072652D636F6E6E6563742061667465B4
:10EE90007277617264732E0A09496620796F752052
:10EEA00061726520636F6E6E656374656420766958
:10EEB00061205553422C206D616E75616C6C792018
:10EEC000646973636F6E6E65637420616E64207233
:10EED00065636F6E6E656374207468652055534278
:10EEE000206361626C652061667465722074686578
:10EEF000207265626F6F742E000A09537065656435
:10EF00002073657420646F6E652E00094445425578
:10EF1000473A207465656E7379206E6F7420726550
:10EF2000626F6F7465643B207265626F6F74206DF1
:10EF3000616E75616C6C790009506F776572206342
:10EF400079636C65206661696C65643A206D6F73E6
:10EF500074206C696B656C792074686520536F66EA
:10EF6000747761726520706F776572206379636C66
:10EF7000652066756E6374696F6E616C6974792063
:10EF8000697320756E737570706F72746564206F2D
:10EF90006E207468697320626F6172642E0A095072
:10EFA0006C6561736520506F776572206379636C5F
:10EFB000652074686520756E6974206D616E756179
:10EFC0006C6C79206E6F77210A0928646973636F0E
:10EFD0006E6E6563742074686520706F776572204B
:10EFE000737570706C79205F616E645F2074686502
:10EFF00020555342206361626C6520696620636F0F
:10F000006E6E656374656429000A09416E2065723D
:10F01000726F7220686173206F63637572726564CA
:10F0200020647572696E6720746869732070726FEE
:10F030006365647572652E20496E20636173652077
:10F04000746865206163747561746F7220626563B2
:10F05000616D6520756E726573706F6E736976652C
:10F060002C20706C6561736520506F77657220434A
:10F0700079636C65207468652068616E64207769C7
:10F0800074682074686520277077722720636F6D1D
:10F090006D616E642E000A506F776572206379632C
:10F0A0006C696E67207468652048616E642E2E2E30
:10F0B000000A095265626F6F74696E672E2E2E000A
:10F0C00009506F776572206379636C6520666169AA
:10F0D0006C65643A206D6F7374206C696B656C7934
:10F0E0002074686520536F66747761726520706F55
:10F0F000776572206379636C652066756E637469E9
:10F100006F6E616C69747920697320756E737570A8
:10F11000706F72746564206F6E207468697320620A
:10F120006F6172642E0A09596F75206D75737420B2
:10F130006D616E75616C6C7920506F7765722063BC
:10F1400079636C652074686520756E6974206279D6
:10F1500020646973636F6E6E656374696E67207493
:10F16000686520706F77657220737570706C792098
:10F170005F616E645F20746865205553422063614F
:10F18000626C6520696620636F6E6E65637465648A
:10F190002E0064666F00647077006470660072739E
:10F1A0007400706F7300686C70006469640064665A
:10F1B000660061687000746D720065656300726559
:10F1C0006500696E65006361700062746900627752
:10F1D0006E0062777000626170006F706500636C32
:10F1E0006F007373700070777200726562007265F1
:10F1F000770077726200777277000A4552524F5259
:10F200003A20556E6B6E6F776E206F7220696E7646
:10F21000616C696420636F6D6D6D616E642E205446
:10F220007970652027686C702720666F72206120D6
:10F230006C697374206F6620617661696C61626CC1
:10F240006520636F6D6D616E64730054686973202F
:10F2500066756E6374696F6E206973206375727270
:10F26000656E746C79206E6F7420696D706C656D5D
:10F27000656E74656420696E2074686973204657F2
:10F280002076657273696F6E2E000A44656D6F6E2D
:10F290007374726174696E672045787465726E610B
:10F2A0006C20466F72636520666565646261636B9E
:10F2B000206F6E206163747561746F72200041630A
:10F2C000747561746F722077696C6C206265206D53
:10F2D0006F76656420746F20696E7465726D656405
:10F2E0006961746520706F736974696F6E2E205543
:10F2F000736520796F75722068616E6420746F2069
:10F3000067656E746C7920666F72636520746865DA
:10F31000206163747561746F7220435720616E645D
:10F320002043435720616E64206F62736572766577
:10F33000207468652072656164696E67732E00438E
:10F34000435720666F7263652000435720666F72D3
:10F3500063652020000A44656D6F6E73747261747A
:10F36000696E67205265616C2054696D6520706F0D
:10F37000736974696F6E20666565646261636B2092
:10F380006F6E206163747561746F7220004D6F76CB
:10F390006520746865206163747561746F7220778D
:10F3A00069746820796F75722068616E642077686F
:10F3B000696C65207468652063757272656E74206F
:10F3C000706F736974696F6E2069732064697370FC
:10F3D0006C6179656420686572652E004375727290
:10F3E000656E7420706F736974696F6E3A00496E50
:10F3F00076616C6964206163747561746F722E004C
:10F400000A526573657474696E67204F7665726C15
:10F410006F61642073746174652C20746F727175F0
:10F42000652C20706F776572207361766520616E40
:10F430006420666F72636520636F6E74726F6C20F8
:10F440006F6E206163747561746F7220000A4F7073
:10F45000656E696E672048616E642E0028746F7255
:10F46000717565206973206175746F6D617469636E
:10F47000616C6C7920656E61626C656420696620E0
:10F480006E65636573736172793B20746F20646984
:10F490007361626C6520746F727175652075736538
:10F4A00020277273742720696E7374727563746990
:10F4B0006F6E29000A436C6F73696E672048616E36
:10F4C000642E000A4649524D57415245204552523A
:10F4D0004F523A20436F6D6D616E642072656163B7
:10F4E00068656420656E64206F6620537769746375
:10F4F000682073746174656D656E742E2054797024
:10F50000652027686C702720666F7220696E73749F
:10F5100072756374696F6E732E000A4D6F76696E33
:10F5200067206163747561746F72200020746F20AE
:10F53000706F736974696F6E20000A496E76616C32
:10F54000696420706F736974696F6E2E2041636304
:10F5500065707461626C652072616E676520666FAC
:10F56000722074686973206163747561746F7220AE
:10F57000697320307E006D616C6C6F632066616919
:10F580006C2034006D616C6C6F63206661696C2067
:10F5900035005061636B65743A2000307846462030
:10F5A0003078464620307800466F756E6420636F71
:10F5B0006D6D616E6420666F722044594E2049441F
:10F5C0003A20006D616C6C6F63206661696C20335A
:10F5D000006D616C6C6F63206661696C2032006D38
:10F5E000616C6C6F63206661696C00636C73464983
:10F5F000464F4C6973743A20417474656D7074653C
:10F600006420746F206765744669727374496E2054
:10F6100066726F6D20616E20656D707479206C6903
:10F6200073742100636C734649464F4C6973743A96
:10F6300020617474656D7074656420746F207265E8
:10F640006D6F7665206D6F7265206974656D7320CE
:10F650007468616E2077686174206578697374736B
:10F6600020696E20746865206C6973742100496E8E
:10F6700076616C696420737461746520696E2073AF
:10F6800077697463685F706879736963616C5F6CD4
:10F6900065645F6F6E3A2074686520637572726589
:10F6A0006E7420736572766F20626C696E6B696E22
:10F6B00067206973206E6F7420696E2061206B6E05
:10F6C0006F776E2073746174650043757272656E36
:10F6D0007420736572766F20626C696E6B696E67F9
:10F6E0003A20004572726F7220696E697469616CAC
:10F6F000697A696E6720736572766F2E20556E6B1E
:10F700006E6F776E20736572766F20696E207365F9
:10F71000745F746F727175655F6F6E5F646566614B
:10F72000756C745F706F736974696F6E2E0023005F
:10F73000496E76616C69642073657474696E6720C4
:10F74000666F72204C45442077726974650041747D
:10F7500074656D7074696E6720746F207265616482
:10F76000206120424954206F6E2061206269746DCF
:10F770006170206275742069742773206F7574201E
:10F780006F662072616E67653B2074686520616CEE
:10F790006C6F7765642072616E67652069732030D5
:10F7A0007E31352E00454550524F4D207772697499
:10F7B000652064656E69656420627920696E746590
:10F7C000726E616C2070726F74656374696F6E2EF7
:10F7D000204E72206F6620777269746573206174A1
:10F7E00074656D7074656420696E20746869732037
:10F7F00073657373696F6E3A2000417474656D7040
:10F8000074696E6720746F20777269746520612057
:10F81000424954206F6E2061206269746D617020CE
:10F820006275742069742773206F7574206F662069
:10F8300072616E67653B2074686520616C6C6F77E0
:10F8400065642072616E676520697320307E313592
:10F850002E00496E74657272757074696F6E2873CC
:10F86000292064697361626C6564206265636175F7
:10F87000736520454550524F4D206973206E6F745B
:10F8800020636F6E66696775726564206F72206DA4
:10F89000697373696E6720696E666F726D617469F2
:10F8A0006F6E2E00FFFFFFFF000000000000000051
:10F8B00049670000378900001367000035670000C2
:10F8C0002167000005670000050E08090D0C0607FA
:10F8D0000F04001303931A9217C585848687C4FF0B
:10F8E0006FF07F030370037813F0800FFBD0704735
:10F8F0004008FE4340A004404408FE4344A00440A6
:10F900000018FE4300C004403000FE433090044025
:10F910003400FE43349004401C18FE431CC00440D5
:10F920001018FE4310C004400818FE4308C00440ED
:10F930000C18FE430CC004400C10FE430CB00440F5
:10F940001010FE4310B004401810FE4318B00440DD
:10F950001C10FE431CB004401410FE4314B00440BD
:10F960000418FE4304C004400010FE4300B00440ED
:10F970000008FE4300A004400408FE4304A0044025
:10F980000C08FE430CA004400808FE4308A00440F5
:10F990001418FE4314C004401818FE4318C0044055
:10F9A0000410FE4304B004400810FE4308B00440B5
:10F9B0001400FE43149004404C08FE434CA0044045
:10F9C0000420FE4304D004402410FE4324B004402D
:10F9D0002010FE4320B004402810FE4328B004400D
:10F9E0002C10FE432CB004400020FE4300D0044005
:10F9F0004808FE4348A004401000FE431090044015
:10FA0000090AFFFFFFFFFFFFFFFFFFFFFFFFFF0DE3
:10FA100000060807FFFF0E0FFF0CFFFFFFFFFFFFB1
:10FA20000B05FFFFFFFFFFFF0000000000000000CC
:10FA3000FD84000015850000E5840000ED840000D1
:10FA4000E9840000F1840000898400009B840000A8
:10FA5000BB840000BF840000C5840000D584000082
:10FA6000F5840000F98400005984000065840000DA
:10FA7000718400007D840000258500000985000058
:10FA80000000000000000000018600001986000050
:10FA9000E9850000F1850000ED850000F585000096
:10FAA0008D8500009F850000BF850000C385000094
:10FAB000C9850000D9850000F9850000FD8500009A
:10FAC0005D85000069850000758500008185000066
:10FAD000298600000D8600000000000000000000E4
:10FAE000058700001D870000ED860000F5860000F8
:10FAF000F1860000F986000091860000A3860000D0
:10FB0000C3860000C7860000CD860000DD860000A9
:10FB1000FD86000001870000618600006D86000000
:10FB200079860000858600002D870000118700007F
:10FB30000D0AFFFFFFFFFFFF0000000000000000B4
:10FB40006F8A0000758A00005F8A0000638A0000E7
:10FB5000678A00006B8A000000151915000100007B
:10FB60007487FF1F12000000000200009E87FF1F25
:10FB70004300000000030000F887FF1F00000000A2
:10FB8000010309048687FF1F000000000203090427
:10FB9000E287FF1F0000000003030904FC87FF1F2A
:10FBA0000000000000000000000000000000000055
:10FBB00065787000FFFFFFFF000000000000E03FDD
:10FBC000000000000000E0BF763C7935EF39EA3DE7
:10FBD000763C7935EF39EABD0000E0FE422EE63F83
:10FBE0000000E0FE422EE6BF4300FFFF1488FF1F27
:10FBF000232D302B2000686C4C0065666745464716
:10FC00000030313233343536373839414243444598
:10FC10004600303132333435363738396162636407
:10FC20006566000020202020202020202028282871
:10FC300028282020202020202020202020202020B4
:10FC400020202020881010101010101010101010FC
:10FC5000101010100404040404040404040410101C
:10FC600010101010104141414141410101010101B9
:10FC70000101010101010101010101010101011065
:10FC8000101010101042424242424202020202028E
:10FC90000202020202020202020202020202021036
:10FCA0001010102000000000000000000000000004
:10FCB0000000000000000000000000000000000044
:10FCC0000000000000000000000000000000000034
:10FCD0000000000000000000000000000000000024
:10FCE0000000000000000000000000000000000014
:10FCF0000000000000000000000000000000000004
:10FD000000000000000000000000000000000000F3
:10FD100000000000000000000000000000000000E3
:10FD200000000000000000000000000000000000D3
:10FD300000000000000000000000000000000000C3
:10FD400000000000000000000000000000000000B3
:10FD500000000000000000000000000000000000A3
:10FD60000000000000000000000000000000000093
:10FD70000000000000000000000000000000000083
:10FD800000000000F8B500BFF8BC08BC9E467047F4
:10FD9000350400005D6300004185000045860000D9
:08FDA00049870000818A000080
:10FDA800000000000C0A04003498FF1F080000003F
:10FDB800FFFFFFFF1201000202000040C01683048B
:10FDC80000010102030118035400650065006E007C
:10FDD800730079006400750069006E006F00090205
:10FDE8004300020100C032090400000102020100C0
:10FDF800052400100105240101010424020605243C
:10FE08000600010705820310004009040100020AE8
:10FE180000000007050302400000070584024000B7
:10FE280000001603550053004200200053006500EF
:10FE38007200690061006C00040309040C030000EF
:10FE480000000000000000000000000000000000AA
:10FE5800000001000000000024FD000044FD000037
:10FE680064FD000000000000000000000000000029
:10FE780000000000E8FB0000000000000000000097
:10FE8800000000000000000000000000000000006A
:10FE9800000000000000000000000000000000005A
:10FEA800000000000000000000000000000000004A
:0CFEB800000000001488FF1F23FC000065
:00000001FF
